:020000040000FA
:100000000848040001000000F81F0000F81F00006D
:10001000F81F0000F81F0000F81F0000F81F000084
:10002000F81F0000F81F0000F81F0000F81F000074
:10003000F81F00001AE50000F81F0000F81F00007C
:10004000F81F000040E5000066E50000F81F000012
:10005000F81F0000F81F0000F81F0000F2BD0000AC
:10006000F81F0000F81F00002AD700002AD2000065
:10007000F81F000072EB0000DEE80000F81F00002F
:10008000F81F0000DCE90000F81F0000F81F000066
:10009000F81F00009AE50000C0E5000020E900001C
:1000A000F81F0000F81F0000F81F0000F81F0000F4
:1000B000F81F0000F81F0000F81F0000F81F0000E4
:1000C000F81F0000F81F0000F81F0000F81F0000D4
:1000D000F81F0000F81F000036A40000F81F000001
:1000E000F81F0000F81F0000F81F0000B0D7000044
:1000F000C0D20000F81F0000F81F00004AEB00000B
:100100005AE80000F81F0000F81F0000F81F000068
:10011000F81F0000F81F0000F81F0000F81F000083
:10012000F81F0000F81F0000F81F0000F81F000073
:10013000F81F0000F81F0000F81F0000F81F000063
:10014000F81F0000F81F000036EB0000F81F000049
:10015000F81F0000F81F0000F81F0000F81F000043
:10016000F81F0000F81F0000F81F0000F81F000033
:10017000F81F0000F81F000032D8000056D300001E
:100180004EE00000F81F0000F81F0000F81F0000FC
:10019000F81F0000F81F0000F81F0000F4E5000041
:1001A000F81F0000F81F0000F81F0000F81F0000F3
:1001B000F81F0000F81F0000F81F0000F81F0000E3
:1001C000F81F0000F81F0000F81F0000F81F0000D3
:1001D000F81F0000F81F0000F81F0000F81F0000C3
:1001E000F81F0000F81F0000F81F0000F81F0000B3
:1001F000F81F0000F81F0000F81F0000F81F0000A3
:100200000000000000000000F81F0000F81F0000C0
:10021000F81F0000F81F0000F81F0000F81F000082
:10022000F81F0000F81F0000F81F0000F81F000072
:10023000F81F00001AE50000F81F0000F81F00007A
:10024000F81F000040E5000066E50000F81F000010
:10025000F81F0000F81F0000F81F0000F2BD0000AA
:10026000F81F0000F81F00002AD700002AD2000063
:10027000F81F000072EB0000DEE80000F81F00002D
:10028000F81F0000DCE90000F81F0000F81F000064
:10029000F81F00009AE50000C0E5000020E900001A
:1002A000F81F0000F81F0000F81F0000F81F0000F2
:1002B000F81F0000F81F0000F81F0000F81F0000E2
:1002C000F81F0000F81F0000F81F0000F81F0000D2
:1002D000F81F0000F81F000036A40000F81F0000FF
:1002E000F81F0000F81F0000F81F0000B0D7000042
:1002F000C0D20000F81F0000F81F00004AEB000009
:100300005AE80000F81F0000F81F0000F81F000066
:10031000F81F0000F81F0000F81F0000F81F000081
:10032000F81F0000F81F0000F81F0000F81F000071
:10033000F81F0000F81F0000F81F0000F81F000061
:10034000F81F0000F81F000036EB0000F81F000047
:10035000F81F0000F81F0000F81F0000F81F000041
:10036000F81F0000F81F0000F81F0000F81F000031
:10037000F81F0000F81F000032D8000056D300001C
:100380009E480100F81F0000F81F0000F81F000041
:10039000F81F0000F81F0000F81F0000F4E500003F
:1003A000F81F0000F81F0000F81F0000F81F0000F1
:1003B000F81F0000F81F0000F81F0000F81F0000E1
:1003C000F81F0000F81F0000F81F0000F81F0000D1
:1003D000F81F0000F81F0000F81F0000F81F0000C1
:1003E000F81F0000F81F0000F81F0000F81F0000B1
:1003F000F81F0000F81F0000F81F0000F81F0000A1
:1004000000480400010000002F412300607D24000B
:1004100000018800000000000B00070020D42A0023
:100420000100200010000700000020000000E00094
:100430000200320000000200000000007CB2020056
:10044000000000000000FE004440A900408421009C
:100450000000E0000300320000002000A00188003E
:100460004440A80000000600F8FF2000591C2100AD
:1004700091018800800078000000EB001A0037002E
:100480008180E80032A0B4009101BA00E28040000F
:1004900032A0B4009102BA00E280400032A0B40061
:1004A0000002EB00472BDE00F507B200602CE100F4
:1004B00009003A00330007000700E00002003200A4
:1004C0000059EB00010037000201E8008301E90058
:1004D000F8FF3E00040037006128E100010032000F
:1004E0000082EB00040007001101BA000200E000E6
:1004F000E3FF3A0000000600220007000700E000CA
:10050000020032003159BA00020037008100E800D1
:100510000201E8008301E90017003200190007001A
:100520000700E000020032002159BA000200370043
:100530008100E9000201E8008301E9000D003200BA
:100540000400E00003003A00E280400032A0B40062
:10055000E9FF37000B0007000700E000020032004F
:1005600011D9BA00010037000201E8008301E90057
:10057000F5FF3A008100E800E180400032A0B400BD
:10058000000006000810E600020037000910E6002F
:10059000020037008083EB00000006008003EB00C0
:1005A0000000060091018800800078000000EB0048
:1005B00015003700E280400032A0B4009101BA007B
:1005C000E280400032A0B4009102BA00E280400014
:1005D00032A0B4000002EB00472BDE00F507B200AA
:1005E000602CE10004003A000059EB008301E900AF
:1005F000FDFF3E00040037006128E10001003200E9
:100600000082EB00040007001101BA000200E000C4
:10061000E8FF3A00000006003159BA008301E90002
:100620000C0032002159BA008301E90008003200B1
:100630000400E00003003A00E280400032A0B40071
:10064000F5FF370011D9BA008301E900FAFF3A003B
:100650008100E800E180400032A0B4000000060004
:1006600052800400000000006881040000000000C7
:10067000B8EB04000000000086C704000000000082
:1006800048D104000000000024E404000000000041
:100690006EB4040000000000CEA5040000000000BD
:1006A000A2A90400000000009EA9040000000000B0
:1006B00044AA04000000000012AA04000000000088
:1006C000A6A9040000000000AC6A040000000000BD
:1006D000DE6A0400000000000E6B04000000000051
:1006E000506B040000000000946B04000000000048
:1006F000D86B0400000000001A6C04000000000029
:10070000866C040000000000CE6C040000000000B5
:10071000166D040000000000726D0400000000006F
:10072000E86D040000000000646E0400000000009A
:10073000B86E040000000000D46E04000000000049
:10074000666F040000000000B26F040000000000AB
:10075000EE6F0400000000002A700400000000009A
:10076000DE700400000000000672040000000000BB
:1007700026900400000000009A9004000000000091
:100780005A90040000000000DA900400000000000D
:100790001A910400000000006091040000000000B5
:1007A000EC910400000000005092040000000000E2
:1007B0001E920400000000003894040000000000B5
:1007C0008292040000000000E0920400000000009B
:1007D0009493040000000000CA930400000000008D
:1007E000E6930400000000000294040000000000F2
:1007F0006A94040000000000A294040000000000BD
:10080000BE940400000000002C95040000000000CD
:100810005E950400000000009095040000000000B8
:1008200036B2040000000000C0B104000000000067
:10083000F0B00400000000000AB104000000000055
:100840005CB10400000000004EDA0400000000006B
:1008500032BD040000000000839F68000100E0003A
:1008600002003D0060001000E08018000300E0007E
:1008700002003D0060011100E08119000D00070039
:100880004F00E00002003B0060001000E080180014
:100890000000060080017800110009008280D80065
:1008A0008001FD00110009004288D8008300780013
:1008B000000006006022B800060220000000D00000
:1008C0008180D2000482D2008582D2000000A00084
:1008D0000202520083825A000300310002024200E9
:1008E00083824A000000A1000603E900F3FF3A00FA
:1008F00000000600020AB900001BB9000200B8009F
:10090000810042008100430000000600889FBE0075
:100910008A9FBE003004BE002005BE0004044400CF
:1009200085844C0006054D0087854D000898BE0063
:100930000A90BE000440E10005C8E10006D0E100D5
:1009400007D8E10002003100680040001008E8000C
:100950004F05BE004F04BE0000000600889FBE0089
:100960008A9FBE008C1F7800000678003C04BE0001
:100970002C05BE000400540085805C0006015D006B
:1009800087815D00009EBE00029EBE001000200018
:100990000440E10005C8E10006D0E10007D8E1000D
:1009A000010039000000EB001C0E10004F0678001B
:1009B0004F05BE004F04BE00000006001200FA0002
:1009C000889FBE008A9FBE008C9FBE000205BE00AD
:1009D0000004BE00E4B79F00F5B79F0086BF9F00EC
:1009E00097BF9F000000EB00D0B79F00C0B79F00EB
:1009F000B0B79F00A0B79F0090B79F000006780097
:100A0000FD032000DFB197004FB097000381410044
:100A1000BFB09700E08F510004003D00290007009F
:100A20007E805700B9FF070003003700250007004C
:100A30007E805700C9FF0700DFB09700E08F5000AD
:100A40000700350014002000050020006033B800C6
:100A500008047200898472000A0573008B85730094
:100A60000C06E8008D0F5600E6FF3400E08F5000C2
:100A700006003D006FB29700FFB297000FBB9700D2
:100A80009FBB97007E805700A0FF07005FA89700DC
:100A9000E00F500004003A001FB49700AFB4970075
:100AA0003FB59700CFB597000800BE000A01BE0011
:100AB0004F06BE004F05BE004F04BE000080FA0086
:100AC00000000600CF01DE0002817100B2B79F0076
:100AD0004F09DE000000400000007100A0B79F0039
:100AE0000FB097004F01DE0081804000810071004F
:100AF00091B79F007FAA9700CF20DE000000400042
:100B00000080700080B79F000800BE000A01BE0090
:100B10004F18DE000402420000027200F4AF9F0092
:100B20000804440089844C000A054D008B854D0063
:100B30004FB29700DFB297006FB39700FFB39700F3
:100B400000000600881F780018002000881F780029
:100B50009AFF07008F87E9004F0478000000060025
:100B6000801FEB0095FF07008F87E900000006005B
:100B7000889FBE008A9FBE008C1F7800E00F500047
:100B8000E08F5800E00F5900E08F59000F003D0042
:100B90006044B8006055B8000000540081805C00DB
:100BA00002015D0083815D001C0020000820E1003F
:100BB00009A8E1000AB0E1000BB8E1000D003D001A
:100BC000190007000006EB000A0037000006EB00E2
:100BD000E00F5200E08F5A00E00F5B00E08F5B00F7
:100BE00004003D006044B8006055B8000E000700E6
:100BF0001C002000D3FF0700E00F56000600320063
:100C00006022B8006033B8000000520081805A00B2
:100C100002015B0083815B004F0678004F05BE0038
:100C20004F04BE00000006000402540085825C00F0
:100C300006035D0087835D0000000600889FBE00FC
:100C40008A9FBE008C1F7800E00F5000E08F580094
:100C5000E00F5900E08F59000D003D006044B800DE
:100C60006055B8000000540081805C0002015D0006
:100C700083815D001C0020000820E10009A8E1003C
:100C80000AB0E1000BB8E1000D003D00080037009C
:100C90000006EB00E00F5200E08F5A00E00F5B000F
:100CA000E08F5B0006003D006044B8006055B8006E
:100CB0000402540085825C0006035D0087835D00AA
:100CC000A7FF0700E00F5600060032006022B800C0
:100CD0006033B8000000520081805A0002015B00BE
:100CE00083815B004F0678004F05BE004F04BE00B5
:100CF00000000600889FBE008A9FBE008C1F7800FF
:100D00000006EB00E00F5000E08F5800E00F5900A4
:100D1000E08F590007003D006044B8006055B800FE
:100D20000000540081805C0002015D0083815D0051
:100D30001C002000E00F5200E08F5A00E00F5B0023
:100D4000E08F5B0007003D006044B8006055B800CC
:100D50000402540085825C0006035D0087835D0009
:100D60000C00A2000C000700E00F56000600320045
:100D70006022B8006033B8000000520081805A0041
:100D800002015B0083815B004F0678004F05BE00C7
:100D90004F04BE0000000600889FBE008A9FBE0070
:100DA0008C9FBE000404B8000506B8008904460004
:100DB00060854E000606B8000A054600E0854E0034
:100DC0000706B8008B054600040EB80089044600EB
:100DD0000A854E00E0854D00050EB8000A05460064
:100DE0008B854E00060EB8008B0546000416B80031
:100DF0000A0546008B854E000516B8008B05460097
:100E0000041EB8008B0546000800BE000A01BE00A3
:100E10004F06BE004F05BE004F04BE000000060096
:100E2000E68747008E1F7800D0BF9F006687570077
:100E3000012F78000E003700DFB9970013417800CA
:100E40006FB8970090407800814F51000400320045
:100E50000280FB008180FB00010050000800370089
:100E60008301E800D3BF9F00000FE8000401780071
:100E70000202E900E00F5100EFFF3A0002007800A3
:100E80004F0778006F00B100000006008001780075
:100E900002003700B1597800040178000202E9002D
:100EA000E00F5100FBFF3A000000060080017800CF
:100EB0000200370081597800040178000202E9003D
:100EC000E00F5100FBFF3A000000060080007800B0
:100ED0000041EB00B14F1100FDFF3A000080EA0035
:100EE00000804000000006006D6100007468000092
:100EF0002E6300006F70000079000000636F000037
:100F000070690000657300002073000072630000C8
:100F1000207400006F2000006465000073740000FE
:100F2000206500006C6500006D6500006E740000B7
:100F30002062000079200000656C0000656D0000F3
:100F4000656E0000740000006465000073740000AA
:100F5000007300007263000000000000748700004E
:100F60007E870000FFFF0000A4870000FFFF000055
:100F7000A987000000000000000000006D61000073
:100F8000746800002E660000696C00006C000000B0
:100F9000666900006C6C000073200000646500004E
:100FA000737400002077000069740000682000005E
:100FB000636F00006E730000746100006E740000C7
:100FC00020760000616C000075650000007600006E
:100FD000616C00007565000000000000BE87000025
:100FE000C8870000FFFF0000A48700000100000088
:100FF000E787000000000000000000006D610000B5
:10100000746800002E6100006464000073630000D7
:10101000616C000061720000006100006464000007
:1010200020730000636100006C610000722000000A
:10103000746F0000206500006163000068200000FC
:10104000656C0000656D0000656E00007420000096
:101050006F660000207300007263000020610000D2
:101060006E64000020730000746F00007265000061
:101070002072000065730000756C00007420000091
:10108000746F0000206400006573000074000000AD
:1010900073630000616C00006172000000000000DA
:1010A000FE8700000D880000FFFF0000A4870000FD
:1010B000FFFF0000A9870000010000004888000031
:1010C00000000000000000006D6100007468000076
:1010D0002E61000064640000006100006464000090
:1010E0007320000073720000633100002061000073
:1010F0006E64000020730000726300003220000064
:10110000746F00002064000065730000742C000000
:10111000206500006C6500006D6500006E740000C5
:101120002062000079200000656C0000656D000001
:10113000656E0000740000007372000063310000EF
:101140000073000072630000320000006488000039
:101150006D880000FFFF0000A4870000FFFF000073
:101160009C880000FFFF0000A18800000000000034
:10117000000000006D610000746800002E73000024
:101180007562000000730000756200007374000057
:10119000726100006374000073200000737200002D
:1011A0006332000020660000726F00006D200000B6
:1011B0007372000063310000207400006F20000093
:1011C00064650000737400002C200000656C000052
:1011D000656D0000656E00007420000062790000FB
:1011E000206500006C6500006D6500006E740000F5
:1011F00000000000BA880000C3880000FFFF000064
:10120000A4870000FFFF00009C880000FFFF000093
:10121000A188000000000000000000006D610000D7
:10122000746800002E6D0000756C0000006D0000F9
:10123000756C000074690000706C00006965000046
:101240007320000073720000633100002061000011
:101250006E64000020730000726300003220000002
:10126000746F00002064000065730000742C00009F
:10127000206500006C6500006D6500006E74000064
:101280002062000079200000656C0000656D0000A0
:10129000656E0000740000000E89000017890000D0
:1012A000FFFF0000A4870000FFFF00009C880000F3
:1012B000FFFF0000A1880000000000000000000007
:1012C0006D610000746800002E6400006976000003
:1012D0000064000069760000696400006573000026
:1012E000207300007263000031200000627900006A
:1012F000207300007263000032200000746F000051
:101300002064000065730000742C0000206500005C
:101310006C6500006D6500006E74000020620000C6
:1013200079200000656C0000656D0000656E0000AE
:10133000740000006089000069890000FFFF000060
:10134000A4870000FFFF00009C880000FFFF000052
:10135000A188000000000000000000006D61000096
:10136000746800002E6D0000696E000000770000B8
:10137000726900007465000073200000746800004A
:10138000652000006D6900006E6900006D75000049
:101390006D2000006F660000207300007263000083
:1013A00031200000616E00006420000073720000B4
:1013B00063320000207400006F20000064650000AC
:1013C000737400002C200000656C0000656D000047
:1013D000656E000074200000627900002065000046
:1013E0006C6500006D6500006E7400000000000078
:1013F000AE890000B7890000FFFF0000A48700004D
:10140000FFFF00009C880000FFFF0000A188000093
:1014100000000000000000006D6100007468000022
:101420002E6D0000617800000077000072690000F6
:1014300074650000732000007468000065200000DF
:101440006D610000786900006D7500006D2000007E
:101450006F660000207300007263000031200000FE
:10146000616E0000642000007372000063320000AF
:10147000207400006F200000646500007374000099
:101480002C200000656C0000656D0000656E00009A
:101490007420000062790000206500006C65000087
:1014A0006D6500006E740000000000000C8A0000F2
:1014B000158A0000FFFF0000A4870000FFFF000066
:1014C0009C880000FFFF0000A188000000000000D1
:1014D000000000006D610000746800002E630000D1
:1014E0006C6100006D700000006300006C61000022
:1014F0006D70000020730000726300002074000013
:101500006F2000006C6F0000772F000068690000FA
:1015100067680000206200006F7500006E640000C4
:1015200073200000696E0000746F000020640000EA
:1015300065730000742C0000206500006C650000DD
:101540006D6500006E7400002062000079200000CC
:10155000656C0000656D0000656E000074000000A1
:101560006C6F000077000000686900006768000089
:10157000000000006A8A0000758A0000FFFF00007A
:10158000A4870000FFFF0000A9870000FFFF000004
:10159000B08A0000FFFF0000B48A000000000000D5
:1015A000000000006D610000746800002E640000FF
:1015B0006F7400000077000072690000746500001D
:1015C000732000007468000065200000646F000054
:1015D00074200000707200006F64000075630000EA
:1015E000742000006F66000020730000726300002A
:1015F00031200000616E0000642000007372000062
:1016000063320000207400006F2000006465000059
:10161000737400002C2000006166000074650000F7
:1016200072200000612000007368000069660000FD
:101630007400000073680000696600007400000018
:10164000D28A0000DB8A000001000000A4870000AD
:10165000FFFF00009C880000FFFF0000A188000041
:10166000010000001A8B00000000000000000000D4
:101670006D610000746800002E730000746100004A
:101680007400000070650000726600006F72000058
:101690006D73000020730000746100007469000025
:1016A0007374000069630000732000006F6E000017
:1016B0002073000072630000006D0000696E00007E
:1016C000006D000061780000006D000065610000A1
:1016D0006E000000388B0000428B0000FFFF00000E
:1016E000A9870000010000005D8B000001000000E0
:1016F000618B000001000000658B0000000000000D
:10170000000000006D610000746800002E610000A0
:1017100072670000626F0000756E00006473000065
:101720000067000065740000207400006865000018
:10173000206900006E6400006963000065730000AA
:101740002028000061720000676D0000696E0000D3
:101750002C20000061720000676D000061780000BD
:10176000292000006F6600002074000068650000FA
:10177000206C0000696D0000697400002076000094
:10178000616C000075650000732000006F6600004A
:1017900020730000726300000061000072670000A7
:1017A0006D6900006E00000061720000676D00004E
:1017B0006178000000000000828B0000918B000027
:1017C000FFFF0000A987000001000000CD8B000092
:1017D00001000000D48B00000000000000000000A9
:1017E0006D610000746800002E7300006F720000CD
:1017F00074000000736F000072740000206100002C
:101800007272000061790000206900006E20000003
:10181000706C0000616300006500000061720000F0
:101820007261000079000000F08B0000FA8B00006C
:10183000FFFF00000E8C0000000000000000000010
:101840006D610000746800002E6D0000756C000072
:101850006469000076000000706500007266000098
:101860006F7200006D73000020640000657300005B
:10187000742000003D200000286100002A62000062
:10188000292F000063200000696E00002033000053
:1018900032200000626900007473000020650000BF
:1018A0006C6500006D6500006E7400002062000031
:1018B00079200000656C0000656D0000656E000019
:1018C000740000006100000062000000630000007E
:1018D000208C00002C8C0000FFFF0000A48700007B
:1018E000FFFF0000628C0000FFFF0000648C00001E
:1018F000FFFF0000668C00000000000000000000F8
:101900006D610000746800002E61000074610000C9
:101910006E3200000070000065720000666F00000B
:10192000726D000073200000646500007374000095
:10193000203D000020610000746100006E32000054
:10194000287900002C78000029200000656C000038
:10195000656D0000656E0000742000006279000073
:10196000206500006C6500006D6500006E7400006D
:10197000007900000078000000000000808C00006A
:101980008B8C0000FFFF0000A4870000FFFF000019
:10199000B98C0000FFFF0000BB8C000000000000BD
:1019A000000000006D610000746800002E730000EC
:1019B000696E00000070000065720000666F000034
:1019C000726D0000732000006465000073740000F5
:1019D000203D000020730000696E000028780000A0
:1019E00029200000656C0000656D0000656E000038
:1019F0007420000062790000206500006C65000022
:101A00006D6500006E74000000000000D28C0000C4
:101A1000DB8C0000FFFF0000A4870000FFFF000038
:101A2000BB8C000000000000000000006D610000A1
:101A3000746800002E6300006F73000000700000E7
:101A400065720000666F0000726D00007320000078
:101A50006465000073740000203D000020630000F6
:101A60006F7300002878000029200000656C0000DA
:101A7000656D0000656E0000742000006279000052
:101A8000206500006C6500006D6500006E7400004C
:101A900000000000168D00001F8D0000FFFF0000F9
:101AA000A4870000FFFF0000BB8C000000000000C6
:101AB000000000006D610000746800002E720000DC
:101AC0006F74000032000000726F0000746100004B
:101AD0007465000073200000762000006F6600002F
:101AE000206100006E6700006C650000206100004E
:101AF000207400006F200000646500007374000013
:101B000000760000000000005A8D0000648D000087
:101B100002000000A487000002000000818D000088
:101B200001000000628C00000000000000000000C6
:101B30006D610000746800002E7300007172000077
:101B40007400000070650000726600006F72000093
:101B50006D730000206400006573000074200000B5
:101B60003D200000737100007274000028780000AE
:101B700029200000656C0000656D0000656E0000A6
:101B80007420000062790000206500006C65000090
:101B90006D6500006E74000000000000988D00006C
:101BA000A28D0000FFFF0000A4870000FFFF0000DF
:101BB000BB8C000000000000000000006D61000010
:101BC000746800002E6E00007A73000065710000DA
:101BD0000077000072690000746500002074000046
:101BE0006F20000064650000737400002074000022
:101BF00068650000206D000069640000646C0000EE
:101C000065200000696E0000646500007820000017
:101C10006F6600002074000068650000206C000002
:101C2000617200006765000073740000207300009B
:101C300065710000756500006E630000652000009E
:101C40006F660000206E00006F6E00002D7A0000AD
:101C5000657200006F200000656C0000656D00007B
:101C6000656E00007473000020660000726F000053
:101C70006D20000073720000632C0000202D000016
:101C80003120000069660000206E00006F740000C3
:101C9000206600006F7500006E640000206F000079
:101CA0007220000069660000207300006D61000072
:101CB0006C6C000065720000207400006861000018
:101CC0006E2000006D6900006E4C0000656E000023
:101CD00067740000680000006D6900006E4C000031
:101CE000656E00006774000068000000DE8D000073
:101CF000E98D000001000000A4870000FFFF000044
:101D0000A9870000010000006C8E000000000000A8
:101D1000000000006D610000746800002E72000079
:101D2000616E000064000000666900006C6C0000D9
:101D300020610000727200006179000020770000CD
:101D40006974000068200000726100006E64000089
:101D50006F6D000020760000616C0000756500006A
:101D6000730000008A8E0000948E0000FFFF0000C8
:101D7000A487000000000000000000000000000038
:101D80009301000024030000B7040000480600008F
:101D9000DA0700006B090000FC0A00008C0C000050
:101DA0001C0E0000AB0F00003B110000C812000029
:101DB00056140000E31500006E170000F91800002B
:101DC000831A00000C1C0000941D00001A1F000064
:101DD000A020000024220000A723000029250000E5
:101DE000A826000027280000A4290000202B0000BE
:101DF000992C0000122E0000872F0000FC300000FC
:101E00006F320000DF3300004E350000BA360000AC
:101E1000253800008D390000F33A0000573C0000DF
:101E2000B93D0000173F000074400000CE410000A3
:101E3000264300007B440000CD4500001D47000004
:101E40006A480000B4490000FC4A0000404C000011
:101E5000824D0000C04E0000FC4F000034510000D5
:101E6000695200009B530000CA540000F655000060
:101E70001E5700004358000064590000835A0000B8
:101E80009D5B0000B45C0000C85D0000D75E0000F0
:101E9000E45F0000EC600000F1610000F26200000D
:101EA000EF630000E9640000DE650000D06600001A
:101EB000BD670000A76800008C6900006E6A000022
:101EC0004B6B0000246C0000F96C0000CA6D000030
:101ED000976E00005F6F000023700000E370000049
:101EE0009E7100005572000008730000B673000078
:101EF0006074000005750000A575000042760000C2
:101F0000D97600006C770000FB7700008478000031
:101F1000097900008A790000067A00007D7A0000C5
:101F2000EF7A00005D7B0000C67B00002A7C000089
:101F3000897C0000E47C0000397D00008A7D00007F
:101F4000D77D00001D7E0000607E00009D7E0000A9
:101F5000D67E0000097F0000397F0000627F00000C
:101F6000877F0000A77F0000C27F0000D87F0000AD
:101F7000EA7F0000F67F0000FE7F0000FF7F000088
:101F80008C020000DF02000030030000800300002C
:101F9000D10300002204000073040000C20400000A
:101FA00014050000B305000054060000F10600000F
:101FB0008F0700002D080000CA0800006309000018
:101FC000FC090000340B00005C0C0000820D0000D6
:101FD000A40E0000BD0F0000D3100000E2110000AD
:101FE000E7120000EF140000CC1600009218000069
:101FF000401A0000D61B0000531D0000B51E000053
:102000000B200000792200008D2400006F260000C4
:102010001428000090290000E02A0000112C000084
:10202000252D0000052F000089300000D33100006D
:10203000EC320000DD330000AE34000067350000F4
:102040000D36000020370000FB370000B2380000DA
:102050004A390000CC3900003B3A00009B3A0000AE
:10206000F33A0000833B0000F43B0000513C0000C9
:102070009F3C0000E13C00001A3D00004B3D000089
:10208000783D0000C03D0000F93D0000283E000002
:102090004F3E0000703E00008D3E0000A53E000057
:1020A000BC3E0000E03E0000FD3E0000143F00008A
:1020B000283F0000383F0000473F0000533F00002A
:1020C0005E3F0000703F00007F3F00008A3F00003D
:1020D000943F00009C3F0000A43F0000AA3F000086
:1020E000AF3F0000B83F0000C03F0000C53F000008
:1020F000CB3F0000CE3F0000D23F0000D53F0000A4
:10210000D83F0000DC3F0000E03F0000E33F00005C
:10211000E53F0000E83F0000E93F0000EB3F000022
:10212000EC3F0000EE3F0000F13F0000F13F0000F7
:10213000F33F0000F43F0000F53F0000F53F0000D2
:10214000F73F0000F73F0000F93F0000F83F0000B4
:10215000FA3F0000FA3F0000FA3F0000FB3F00009A
:10216000FB3F0000FC3F0000FC3F0000FC3F000084
:10217000FE3F0000FD3F0000FD3F0000FD3F00006E
:10218000FE3F0000FE3F0000FE3F0000FE3F00005B
:10219000FE3F0000FE3F000000400000FF3F000047
:1021A000FF3F0000FF3F0000FF3F0000FF3F000037
:1021B000FF3F0000FF3F0000FF3F0000FF3F000027
:1021C000FF3F0000FF3F0000004000000040000013
:1021D00000400000004000000040000000400000FF
:1021E00000400000004000000040000000400000EF
:1021F00000400000004000000040000000400000DF
:10220000004000004164000064720000657300003B
:10221000732000006F750000742000006F660000DE
:102220002073000065740000746900006E67000090
:1022300073000000536C0000656500007020000012
:102240006D6F000064650000206E00006F74000078
:102250002073000075700000706F00007274000041
:102260006564000000450000727200006F7200009B
:102270003A2000006D6900006E2000003D3D000026
:102280002030000078460000464600004646000028
:102290004646000046200000210000004572000074
:1022A000726F0000723A0000205500006E6100005D
:1022B000626C000065200000746F00002066000062
:1022C0006C610000736800002062000079740000F7
:1022D000656300006F640000652000002831000085
:1022E000292000002100000045720000726F0000EC
:1022F000723A0000205500006E610000626C000020
:1023000065200000746F0000206600006C61000012
:1023100073680000206200007974000065630000AB
:102320006F640000652000002832000029200000B2
:102330002100000045720000726F0000723A000038
:10234000205500006E610000626C000065200000F6
:10235000746F0000206600006C610000736800006C
:102360002062000079740000656300006F64000063
:102370006520000028330000292000002100000013
:10238000466C000061730000686900006E67000021
:10239000204F00004B00000074680000796D0000C1
:1023A000696F00002D490000490000005F690000CE
:1023B0006400000065760000656E0000742E000069
:1023C000736F000075720000636500000065000017
:1023D000766500006E7400002E61000072670000D8
:1023E000730000005F6600007776000065720000F1
:1023F000736900006F6E0000005F000070720000E3
:102400006F64000075630000744900006400000000
:1024100062750000747400006F6E0000732E00007F
:102420005F720000617700000062000075740000B8
:10243000746F00006E2E000062610000636B00008C
:102440007761000072640000006200007574000093
:10245000746F00006E2E00006C6500006674000052
:102460000062000075740000746F00006E2E0000A2
:10247000636500006E740000657200000062000079
:1024800075740000746F00006E2E0000666F00000F
:102490007277000061720000640000006275000045
:1024A000747400006F6E00002E72000069670000F7
:1024B000687400000062000075740000746F000012
:1024C0006E7300002E5F00006D650000616E0000FD
:1024D0000062000075740000746F00006E730000ED
:1024E0002E5F00006E6F0000697300006500000041
:1024F000707200006F7800002E6800006F7200009C
:10250000697A00006F6E0000746100006C000000CA
:10251000707200006F7800002E6300006F6D000085
:102520006D2E0000727800002E5F000070610000C8
:10253000796C00006F61000064730000007000009F
:10254000726F0000782E0000636F00006D6D000058
:102550002E720000782E00005F6900006E7400008B
:10256000656E000073690000746900006573000007
:1025700000700000726F0000782E0000636F000092
:102580006D6D00002E720000780000007072000077
:102590006F7800002E6300006F6D00006D2E00004C
:1025A0007478000000700000726F0000782E000048
:1025B000677200006F7500006E6400002E610000FD
:1025C0006D620000696100006E7400000070000020
:1025D000726F0000782E0000677200006F750000B7
:1025E0006E6400002E720000656600006C650000DD
:1025F000637400006564000000700000726F0000EA
:10260000782E0000677200006F7500006E64000095
:102610002E640000656C000074610000006D000015
:102620006F7400006F7200002E6C00006566000081
:10263000742E000074610000726700006574000071
:10264000006D00006F7400006F7200002E720000B9
:1026500069670000687400002E7400006172000059
:1026600067650000740000005F7600006261000092
:10267000740000005F6900006D6F000074000000CE
:102680006D6F0000746F0000722E00006C6500001A
:10269000667400002E730000706500006564000021
:1026A000006D00006F7400006F7200002E72000059
:1026B00069670000687400002E73000070650000F8
:1026C00065640000006D00006F7400006F72000010
:1026D0002E6C000065660000742E0000707700000C
:1026E0006D0000006D6F0000746F0000722E00001E
:1026F0007269000067680000742E000070770000A7
:102700006D0000006163000063000000746500005C
:102710006D70000065720000617400007572000049
:102720006500000072630000352E00006164000047
:1027300064720000657300007300000072630000A3
:10274000352E0000636F00006D6D0000616E0000AB
:10275000640000006D690000632E0000696E0000D7
:10276000746500006E730000697400007900000059
:102770006D690000632E000074680000726500003F
:10278000736800006F6C0000640000006D69000059
:10279000632E00005F6D0000656100006E000000A8
:1027A000746900006D650000722E00007065000005
:1027B000726900006F640000006100006363000044
:1027C0002E5F00007461000070000000CC910000DA
:1027D00001000000D691000001000000DA91000025
:1027E00020000000E791000002000000F2910000CC
:1027F00001000000FD9100000500000008920000AB
:102800000100000015920000010000002592000068
:102810000100000031920000010000003F92000022
:10282000010000004E920000050000005B920000D5
:102830000500000069920000070000007892000087
:102840000700000088920000070000009F9200002F
:1028500001000000B992000001000000C6920000D3
:1028600002000000D392000002000000E792000086
:1028700002000000FD920000010000000F93000024
:1028800001000000219300000200000034930000CA
:10289000020000003A930000010000004093000095
:1028A000010000005193000001000000639300004C
:1028B00001000000729300000300000082930000FA
:1028C00001000000869300000100000092930000C8
:1028D000010000009E93000001000000AA93000088
:1028E00001000000B893000001000000C693000042
:1028F00002000000D093000001000000DD93000002
:102900000000000000000000DE000000AD0000003C
:10291000CA000000FE000000BE000000EF00000042
:1029200004000000020000009EA9000044AA00006C
:1029300012AA0000A6A90000AC6A0000DE6A00002E
:102940000E6B0000506B0000946B0000D86B000011
:102950001A6C0000866C0000CE6C0000166D000042
:10296000726D0000E86D0000646E0000B86E00003B
:10297000D46E0000666F0000B26F0000EE6F0000C2
:102980002A700000DE700000067200002690000031
:102990009A9000005A900000DA9000001A9100000E
:1029A00060910000EC910000509200001E92000027
:1029B0003894000082920000E0920000949300009E
:1029C000CA930000E6930000029400006A9400009D
:1029D000A2940000BE9400002C9500005E950000BB
:1029E0009095000036B2000042610000636B000069
:1029F00077610000726400002062000075740000BE
:102A0000746F00006E200000737400006174000099
:102A10007573000020630000686100006E670000AD
:102A200065640000004C0000656600007420000032
:102A300062750000747400006F6E00002073000067
:102A4000746100007475000073200000636800006A
:102A5000616E0000676500006400000043650000CF
:102A60006E74000065720000206200007574000042
:102A7000746F00006E200000737400006174000029
:102A80007573000020630000686100006E6700003D
:102A900065640000004600006F720000776100006E
:102AA000726400002062000075740000746F000002
:102AB0006E200000737400006174000075730000E4
:102AC00020630000686100006E670000656400001C
:102AD0000052000069670000687400002062000076
:102AE00075740000746F00006E20000073740000A5
:102AF00061740000757300002063000068610000CD
:102B00006E670000656400000062000075740000DC
:102B1000746F00006E7300000042000075740000C6
:102B2000746F00006E73000020760000616C00007E
:102B3000756500007320000075700000646100007E
:102B40007465000064000000707200006F7800007F
:102B500000500000726F0000786900006D6900008D
:102B60007479000020760000616C0000756500003B
:102B7000732000007570000064610000746500003F
:102B800064000000707200006F7800002E63000087
:102B90006F6D00006D000000446100007461000072
:102BA0002072000065630000656900007665000022
:102BB000642000006F6E0000207400006865000053
:102BC00020700000726F0000786900006D690000DD
:102BD00074790000206300006F6D00006D750000C7
:102BE0006E69000063610000746900006F6E000090
:102BF00000740000617000000041000020740000BB
:102C0000617000002069000073200000646500000E
:102C100074650000637400006564000000410000FA
:102C200063630000656C0000657200006F6D00005A
:102C3000657400006572000020760000616C000081
:102C4000756500007320000075700000646100006D
:102C500074650000640000006D69000063000000FE
:102C6000466900007265000064200000776800007B
:102C7000656E0000206D000069630000726F000047
:102C8000706800006F6E000065200000696E000033
:102C9000746500006E730000697400007920000004
:102CA0006973000020610000626F0000766500001B
:102CB000207400006872000065730000686F0000F7
:102CC0006C640000007300006F7500006E6400000B
:102CD0002E660000696E00006973000068650000E0
:102CE0006400000046690000726500006420000076
:102CF00077680000656E00002074000068650000C1
:102D0000207000006C6100007962000061630000C7
:102D10006B2000006F66000020610000207500003D
:102D20007365000072200000696E00006974000085
:102D3000696100007465000064200000736F00008A
:102D4000756E0000642000006973000020660000BA
:102D5000696E00006973000068650000640000008F
:102D6000546500006D700000657200006174000021
:102D70007572000065200000766100006C7500002F
:102D8000652000007570000064610000746500003B
:102D90006400000072630000350000005243000030
:102DA000352000006D65000073730000616700004E
:102DB0006520000072650000636500006976000010
:102DC00065640000006D00006F7400006F72000009
:102DD000004D00006F7400006F720000207400004E
:102DE000696D00006572000000740000696D0000EC
:102DF0006572000030000000546900006D6500003D
:102E00007220000030000000746900006D65000051
:102E10007231000000540000696D0000657200000E
:102E2000203100000000000015920000F494000022
:102E30002592000013950000319200002E950000AD
:102E40003F9200004B9500004E92000069950000F3
:102E5000859500008D950000A4950000A9950000BF
:102E6000C2950000CC950000F9950000FD9500008A
:102E7000829300000F9600002C9600003096000010
:102E8000639600007296000086930000B0960000E2
:102E9000CA960000CE960000E3960000E996000076
:102EA000F5960000FC960000049700000B970000C8
:102EB00000000000000000005F7300007973000054
:102EC000746500006D2E000072650000626F0000E6
:102ED0006F74000000520000656200006F6F000018
:102EE0007420000074680000652000006D69000017
:102EF000637200006F6300006F6E00007472000068
:102F00006F6C00006C650000720000005F730000D1
:102F100079730000746500006D2E00007365000079
:102F200074740000696E0000677300002E72000068
:102F300065610000640000005265000061640000EB
:102F400020610000207300006574000074690000B7
:102F50006E6700000061000064640000726500009C
:102F60007373000000760000616C0000756500005E
:102F7000005F00007379000073740000656D00004D
:102F80002E73000065740000746900006E67000015
:102F9000732E000077720000697400006500000065
:102FA0005772000069740000652000006120000075
:102FB0007365000074740000696E00006700000013
:102FC0005F73000079730000746500006D2E0000CF
:102FD0007365000074740000696E00006773000080
:102FE0002E6600006C61000073680000005700004E
:102FF00072690000746500002074000068650000BC
:103000002073000065740000746900006E670000A2
:1030100073200000696E0000746F000020660000DD
:103020006C61000073680000000000004572000041
:10303000726F0000723A000020730000616D0000A2
:10304000706C000065730000206D00007573000057
:103050007420000062650000206900006E200000FE
:103060005B2D000031320000382C000031320000AE
:10307000375D000020720000616E0000676500008F
:10308000005F00006C650000647300002E73000098
:103090006574000000530000657400002074000097
:1030A00068650000206C000065640000006C000092
:1030B000656400000062000072690000676800003B
:1030C000746E00006573000073000000736F0000F1
:1030D000756E0000642E000072650000636F0000D2
:1030E00072640000005300007461000072740000FC
:1030F00020720000656300006F72000064690000C8
:103100006E670000206F000066200000724E000015
:103110002E77000061760000004E00000073000072
:103120006F7500006E6400002E7000006C6100007E
:1031300079000000537400006172000074200000E8
:10314000706C00006179000062610000636B000038
:10315000206F000066200000704E00002E770000F7
:1031600061760000007300006F7500006E6400005F
:103170002E720000657000006C6100007900000094
:10318000537400006172000074200000706C000035
:103190006179000062610000636B0000206F000035
:1031A00066200000724E00002E770000617600005D
:1031B000007300006F7500006E6400002E73000045
:1031C00079730000746500006D0000005374000006
:1031D0006172000074200000706C000061790000D2
:1031E00062610000636B0000206F00006620000039
:1031F0007379000073740000656D00002073000097
:103200006F7500006E640000204E0000006C00002E
:1032100065640000732E00006369000072630000A3
:103220006C6500000053000065740000206300001E
:1032300069720000637500006C610000722000007C
:10324000726900006E670000206C00006564000079
:10325000730000006C300000006C000031000000C2
:103260006C320000006C0000330000006C34000081
:10327000006C0000350000006C360000006C00009F
:10328000370000006C650000647300002E740000BD
:103290006F700000005300006574000020520000B1
:1032A00047420000207400006F700000206C000096
:1032B00065640000007200006564000000670000A3
:1032C00072650000656E0000006200006C75000011
:1032D000650000006C650000647300002E62000051
:1032E0006F740000746F00006D2E000072690000A2
:1032F000676800007400000053650000742000003F
:103300005247000042200000626F0000746F00000E
:103310006D200000726900006768000074200000E2
:103320006C650000640000006C65000064730000C0
:103330002E6200006F740000746F00006D2E00009C
:103340006C650000667400000053000065740000A6
:103350002052000047420000206200006F7400000D
:103360006F6D0000206C0000656600007420000096
:103370006C650000640000006C6500006473000070
:103380002E62000075740000746F00006E73000000
:103390000053000065740000206200007574000096
:1033A000746F00006E730000206C00006564000004
:1033B000730000006C650000647300002E70000054
:1033C000726F0000782E0000680000005365000056
:1033D00074200000686F0000726900007A6F0000BE
:1033E0006E740000616C000020700000726F0000BD
:1033F000786900006D69000074790000206C00009D
:1034000065640000730000006C65000064730000D8
:103410002E700000726F0000782E00007600000011
:10342000536500007420000076650000727400008F
:1034300069630000616C000020700000726F000082
:10344000786900006D69000074790000206C00004C
:1034500065640000730000006C6500006473000088
:103460002E7200006300000053650000742000000D
:1034700072630000206C000065640000006C0000B6
:1034800065640000732E0000736F0000756E00000D
:10349000640000005365000074200000736F00009A
:1034A000756E0000642000006C6500006400000080
:1034B0006C650000647300002E740000656D0000F0
:1034C0007065000072610000747500007265000094
:1034D0000053000065740000206E0000746300005B
:1034E000206C000065640000007300006F75000030
:1034F0006E6400002E66000072650000710000001E
:10350000506C0000617900002066000072650000C8
:1035100071750000656E00006379000000480000CE
:103520007A00000064730000007300006F750000F3
:103530006E6400002E7700006176000065000000D8
:1035400053650000742000007468000065200000CE
:1035500070720000696D0000617200007920000047
:103560007761000076650000206F00006620000093
:103570007468000065200000746F00006E65000034
:1035800020670000656E0000657200006174000035
:103590006F72000000770000617600006500000097
:1035A000707200006F7800002E6300006F6D0000E5
:1035B0006D2E0000656E0000616200006C65000009
:1035C000004500006E610000626C00006520000094
:1035D0006F720000206400006973000061620000E7
:1035E0006C65000020740000686500002070000019
:1035F000726F0000786900006D6900007479000046
:10360000206300006F6D00006D7500006E690000A2
:1036100063610000746900006F6E000000730000B9
:10362000746100007465000000730000642E0000E7
:103630006F700000656E0000004F000070650000B4
:103640006E20000061200000666900006C650000CB
:10365000206F00006E2000007468000065200000EC
:103660005344000020630000617200006400000009
:103670006E7500006D62000065720000007300004E
:103680007461000074750000730000007364000032
:103690002E7700007269000074650000005700007A
:1036A000726900007465000020640000617400000D
:1036B00061200000746F0000207400006865000045
:1036C000206F0000706500006E650000642000003F
:1036D000666900006C650000006400006174000011
:1036E00061000000777200006974000074650000DA
:1036F0006E000000736400002E720000656100001F
:103700006400000052650000616400002064000055
:103710006174000061200000667200006F6D00009F
:103720002074000068650000206F000070650000D4
:103730006E65000064200000666900006C65000092
:103740000072000065610000640000007364000006
:103750002E730000656500006B00000053650000DB
:10376000656B00002074000068650000206F000099
:10377000706500006E65000064200000666900004E
:103780006C650000007000006F7300006974000039
:10379000696F00006E000000733000002E7700009B
:1037A0006176000000730000322E00007761000097
:1037B00076000000733300002E7700006176000071
:1037C00000730000342E00007761000076000000D6
:1037D000733500002E770000617600000073000052
:1037E000362E00007761000076000000733700007D
:1037F0002E7700006176000000000000480D0000F8
:103800000D0000003011000007000000EC13000064
:10381000070000000019000007000000781E0000EB
:10382000070000000000000000000000781E0000FB
:103830000D0000000019000007000000EC1300005C
:10384000070000003011000007000000480D0000D4
:103850000700000000000000000000004C04000011
:1038600007000000980800000700000000000000AA
:1038700000000000E40C0000070000003011000010
:103880000D000000C8190000070000000000000043
:10389000000000009C27000002000000AB22000096
:1038A000010000009D1C000002000000FB18000049
:1038B000020000002D32000001000000322D000047
:1038C000010000004628000002000000E826000079
:1038D00001000000BF22000002000000FB180000F1
:1038E00002000000FF32000001000000C6200000BE
:1038F00001000000762F0000020000002C2E0000C6
:1039000001000000CE2C000001000000FD39000085
:10391000020000000000000000000000C8190000C4
:1039200005000000BE0A00000400000000000000C6
:103930000000000030110000070000007C150000AE
:10394000070000000000000000000000301100002F
:10395000070000007C15000007000000C8190000E7
:10396000070000000000000000000000222A000004
:103970002B2C00003A3B00003C3D00003E3F000085
:103980005B5D00007C7F0000008000009A900000DA
:10399000418E0000418F0000804500004545000039
:1039A00049490000498E00008F900000929200006B
:1039B0004F9900004F55000055590000999A00009A
:1039C0009B9C00009D9E00009F410000494F00000D
:1039D00055A50000A5A60000A7A80000A9AA000000
:1039E000ABAC000021AE0000AFB00000B1B20000EF
:1039F000B3B40000B5B60000B7B80000B9BA000013
:103A0000BBBC0000BDBE0000BFC00000C1C20000C2
:103A1000C3C40000C5C60000C7C80000C9CA000072
:103A2000CBCC0000CDCE0000CFD00000D1D2000022
:103A3000D3D40000D5D60000D7D80000D9DA0000D2
:103A4000DBDC0000DDDE0000DFE00000E1E2000082
:103A5000E3E40000E5E60000E7E80000E9EA000032
:103A6000EBEC0000EDEE0000EFF00000F1F20000E2
:103A7000F3F40000F5F60000F7F80000F9FA000092
:103A8000FBFC0000FDFE0000FF0000002E2E0000E9
:103A90002F2E00002E2F0000446F000063750000E1
:103AA0006D6500006E740000732F0000436F00000E
:103AB000646500002064000073500000494300006A
:103AC0002F6D00006F6C00006F6C0000652F000010
:103AD00069320000632F000069320000635F00005C
:103AE00070720000697600002E680000002E000051
:103AF0002E2F00002E2E00002F4400006F630000C8
:103B0000756D0000656E0000747300002F430000A7
:103B10006F640000652000006473000050490000DD
:103B2000432F00006D6F00006C6F00006C6500009B
:103B30002F690000326300002F6D000061730000E8
:103B400074650000725F0000707200006F74000006
:103B50006F6300006F6C00002E6300000000000027
:103B60002E2E00002F2E00002E2F0000446F00008C
:103B7000637500006D6500006E740000732F000017
:103B8000436F000064650000206400007350000073
:103B9000494300002F6D00006F6C00006F6C000047
:103BA000652F000069320000632F000069320000B9
:103BB000635F000070720000697600002E680000EC
:103BC000002E00002E2F00002E2E00002F4400009B
:103BD0006F630000756D0000656E00007473000077
:103BE0002F4300006F640000652000006473000034
:103BF00050490000432F00006D6F00006C6F000003
:103C00006C6500002F690000326300002F6D00001A
:103C10006173000074650000722E000063000000F4
:103C20002E2E00002F2E00002E2F0000446F0000CB
:103C3000637500006D6500006E740000732F000056
:103C4000436F0000646500002064000073500000B2
:103C5000494300002F6D00006F6C00006F6C000086
:103C6000652F000069320000632F000069320000F8
:103C7000635F000070720000697600002E6800002B
:103C8000002E00002E2F00002E2E00002F440000DA
:103C90006F630000756D0000656E000074730000B6
:103CA0002F4300006F640000652000006473000073
:103CB00050490000432F00006D6F00006C6F000042
:103CC0006C6500002F690000326300002F73000054
:103CD0006C610000766500002E63000000000000AB
:103CE0002E2E00002F2E00002E2F0000446F00000B
:103CF000637500006D6500006E740000732F000096
:103D0000436F0000646500002064000073500000F1
:103D1000494300002F6D00006F6C00006F6C0000C5
:103D2000652F0000746900006D650000722F0000AF
:103D3000746900006D650000722E000063000000D1
:103D4000010000000000000008000000000000006A
:103D50004000000000000000000100000000000022
:103D60002E2E00002F2E00002E2F0000446F00008A
:103D7000637500006D6500006E740000732F000015
:103D8000436F000064650000206400007350000071
:103D9000494300002F6D00006F6C00006F6C000045
:103DA000652F000069320000632F000069320000B7
:103DB000635F000070720000697600002E680000EA
:103DC000000000002E2E00002F2E00002E2F0000DD
:103DD000446F0000637500006D6500006E740000A4
:103DE000732F0000436F0000646500002064000032
:103DF00073500000494300002F6D00006F6C0000FD
:103E00006F6C0000652F0000666C0000617300009D
:103E1000682F0000666C000061730000682E0000CF
:103E20006300000052490000464600000000000008
:103E3000000000005741000056450000666D00007C
:103E400074200000100000000000000001000000CD
:103E500001000000841E000000000000841E00001D
:103E60000000000001000000080000006461000084
:103E70007461000000000000000000005F4C0000C2
:103E80004F470000445500004D5000002E23000015
:103E900040210000005F0000544500005354000022
:103EA0004D4F0000442E0000234000002100000080
:103EB000564D0000434F0000444500002E410000D5
:103EC000424F0000000000002E2E00002F2E0000A8
:103ED0002E2F000074680000796D0000696F0000EB
:103EE0002D670000697400002F74000068790000DD
:103EF0006D6900006F2F00006D6D000061370000DC
:103F000036360000302E0000630000005F700000B5
:103F10006F770000657200006F66000066000000A9
:103F2000506F000077650000726F00006666000049
:103F3000000000005F4200004C570000484C0000A9
:103F4000564C00002E4400004154000000000000C8
:103F500010110000141200001300000001160000F0
:103F600017000000038000000F0F00000F0000008A
:103F700053032000830F51000A003200E381410007
:103F8000830F51000E003200E6815100830F510073
:103F900013003A000045880011458800E482A8001B
:103FA0000000060020458800014580000100500007
:103FB00040458800E482A900DCC2A8000000060099
:103FC00031458800104580008080500051458800B0
:103FD000DCC2A9000104200080CD20001088700000
:103FE00000000600DCC2A900E482A900000006006F
:103FF0000040DA000000FE000000000000000000A9
:1040000000000000000000000000000000000000B0
:1040100000000000000000000000000000000000A0
:104020000000000000000000000000000000000090
:104030000000000000000000000000000000000080
:107000000200370031587800030178008201E9005E
:10701000E00F5100FBFF3A000000060002003700BD
:1070200001587800030178008201E900E00F510067
:10703000FBFF3A0000000600889FBE008A9FBE004A
:107040008C9FBE008E1F7800000678000205BE00EF
:107050005C149000EC1490000001EB008A0F5400C7
:107060008B8F5C00380032004C409000E04F5000A5
:1070700024003200EE0220000C07470014C0B300C9
:107080000801BE008E0078001C409000A49E020003
:107090000000000012002000E00F50002A003A001B
:1070A000404698005C099000EC0990007C08900034
:1070B0008C1090000200400083804800800F540034
:1070C000818F5C000F003100BC4690000B00370040
:1070D0005C089000EC089000080440008984480097
:1070E00014C0B3000801BE008E0078001C40900060
:1070F000A49E0200000000008D46E900E1CF56008A
:10710000F3FF3E000001EB00E00F5500E08F5D0053
:107110000D003200E10220008C80400014C0B3005A
:107120000A01BE001C409000309E020000000000DA
:1071300012002000E00F500003003A005A16980099
:107140006B16980000017800020078004F07780065
:107150004F06BE004F05BE004F04BE0000000600F3
:10716000881F780000047800E10220008880400039
:1071700014C0B30018409000309E020000000000D0
:1071800031C0B300E00F50004C003A00D122200083
:1071900088804000914078008181FB00C819DD00A3
:1071A000C122200088804000914078008180FB004F
:1071B0008181710021C0B30052A52A00828F510045
:1071C0003E003A0078E39000C833DD00060020005E
:1071D00068E190008281FB0002002000020373003E
:1071E0008383730048E190000281FB0003002000CC
:1071F000020373008383730058E190004811DD009F
:107200000300200002037300838373000782FB00E6
:1072100005002000C021DD00020020006132B8001E
:10722000040171008581710064142400450520006B
:1072300080407800840F5100858F59001F00320074
:1072400038439100C833DD0006002000284091003B
:107250008080FB0000002000000373008183730026
:10726000084091000080FB00010020000003730033
:1072700081837300184091004800DD000100200068
:1072800000037300818373000781FB00030020006B
:10729000C010DD00000020006131B8000200700065
:1072A0008380700004006800858068000100700021
:1072B0008000EA0000807000CF00DE00014078000E
:1072C0004F0478000000060092002000E00F5000FC
:1072D0000C0032008041EB0090CF11000900320019
:1072E000B0019000818F510006003A0010409000DC
:1072F000249E0200000000006101600001003200D5
:10730000320020000200780000000600889FBE00C6
:107310008A1F7800000478006011B8000800780027
:1073200045FF070080047800E08F54005F003A00BA
:1073300030C0B300984F100054003A0058409000FD
:10734000E04F5000510032006000B8005014980027
:1073500061149800EA022000080545000220200080
:10736000890078000A0078002CFF0700C022200066
:107370000800400052C5B30002487800D022200027
:1073800008004000A2CAB3000248780022C5B3003A
:10739000626C9800726C98006F4141000274980012
:1073A00013C4B3001374980020212000080040008B
:1073B00024C7B300044878003021200008004000B2
:1073C000044878004021200008004000034878006D
:1073D0005021200008004000024878007801900009
:1073E00088099000602120000800400002487800D1
:1073F00071212000888040004810DE00804878001D
:107400008021200008004000401ADE000500200016
:107410000448780090212000080040004819DE0050
:107420000248780058019000E8019000A021200057
:107430000800400002487800B12120008880400008
:107440004810DE0080487800C0212000080040007D
:10745000401ADE000500200004487800D0212000FA
:10746000080040004819DE000248780014C0B3004C
:1074700018099000A80990008A0078001840900030
:10748000A49E020000000000594498000001EB0097
:107490008040EB00184090003C9F0200000000007C
:1074A0008004EA0080847400CF4CDE00090078007C
:1074B0004F0578004F04BE0000000600F687470025
:1074C000889FBE008A9FBE008C9FBE008E1F7800E2
:1074D00002447800900178001302FB000403B1001D
:1074E000E90F520009003E0093429000A2C3B3008E
:1074F00082CF520005003A000388E800B000200067
:10750000F0B79F00E00F5200E6013A003ECD800048
:107510008E087800C1002000F1B79F00E00F5700EF
:10752000E00132000041EB009E4F11000F003200DD
:107530001E409000249E0200000000008080FB009E
:107540006180600009003A00F0B79F00E04F5400EE
:10755000D4013200E4806000A3002000F3B79F0054
:10756000D0013A00F1B79F00CE0137000040EB0098
:10757000004F780010479800FE9C020000000000B9
:107580008080FB006180600032002000F2B79F0025
:10759000C4013A00E04F540004003200E48060006F
:1075A000A3002000F3B79F00BE013A006011B800AD
:1075B0000E007800EAFE07006066B800E14F500058
:1075C0001A003A000EF09300D1002000F1B79F009E
:1075D000E04F5000B30132007EF19300C811DD008E
:1075E000020020006EF093008080FB00000020006D
:1075F00000017100818171004EF093000080FB005A
:107600000100200000017100818171005EF0930093
:107610004800DD0001002000000671008186710035
:107620000C01BE000E007800CDFE07001200200005
:10763000F2B79F00E34F50009A013200D3002000C0
:10764000F3B79F00E04F500096013A00AE789000EB
:10765000C808DD001E7890000080FB00808070006C
:1076600000202000808F50008E013A005EC59000FF
:107670004855DD004EC090000080FB0000057500FD
:107680000B002000E00F5500E08F5D0012003A0073
:107690005ED59000C855DD000A0020004ED0900055
:1076A0008080FB00000020000005750081857500CA
:1076B0002ED090000080FB00010020000005750026
:1076C000818575003ED090004800DD00010020005B
:1076D00000057500818575005A0F98006B0F9800A2
:1076E000EE789000314798000141E900D000200079
:1076F000F0B79F00E14F51006A013E003E799000D3
:10770000A2EF9F0022479800E04F51006501320030
:10771000AFE997000381FB000200E900020160006D
:1077200060013A000EC190004811DD007E789000A3
:107730000080FB0000007100E0B79F004007980048
:10774000000178006F00610056013A002EC19000E0
:107750004811DD001EC090000080FB000001710098
:107760006114B800E00F5400E08F5C0014003A0090
:107770001ED190000281FB0003002000C813DD0031
:10778000060020000ED190008281FB000200200044
:1077900002017300838173006ECC90000884FB00AB
:1077A0000900200008037100898371007EC99000E0
:1077B0004811DD000300200002047300838473007D
:1077C0005E7B90004833DD004E7890000080FB0027
:1077D00000037300D3002000F3B79F003101320093
:1077E0000182FB00050020000401BE000A00BE006B
:1077F00086BF9F007A0402000000000090B79F003F
:10780000A1B79F000FBB97006130B800F0AF9F0099
:1078100081B79F00EFB097004408DE007FA9970072
:107820008FB1970000004100E08049001FB1970030
:10783000AFB197000001410081814900B2B79F00BC
:10784000C3B79F00820F5400838F5C00150139007D
:107850000203540083835C00AFE997000382FB00BE
:10786000050020000401BE000600BE005A0402000C
:10787000000000000002BE00E00F5000E08F580042
:107880000801320016C0B30050FF2000800F5200E4
:10789000E08F5A000500360036C0B300EB0F4200FF
:1078A000E08F5A0001003E0026C0B300620442008F
:1078B000E0844A00380F9800490F98003FB19700C4
:1078C000CFB197000200460083804E003017980029
:1078D000411798007FA897008FB097000C014000D7
:1078E0008D814800720F980003179800E34F5300F2
:1078F0001E003A00D1002000F1B79F006FB1970041
:10790000E00F5100E7003A005ED99000C811DD0099
:10791000020020004ED890008080FB000000200074
:1079200000007100818071002ED990000281FB005F
:107930000300200002007000838070003ED9900098
:107940004811DD00030020000200700083807000F9
:1079500010179800211798004248DD00CE40DE0045
:10796000810070004240DD001C003700D000200084
:10797000F0B79F00EFB09700E08F5000C9003200D1
:107980001FB09700AFB0970000014100818149000E
:107990001217980023179800E24F530003003A0093
:1079A0000800440089804C000C00370032002000A1
:1079B000030020000800BE0086BF9F007A0402007A
:1079C000000000008100D1000080D3006104640049
:1079D00008004000E08048000FBB9700F01FB00097
:1079E0000180B0004709DD004900DE0000007100A1
:1079F000C908DE00D3002000F3B79F00800F5500B8
:107A0000818F5D00A70039000080EB008080EB00D3
:107A100070079800010F98006000B80050079800A8
:107A200061079800E34F530093003A000040EB00D9
:107A3000504798007ED990004811DD006ED8900024
:107A40000080FB000001710002014600E0814E0051
:107A5000120F9800230F9800E10220008E80400052
:107A600014C0B3001E40900086BF9F00309E0200ED
:107A7000000000000FBB9700E00F50007E003A00AE
:107A8000D02220000E004000104078008080FB00D3
:107A9000C808DD00C02220000E0040001040780021
:107AA0000080FB008080700050A52A00808F50006D
:107AB00071003A001E719000C811DD000200200024
:107AC0000E7090008080FB0000002000000171001B
:107AD000818171006E6890000080FB000100200031
:107AE00000017100818171007E6890004800DD0016
:107AF0000100200000017100818171002025250016
:107B000011162400800F5100818F59005A003A004D
:107B1000502120000E00400010417800C811DD0007
:107B200002002000402120000E004000104078009C
:107B30008080FB0000002000000171008181710045
:107B4000202120000E004000104078000080FB0043
:107B500001002000000171008181710030212000AE
:107B60000E004000104078000080FB004800DD005F
:107B70000100200000017100818171002027270091
:107B800011142600800F5100818F59003A003A00ED
:107B9000D02120000E00400010417800C811DD0007
:107BA00002002000C02120000E004000104078009C
:107BB0008080FB00000020000000710081807100C7
:107BC000A22120000E014100124178000281FB0039
:107BD000030020000200700083807000B2212000AA
:107BE0000E014100124178000281FB004811DD00C6
:107BF000030020000200700083807000500798008E
:107C000061079800902120000E004000104178008C
:107C1000C811DD0002002000802120000E0040007D
:107C2000104078008080FB00000020000000710000
:107C300081807100622120000E0141001241780014
:107C40000281FB00030020000200700083807000AE
:107C5000722120000E014100124178000281FB00D8
:107C60004811DD00030020000200700083807000D6
:107C700070079800010F9800064F7800A819EC00D3
:107C800040CD8800300798006000B8005017980079
:107C9000611798000040EB00404798000000EB009F
:107CA000F0B79F007FB097004F0778004F06BE00E7
:107CB0004F05BE004F04BE006F01B100000006007A
:107CC00000017800B00020008001E900E00F5000C2
:107CD0000A003200124078000082FB0091427800D6
:107CE0000580FB000000520004003A000201E80099
:107CF0008100E80003007800F3FF37000000060071
:107D00008001780061CB2900010037008100E80084
:107D1000114178000200FB00E04F510002003200E8
:107D2000830F5000F9FF3A0000000600E887470083
:107D3000889FBE008A9FBE008C9FBE008E1F780069
:107D4000E1B79F0091067800F4C2B300C3C5B30049
:107D5000010037008D06E8001D417800844F510076
:107D6000FCFF3200834F5100FAFF3200900578008B
:107D7000B2002000010220000B007800A7FC0700E1
:107D80000005EB000A0778008C0020008A44780088
:107D900002C2B30051CC29006D447F000E07E800F9
:107DA000824F540033003600F0C2B300804F5400BD
:107DB00030003200C0C5B300804F54002D003200A7
:107DC000E0C2B300804F5400020032008C0F550017
:107DD0000A003900E80F560045003A00E0C2B3003F
:107DE000804F540042003A0020002000804CDD000B
:107DF0000C057800BC002000E7FF3700E04F54007E
:107E000004003D003940B3000884FB000808B100BD
:107E100061447C000880FB0081BF9F00F2B79F0097
:107E2000B7FF07008FB897007FB19700E00F5000B1
:107E30002F003A00F0CBB30000404400F94F50004F
:107E400002003E000914A00007003700F0C9B3008B
:107E500000404400F94F500003003E000904A00018
:107E600000CEB3000044440088757D000A05E80098
:107E7000C9FF37006FB097000E8846008040EB00C6
:107E800000C2B300804F540001003E0041C0B30067
:107E900060002000E00F55001600320050CEB30005
:107EA0009B4F100002003A0050C0B300804D780094
:107EB000E80F560002003A0020002000804CDD0050
:107EC0008984FB0063806400E10F500001003A00E8
:107ED0000144A000EC846400E48F540001003A00E7
:107EE0000134A000B14D98000000EB000100370004
:107EF000600020004F0778004F06BE004F05BE000F
:107F00004F04BE008F00B10000000600881F7800FB
:107F10000004780062005100E0805900380A9000A7
:107F2000C80A900062025200E0825A006011B80054
:107F3000840F5000858F58000900310028419000BF
:107F40000281FB00030020007A0402000000000010
:107F500038119000C8119000000141008181490052
:107F60000200BE004F04780000000600889FBE009B
:107F70008A9FBE008C9FBE008E1F7800000678008E
:107F80000205BE001800200009002000E10F51008A
:107F9000E08F59007D0036003C089000CC0890002E
:107FA000800F5100818F5900780031001C4078000B
:107FB000E24F50002F003200E34F500045003200E6
:107FC0000084EB008084EB00E14F50006F003A002A
:107FD0008206D100828646004969DE007C08900056
:107FE0008C10900002014000E08148000C007800F5
:107FF00011FC07000084EB008084EB00E00F5000D0
:1080000062003A000D007800F01FB200E002B000FC
:108010006C4778008D06E8004969DE007C08900016
:108020008C10900002014000E08148000C007800B4
:1080300001FC0700E00F500054003A000E87FB00DF
:10804000FD1FB200ED02B0006CC07E004804DD00F0
:108050000E04740061056500020032004444DE0035
:1080600002003700FEFF20000E046400090020001B
:10807000460037004859DD004850DE00000071001E
:10808000C858DE007C0990008C119000000141006E
:10809000818149000C007800E7FB07000084EB00B9
:1080A0008084EB00E00F500038003A000A054500DC
:1080B000FA1FB200EA02B0006C447D000884FB00A5
:1080C0000A0546001A4090004800DD0000047400D4
:1080D000E6FF37004959DD004750DE00000071001F
:1080E000C758DE007C0990008C119000000141000F
:1080F000818149000C007800CFFB07000084EB0071
:108100008084EB00E00F500020003A004255DD0073
:10811000FA1FB200EA02B0000A00460020419000B7
:108120000281FB0003002000C012DD0004002000DB
:1081300030419000C811DD000200200002017200F1
:1081400083817200104090004800DD000100200093
:1081500000017100818171006C407D000080FB0096
:10816000010020000001710081817100F0FF2000FA
:108170000300600001002000C004DD0008002000B2
:108180006110B80000047400818474000800BE000F
:108190004F0778004F06BE004F05BE004F04BE00DB
:1081A00000000600881F7800000478000000EB0043
:1081B0002004980038019000C801900021002000A0
:1081C000E10F5100E08F59003D00320018007800A7
:1081D000300A9000C00A9000840F5100858F59002A
:1081E00037003100E00F5100E08F590014003A00D1
:1081F00031C0B30090CF100005003A00101190007C
:10820000A0119000E00F5100E08F59000C003A00DF
:108210006011B80052049800630498004001900077
:1082200021002000E00F51002500320010119000C5
:10823000A011900072049800030C980018003700F9
:10824000A0409000E0CF500010003A0018007800E5
:1082500046FF07000001BE00E10F4000E08F48002C
:1082600014003200E10F5000E08F58001300360078
:1082700018007800C008900030089000800F51006E
:10828000818F5900F1FF39000C003700520498002B
:10829000630498001DFF070070049800010C98000B
:1082A000E302200018804100100C98008000EB00D1
:1082B00003003700110020000100370021002000DA
:1082C000010078004F04780000000600889FBE007F
:1082D0008A9FBE008C9FBE008E1F7800000578002C
:1082E0000204BE000406BE0020002000E10F510081
:1082F000E08F5900960036003A099000CA099000B4
:10830000820F5400838F5C00910031009A40780006
:10831000E2CF500040003200E3CF50005200320064
:10832000E1CF500088003A008805D10088854500DB
:108330004959DE007A0890008A109000020140003E
:10834000E08148000A0078003BFB0700E00F500086
:108350007D003A000B017800F21FB2006104640056
:1083600008003200E002200002004000EA407800ED
:10837000EFC060000C80FB004400DD0000C0700016
:10838000010037000C407800020145006069980048
:108390008B05E80010C0B300404598004959DE0045
:1083A0007A0890008A10900002014000E0814800A5
:1083B0000A00780020FB0700E00F500062003A003E
:1083C000FB1FB200E00F540005003200CC68DD0056
:1083D0004466DE000C867000C46EDE000B003700C1
:1083E000E10220008B8040006AC1780001CFB30019
:1083F000814061004869DD004866DE000C067100BE
:10840000C86EDE006F4666000CC670008B05450026
:10841000EC6D98004C003700484ADD004840DE0013
:1084200000007200C848DE007A0990008A119000AE
:1084300000014100818149000A007800FEFA07002E
:10844000E00F500040003A0008044400F81FB2005A
:1084500088004500EC689800010478004866DE005A
:108460007C6C9800380037004949DD004740DE0049
:1084700000007100C748DE007A0990008A11900060
:1084800000014100818149000A007800EAFA0700F2
:10849000E00F50002C003A004244DD00F81FB2000B
:1084A000EE022000080747008E004500E3854000EB
:1084B0008184E800194178000281FB00030020005C
:1084C000C012DD00040020001B417800C811DD004F
:1084D0000200200002017200838172005142780084
:1084E0000483FB004833DD00070020000602710012
:1084F000878271006A417F000281FB000300200037
:10850000020172008381720004002F0003016200E7
:1085100003002000C011DD00020020000C067100E5
:108520008D867100080445006C6C98004861DE007F
:10853000824878004069DE0003002000824C780009
:10854000486EDE008C4D780011C0B30041459800A4
:108550004F0778004F06BE004F05BE004F04BE0017
:1085600000000600889FBE008A9FBE008C9FBE0050
:108570008E1F7800000778000204BE00E00F510053
:10858000E08F59000B003A005E069000EE06900066
:10859000E00F5600E08F5E00120032003E089000AF
:1085A000CE089000800F5600818F5E000F003900CA
:1085B0000C0037000E0078006CFE0700E10F500041
:1085C000E08F58004D0036003E099000CE09900023
:1085D000820F5000838F58004E0039000806BE00FD
:1085E000020037001C0020000D0020000C05BE001A
:1085F00061054500E0854D003E089000CE089000E2
:10860000800F5500818F5D0005003900E10F560095
:10861000E08F5E003C0036002A0020000B002000A6
:108620000A01BE000E00780050FE0700E00F500067
:10863000E08F58000A003200E10F4000E08F480050
:1086400034003200E10F5000E08F5800310032005A
:108650008C0F55008D8F5D00E5FF3A002A00370032
:10866000F4FF2F00F5FF20000A01BE000E00780085
:1086700016FF070000017800E00F510018003A00D3
:10868000E00F5400E08F5C00070032000A02BE00D9
:108690000801BE000E0078000CFF07000001780002
:1086A000E00F51000E003A005A0798006B0798003F
:1086B0007E0090008E089000E10F4000E08F48009F
:1086C0001300320061005000E080580070079800ED
:1086D000010F980010C0B300504798000C003700FD
:1086E0001000200001002000E10F510009003A00B5
:1086F0000080EB008080EB000600370010002000B7
:1087000001002000030037006000B80001003700BE
:108710000A00BE004F0778004F06BE004F05BE009E
:108720004F04BE0000000600E4874700889FBE009B
:108730008A9FBE008C9FBE008E1F780000057800C7
:1087400001067800AA0690008D06E8004B00200084
:108750007C0032007A0090008A089000E00F500000
:10876000E08F5800770032006F8766006C003A0097
:1087700061004000E080480070059800010D9800FD
:108780005A019000EA0190001A007800E00F5100B1
:10879000E08F590004003A0040009000808F56009E
:1087A0005F00390067003700A04090008180FB0027
:1087B0008100E900446ADE008480600058003A00CD
:1087C000EAFD07000004BE002B002000E10F50006E
:1087D000E08F58005B0036001B002000E10F4000D6
:1087E000E08F4800570032001A00780030099000EE
:1087F000C0099000820F5400838F5C004100390053
:108800004B002000E00F56004E0032005A0190004D
:10881000EA01900053FF07000004BE007B00200027
:10882000E00F5000E08F5800460032002B0020007F
:10883000E10F5000E08F5800420032001B00200082
:10884000E10F4000E08F48003E0032006011B800A8
:108850001A007800F8F9070000067800E00F5600CB
:1088600038003A00E10220001A8040000220200077
:108870008C007800E9F907001A0278000801BE00B0
:108880000400780084BF9F00A0FD07000FBA970086
:1088900050129800611298000E0037004B4098006B
:1088A0006011B8001A007800E3F90700E00F5000EB
:1088B00023003A001A01780052109000E210900054
:1088C00061004000E080480050119800611198005C
:1088D0000C46E8001A007800A0409000814F560036
:1088E000EEFF39000C81FB000300200050129000C5
:1088F000E01290000201520083815A005210980049
:108900006310980058059800690598000801BE009A
:108910001A0078007DFD070070059800010D980091
:108920002D059800E10220001A8040004577DD0007
:108930000E0740001E0D98008005EB000100370077
:108940001B0020000B0078004F0778004F06BE0088
:108950004F05BE004F04BE004F00B10000000600EE
:10896000889FBE0080047800090078000DFE070093
:1089700000047800E00F540017003A0079019000DD
:108980008909900019007800ABF90700000478000D
:10899000E00F540010003A00190890008040EB00EE
:1089A00090CF10000B003200B0489000E8806000CB
:1089B00004003A00A9089000C1FC0700E00F500035
:1089C000050032008000EB000900780056FF070028
:1089D000E7FF370048002000080078004F04BE0081
:1089E000000006000200FA00889FBE000004780024
:1089F000D1BF9F0011407800F2C2B300824F5000F7
:108A000003003200C2C5B300824F500002003A009A
:108A10008100E800D1BF9F006000B80030049800DA
:108A2000410498005FB89700F1C1B30090CF1000E7
:108A300005003E0008007800DAFD07008000EB002A
:108A4000110C98002B003700F4044400E680570016
:108A500009007800B5FC0700E00F500025003A003F
:108A600008007800BEFF0700A8089000B1489000F9
:108A7000E00F500005003200E40F50001D003A00E6
:108A8000E48060001A0032001A003700E4806000C1
:108A900018003A009808900031489000700060007B
:108AA00013003200515190004811DD0041509000F8
:108AB0000080FB000001710003002000C011DD00F8
:108AC00002002000315A90004822DD00A158900099
:108AD0008180FB000102720005002000040171008A
:108AE000858171003204980043049800D7FF370055
:108AF000500020004F04BE000080FA000000060075
:108B0000889FBE008A1F78008004780009007800E2
:108B1000A4FD070000047800E00F54001D003A0097
:108B200079019000890990001900780042F9070046
:108B300000047800E00F540016003A001908900075
:108B400010407800FB4F400016003200E04F50000C
:108B5000140032001100200009007800F2FE070026
:108B6000ECFF3700190D9000020220008800780009
:108B70000A00780029F90700B2002000A908900037
:108B80000A0078001EF907009900780010C0B300B1
:108B9000C0409800080078004F0578004F04BE00E0
:108BA0000000060079019000890990001900780002
:108BB00021F9070000047800E00F5400F5FF3A00A7
:108BC000E8FF3700889FBE008A9FBE008C9FBE00D2
:108BD000000678000204BE0020002000E10F5100D2
:108BE000E08F59002F0036003C099000CC0990001E
:108BF0001DC0B300820F5400838F5C001F0039003A
:108C0000280037000801BE000C007800D7FC0700E0
:108C10000005BE00E00F5000E08F58001C0032003D
:108C2000E10F5000E08F58001B003200E10F4000C0
:108C3000E08F48001A0032006022B8000801BE0030
:108C40000C007800A1FD0700E00F500015003A006D
:108C50007C0090008C089000E10F4000E08F4800FD
:108C60000500320061004000E08048007006980076
:108C7000010E98005D4698000A04BE003C08900072
:108C8000CC089000800F5400818F5C00DDFF39001C
:108C90000000EB0003003700200020000100370037
:108CA000100020004F06BE004F05BE004F04BE005E
:108CB00000000600B2002000E04F500009003A001A
:108CC00032CD8000E00F51000100320000497800F1
:108CD000E08F5000010032008048EB0031CD880069
:108CE0000001EB0002007800000006006F02B000F7
:108CF000889FBE008A9FBE008C9FBE008E1F78009A
:108D00000007780081BF9F00000FEB00FF46610065
:108D10007E416100A1FD2F008F80400070805700D0
:108D2000E6F90700E1FC2F008F804000F1B79F00BB
:108D3000E00F500004003A008FB89700A0FD2F000C
:108D40000F00400027FF07006FB69700E00F5000AC
:108D500003003A00E00F560001003A0060002000D6
:108D60008D80FB007C81600055003200E00F5000D8
:108D70000A003200E40F500003003A00A0FD2F006B
:108D80000F0040005EFF07006FB69700E00F500035
:108D900090003A000D34A000070037003C499000D5
:108DA00071016100700020008A003A00E4806000D8
:108DB0008000200087003A00688066004C00320086
:108DC0001AA6020000000000604E98004801DE0074
:108DD000724E98004009DE00030020000256980001
:108DE0004808DE00105698008040EB00314E980095
:108DF000415E9800515E9800615E9800715E980037
:108E00007500460074024600FB0246007A034600E5
:108E1000104178000284FB004844DD009441780052
:108E20000381FB000204740009002000C044DD003F
:108E300008002000954378000781FB004811DD0001
:108E4000964378008781FB00030171000300200036
:108E50000204740083847400014B7800814A780016
:108E6000014A7800014878005FA8970011C0B3005C
:108E700041409800E00F5400E08F5C001C0032007D
:108E800050159000E01590000801BE004DFF07004E
:108E9000E00F50004F003A005FA8970061045400B3
:108EA000E0845C0058009800690098000A01BE0048
:108EB00061F80700E00F50000D0032004500370058
:108EC000E00F500043003A003C4990000281FB0053
:108ED000F0016100400020003E003A00E2806000A6
:108EE00003003200610161007000200039003A0087
:108EF00068806600010032000D54A0005FAA970050
:108F000054109000E4109000500F9800610F9800EA
:108F10007C0F98004D479800DC509000C808DD0099
:108F20004C5090000080FB00008070000100200089
:108F3000C000DD0000002000BC599000C819DD0011
:108F40002C5990000281FB00028171000300200077
:108F5000020070008380700070079800010F980075
:108F60007C599000C811DD00020020006C58900070
:108F70008080FB00000020000000710081807100F3
:108F80004C5990000281FB00030020000200700099
:108F9000838070005C5990004811DD0003002000C0
:108FA00002007000838070005007980061079800ED
:108FB0006000B8003007980041079800300F980013
:108FC000410F9800040F78003402900014079800B5
:108FD0000000EB004F0778004F06BE004F05BE00B3
:108FE0004F04BE006F02B10000000600EA87470090
:108FF000889FBE008A9FBE008C9FBE008E1F780097
:10900000000578000104780082057800E3B79F002E
:109010008009EB009A0090001A007800AAF8070077
:1090200000077800E00F5700B4003A004A42900071
:10903000E04F5200AE00350061026200AE00320027
:109040005A029000EA0290003A019000CA01900092
:109050000202520083825A00615BB800840F530001
:10906000858F5B00010036008405780088BF9F0073
:109070000002200000004500F0B79F008E0078003D
:10908000D1B79F000B077800950037003A01900098
:10909000CA019000F01F20000202600074003A0034
:1090A0001A007800C91ADE00C718DD004912DE0078
:1090B00004827000A04590008B45E90084C56500DE
:1090C00011003A00E00F5100E08F590003003A0010
:1090D0007A0090008A089000030037001A09900077
:1090E000AA099000A1FB0700E10F5000E08F580093
:1090F0000D003600E10F4000E08F480055003200BF
:10910000100D9800210D98001A0678001A09900099
:10911000AA0990000C0078007CFB0700E00F5000CB
:10912000E08F580004003A004A4090000074A0000C
:10913000404598006E0037000B84FB0009002000BA
:109140000004440081844C00C976DE002200320015
:109150002C4190008B85FB008B8146000281FB0037
:10916000828F5100010036008B0651000D427800BD
:109170000801BE008FB897001C409000309E02008E
:10918000000000004A429000E00F500023003A0027
:109190000404B2000E0032003A089000CA089000A1
:1091A00008005000898058006169B800820F5000A3
:1091B000838F5800060031004900DD008FB897000A
:1091C0000080400002202000FFB097008CF70700CD
:1091D000496CDD00360037003A089000CA0890005C
:1091E000880F5000898F58001F0032004A419000BC
:1091F0000204B2000E00320014C0B3000001BE0031
:10920000FFB097001C409000A49E020000000000E8
:109210004A429000E00F5000030032000474A000A6
:10922000444598000E0037000464A10044459800AE
:109230001A00780014C0B3000801BE00FFB0970008
:1092400010409000309E020000000000E00F50002F
:10925000050032004A4090000074A000404598008C
:109260001E00200025003700380D9800490D980099
:109270003A019000CA01900082017800F31FB20009
:1092800000202000030150000E047800820F5700D8
:109290000100360002047800FFB09700838140008F
:1092A00008017800830078000FB8970054F7070092
:1092B0000FB897000800400080BF9F003A0190005F
:1092C000CA01900008014100E08149003205980080
:1092D00043059800EFB09700910844000807570035
:1092E000E00F570069FF3A005FB7970003003700AF
:1092F0002E002000010037007E0020000E007800C4
:109300004F0778004F06BE004F05BE004F04BE0059
:10931000AF00B10000000600EA874700889FBE004A
:109320008A9FBE008C9FBE008E1F780000057800CB
:109330000104780082057800E3B79F008009EB0004
:109340009A0090001A007800DFF707000007780005
:10935000E00F5700D6003A004A409000E04F50001E
:109360005F00350062006000D00032005A029000B9
:10937000EA0290000B034200E0834A00840F53008E
:10938000858F5B00010031008E05780088BF9F004B
:109390000002200000004500F0B79F008E0078001A
:1093A000D1B79F000B077800B00037003A0190005A
:1093B000CA019000F01F2000020260008E003A00F7
:1093C0001A027800C91BDE00C718DD004913DE0051
:1093D00006837000A44590008B45E90086C56500B2
:1093E00021003A00E00F5100E08F59000B003A00D5
:1093F0007A0090008A089000E00F5000E08F58003B
:109400000D003A000001BE000400780055FC070082
:1094100070059800010D9800040037001A099000AB
:10942000AA099000040078004EFC0700E00F5000ED
:10943000E08F58008F0032004A429000E10F500048
:10944000E08F580003003A000474A00044459800DF
:1094500023003700E10F4000E08F48001000320089
:10946000100D9800210D98004A4190000204B200AE
:10947000100032001A00780014C0B3003A099000BE
:10948000CA099000FFB0970010409000A49E02000F
:10949000000000004A429000E00F5000030032003C
:1094A0000474A000444598004F0037000464A100F4
:1094B000444598001A0678001A099000AA099000FD
:1094C0000C00780091FA0700E00F5000E08F580080
:1094D00005003A004A4090000074A0004045980002
:1094E0002E002000720037000B84FB0009002000D2
:1094F0000004440081844C00C976DE002300320061
:109500002C4190008B85FB008B8146000281FB0083
:10951000828F5100010036008B0651000D42780009
:109520000801BE008FB897001C409000A49E020066
:1095300000000000E00F500028003A003A089000B8
:10954000CA08900008005000898058006169B8007E
:10955000820F5000838F58000A0031004900DD005F
:109560008FB8970000804000022020008000780023
:109570007FB09700A2F607004A4190000264A10064
:1095800042459800496CDD002C0037003A099000F4
:10959000CA099000880F5100898F590014003200C9
:1095A0003A029000CA0290005A019000EA0190002D
:1095B000820F5200838F5A000D00310014C0B30097
:1095C0000801BE00FFB097001C409000309E0200D2
:1095D00000000000E00F5000050032004A409000FB
:1095E0000074A000404598001E00200030003700A5
:1095F000380D9800490D98003A009000CA0090007C
:10960000F01FB20001202000008150000E047800FD
:10961000820F57000100360002047800FFB0970067
:1096200000804000080178008FB8970074F60700AA
:109630004A4190000264A000424598000FB897008C
:109640000800400080BF9F003A019000CA019000CE
:1096500008014100E0814900320598004305980067
:10966000EFB097009108440008075700E00F57003B
:109670004EFF3A005FB797003A019000CA01900090
:109680005A009000EA009000800F5100818F59002D
:10969000020036005205980063059800CA40900009
:1096A0000154A00041459800010037007E002000D1
:1096B0000E0078004F0778004F06BE004F05BE0031
:1096C0004F04BE00AF00B10000000600889FBE003E
:1096D000000478009800900018007800FAF607005F
:1096E000E00F500042003A00C84090008180FB002B
:1096F000010178000202B2003D0032000104B20014
:10970000100032000102200088804000180078001C
:1097100014C0B30038099000C809900010409000B0
:10972000A49E0200000000008000780010002000CD
:10973000E08F50002E003A00484090000064A100E5
:109740004044980058099000E809900018007800FB
:1097500039F60700E00F500025003A00F80C9000A1
:109760006B8044001054A00028489000C05C980012
:1097700038489000D05C980048489000E05C980021
:1097800058489000F05C980068489000A05C9800F1
:1097900078489000B05C980008509000C054980041
:1097A00018509000D05498001AA602000000000043
:1097B000E05498004801DE00F25498004009DE00B1
:1097C00003002000825C98004808DE00905C98004E
:1097D000484090000054A100404498009800780050
:1097E00010C0B300C040980018007800C7F607000A
:1097F0004F04BE0000000600881F780000047800B7
:1098000008007800B1FF0700E00F500001003A00A7
:10981000000C78004F04780000000600EA8747003B
:10982000889FBE008A9FBE008C9FBE008E1F78005E
:1098300000077800E2B79F00F3B79F009E009000FA
:109840001E007800A0F60700D0B79F00E00F500080
:1098500005013A00CE419000E0CF510000013500F3
:109860005E009000EE0090006FB29700FFB297008C
:10987000800F5200818F5A0004003600E28161009F
:1098800002003A00E0B79F00F1B79F003E0590004C
:10989000CE0590006000B80030079800410798009E
:1098A0006FB29700FFB29700E00F5200E08F5A00AE
:1098B000AA0032001E037800264290000482FB00BA
:1098C00005002000492CDD00C724DE008904740057
:1098D0004924DD00E00F5500E08F5D0028003200D4
:1098E00061055500E0855D006FB19700FFB19700FD
:1098F00061005100E08059000801BE0086BF9F0052
:109900005A040200000000000006BE000801BE006C
:109910000A00BE005A040200000000000FBB9700BE
:10992000800F5600818F5E00150039006000140022
:10993000E0801C00800165000183650007002000B5
:10994000C032DD0004002000611BB8000602720076
:109950008782720034079800450798006FB097001F
:10996000FFB097000400500085805800E0B79F00CA
:10997000F1B79F001E099000AE0990001800370053
:109980007E0190008E099000E00F5100E08F590099
:1099900011003A0006007800F2FA07000001BE004C
:1099A000E10F5000E08F58005F003200E10F4000EF
:1099B000E08F480006003A004E4090000074A0007E
:1099C0004047980012002000D2B79F00A600370041
:1099D00070079800010F9800120F9800230F98004D
:1099E000E00F5100E08F59005F0032003300370074
:1099F000CE409000E2806000070032001E00780038
:109A0000D8FA07000001BE00E00F5000E08F5800B8
:109A100004003A002F0037001E00780053F90700B9
:109A20000001BE00E10F4100E08F490006003A004E
:109A30004E4090000074A0004047980013002000A2
:109A4000D3B79F0088003700E10F5100E08F590025
:109A5000060036009E007800310A9000C10A90008E
:109A6000840F5100858F5900060039004E40900048
:109A70000074A0004047980024002000D4B79F0045
:109A800079003700120F9800230F98003E029000D3
:109A9000CE0290000402440085824C0034079800F6
:109AA000450798006FB09700FFB09700080050007E
:109AB00089805800E0B79F00F1B79F006FB2970010
:109AC000FFB29700880F5200898F5A00C8FF3E00EE
:109AD00002003700E8B79F00F9B79F003E029000F0
:109AE000CE0290006FB09700FFB0970004024000D4
:109AF0008582480034079800450798006FB29700A8
:109B0000F41FB20005002000E00F5200E08F5A0061
:109B1000170032001E007800FCF80700E00F50002C
:109B2000E08F580004003A004E4090000074A000FE
:109B3000404798004A0037006FB19700FFB1970087
:109B4000C91CDE00471ADD004914DE00080472005B
:109B50000004440081844C00060037006FB4970075
:109B6000FFB49700030037000204BE000100370075
:109B70000404BE003E009000F01FB2002B00320033
:109B80003E099000CE099000820F5400838F5C0044
:109B9000260032004E4090000004B2001100320056
:109BA000010220008E8040001E00780014C0B30027
:109BB00010409000A49E020000000000CE409000E3
:109BC000E00F5000050032000174A00041479800EA
:109BD00015002000D5B79F00230037000164A100C5
:109BE00041479800010220008E8040001E0078004E
:109BF00014C0B3000801BE0010409000309E020067
:109C000000000000E00F5000060032004E409000BF
:109C10000074A0004047980010002000D0B79F00BB
:109C200011003700380F9800490F98003E0090004F
:109C3000CE0090005E019000EE019000820F500077
:109C4000838F58000800360050079800610798007D
:109C50004E4090000054A00040479800020037009A
:109C600021002000D1B79F005FB097004F07780018
:109C70004F06BE004F05BE004F04BE00AF00B1004E
:109C8000000006008358EC00804078000100780056
:109C900083F8B7000100FB00E0CF5000080034005B
:109CA00082C2B30082CF50000B00340001C8B30061
:109CB0008000FD0083F8B7008000FD000000060072
:109CC00042002000811F7800110009000200D80026
:109CD000CF0078000000EA0000000600FF4F5000AF
:109CE00002003E0080407800060037008040EB0014
:109CF000F2C3B300824F500002003E0001C4B30023
:109D000080C050000140780000000600889FBE001F
:109D10008A1F7800800478008258EC0082F8B7002F
:109D200001C6B300814F5000010036008278EF0079
:109D30002188210091407800814C78000904780046
:109D400000C2B30000C14000026C780000C6B3003E
:109D5000804F510001003600004C51000985E80099
:109D60000144B000014D780000C6B30080CF500020
:109D70000100360000CD500019407800D7FF0700E1
:109D8000804C780018407800D4FF0700004C780021
:109D90001A407800D1FF0700004D78004F05780089
:109DA0004F04BE0000000600800078000000EB00B9
:109DB000E48F500009003200E88F500007003200A5
:109DC00010002000E08F500004003A00B0C3800073
:109DD0008000EA00008070004F00DE0000000600F6
:109DE000889FBE000004BE00090444000100370043
:109DF00069045400E80F5400FDFF3C0001003700E7
:109E000069044400E00F5400FDFF350008007800AD
:109E1000E5FF0700E00F5000F3FF32000800780074
:109E20004F04BE000000060000102000E48802007D
:109E30000000000000202000E48802000000000074
:109E400000012000E4880200000000004000200023
:109E5000E48802000000000010002000E4880200F6
:109E60000000000000012000E48804000000000061
:109E700001002000E80F5000E08F58002B003E004A
:109E80000060010008003700090037000B003700B0
:109E90000E0037001100370013003700150037009F
:109EA000180037001C0037000041EB000C003700A1
:109EB0000041EB0001C2B300140037000041EB0089
:109EC00001C2B30001407800110037000041EB00EF
:109ED0008240780000C2B3000D00370002C2B30018
:109EE00082407800F7FF370002C2B3008040EB00E9
:109EF000F4FF370002C2B300824078000040EB005C
:109F00000300370002C2B3008040EB00024078003B
:109F10005EC204000000000052C0B300F1C0B300F4
:109F200000C2B3005EC20200000000000000060094
:109F300054FF0700004178008040EB005EC2020041
:109F400000000000FFD7BF000080FB000000EA0017
:109F50004F00DE008000EB00E04F500005003200B3
:109F600071912100914078008180FB008100E9001F
:109F7000CF08DE0017F9B700E08F50000200320072
:109F8000A0F62F00E0C3880002D8BF000080FB00CD
:109F90000000EA004F00DE008000EB00E04F5000C0
:109FA0000500320061912100914078008180FB0022
:109FB0008100E900CF08DE0016F9B700E08F5000FD
:109FC0000200320060092000E0C38800FED7BF0015
:109FD0000080FB000000EA004F00DE008000EB0084
:109FE000E04F50000500320051912100914078006F
:109FF0008180FB008100E900CF08DE0015F9B70081
:10A00000E08F500007003200E0C38000E00F5000F6
:10A01000020032007C38EF0002003700A0F62F006B
:10A020007A38B40001D8BF000080FB000000EA00CD
:10A030004F00DE008000EB00E04F500005003200D2
:10A0400041912100914078008180FB008100E9006E
:10A05000CF08DE0014F9B700E08F5000070032008F
:10A06000E0C38000E00F5000020032007C38EF00B7
:10A0700002003700600920007A38B4000000EB00CD
:10A08000E17F210091407800E0CF500004003200D1
:10A0900001D8BF000080FB000000EA004F00DE0096
:10A0A0008000EB00E04F50000500320031912100AC
:10A0B000914078008180FB008100E900CF08DE003C
:10A0C00013F9B700E08F5000010032007A38EF003A
:10A0D0000000EB002180210091407800E0CF50008B
:10A0E00004003200FFD7BF000080FB000000EA0040
:10A0F0004F00DE008000EB00E04F50000500320012
:10A1000021912100914078008180FB008100E900CD
:10A11000CF08DE0012F9B700E08F500001003200D6
:10A120007C38EF0050468000E00F500048003200BD
:10A1300001022000810F50003000320014003C006A
:10A14000E60F50003C00320006003C00E40F5000D7
:10A150002F0032003B003C00E20F50003B003A0071
:10A1600026003700ED0F50003600320003003C009F
:10A17000E80F500035003A0027003700F00F50007C
:10A180002D003200F10F500030003A00200037005F
:10A1900001052000810F50001800320008003C002B
:10A1A000E3805000810F5000190032008100E80068
:10A1B000810F5000200032001102200005003700FE
:10A1C00051052000810F50001100320004003C00B6
:10A1D000E4805000810F50001C003A000E00370050
:10A1E00061052000810F5000130032008100E8005B
:10A1F000810F500015003A0012003700E0C38000C4
:10A20000E00F500007003A00600920000800370006
:10A21000A0F62F0009003700E0C38000E00F5000D7
:10A22000020032007C38EF0008003700A0F62F0053
:10A230007A38B4000500370060092000E0C38800C8
:10A24000020037007C38EF007A38EF00CA28EF00B0
:10A2500080252000D1C38000808F50000100340091
:10A26000D0C3880080DA2F00D1C38000808F5000D7
:10A2700001003D00D0C3880080252000E1C380009C
:10A28000808F500001003400E0C3880080DA2F0086
:10A29000E1C38000808F500001003D00E0C38800D2
:10A2A000D1C38000E0C38000010140006245880006
:10A2B000008050007045880000000600881F78006C
:10A2C0000004780008007800E9FE07006140B8004B
:10A2D000E80F5000E08F58003E003E000060010093
:10A2E0000800370009003700370037000D0037003D
:10A2F00035003700170037001F00370030003700E7
:10A3000031003700000021003000370040002000FD
:10A31000E48802000000000096A502000000000092
:10A320002C00370000102000E4880200000000002C
:10A3300040002000E4880200000000000041EB0023
:10A3400082407800F0C0B3005EC20200000000004E
:10A350002000370040002000E488020000000000D8
:10A3600000012000E488020000000000600F2000CF
:10A370007046880017003700A0F9290070A8020075
:10A380000000000000047800E00F54000E003A00C6
:10A390002100200080952100FEA80200000000009E
:10A3A00021002000A0952100FEA80200000000006E
:10A3B0000800780070A802000000000002003700CA
:10A3C0007A38EF007C38EF0040002000E48802007B
:10A3D000000000004F0478000000060029FE07007E
:10A3E00000417800804078000040EB005EC202002F
:10A3F00000000000FED7BF000A00320001D8BF00F5
:10A400000800320040458000AA08B4002200200065
:10A41000110009000200D8006009B000C0CA88001D
:10A4200010C0B300F17F210091407800E0CF5000D0
:10A43000120032002180210091407800E0CF5000CE
:10A440000E00320040458000AA08B400220020001F
:10A45000110009000200D800D0CA8800510920006C
:10A46000810F500002003E00800C2000D0CA8800FE
:10A47000A0F62F005A39B40002003700E04F500018
:10A480000D0032008043EB000743780087427800DC
:10A4900007427800874178000741780087407800BC
:10A4A000074078000EC2020000000000AC28EF0058
:10A4B000AE28EF000000060043458000C2CA8000BD
:10A4C000828F5100010031008EF8B700D1CA8000A0
:10A4D000818F51000200360010C0B3008EF8B70023
:10A4E00050458000820F5000010031008F78EF004E
:10A4F000810F50000200360010C0B3008FF8B70083
:10A500008ED8BF00F18821009140780006003A0003
:10A51000E0CF500008003A008000FD008DF8B70041
:10A520008000FD0015003700E14F500002003A00A6
:10A53000E0CF500010003200E1CF500004003A009C
:10A54000E04F500002003A008DF8EF000B0037009A
:10A550008DD8BF004240A9000200340020C0B300E3
:10A5600005003700E04F500002003200E0CFB3009A
:10A5700001003700A0C0B3008DF8B700D7882100D4
:10A5800097437800E0CF53000B003A00C012200040
:10A59000604588007045880007437800874278004E
:10A5A00004C2B300874178000741780087407800F3
:10A5B0000440780036003700E1CF53000B003A002A
:10A5C000C012200060458800AE28EF008043EB00F9
:10A5D00007437800874278000742780003C2B3003F
:10A5E000074178008340780028003700E1CF43001E
:10A5F0000A003A00AC28EF00C01220007045880025
:10A6000007C2B3000043EB0087427800064278009F
:10A6100086417800064178001B003700E2CF4300F6
:10A620000D003A0040ED2F0060458800C012200068
:10A63000704588008043EB0006C2B3008742780073
:10A64000074278008741780007417800874078000A
:10A65000074078000E003700E2CF53000E003A00AA
:10A66000C01220006045880040ED2F007045880032
:10A670008043EB0007437800874278000742780068
:10A680008741780002C2B300864078000640780017
:10A690000EC2040000000000EACF530004003A009C
:10A6A000C01220006045880040ED2F0070458800F2
:10A6B000000006000400FA00881F78000040200017
:10A6C000C16680000080600044003200F1BF2F00AE
:10A6D00080CD200010886000B78821009743780063
:10A6E000E0CF53000C003A00070078008CF8B70068
:10A6F00010C0B3008BF8B70007437800874278009A
:10A700000742780087417800074178008740780049
:10A710007F404000150037008CD8BF00E1CF5300C8
:10A7200015003A00E24F50002C003400FD4F50005D
:10A730002A003C0021C0B3008000FD008BF8B70068
:10A740008000FD000040E80088F8B700FFC3430028
:10A750000043EB008642780006427800864178008C
:10A760000641780087407800074078000EC202005A
:10A770000000000019003700E2CF530017003A0034
:10A78000818821009140780080CF500013003D0067
:10A7900071C2B300814F500010003C0030C0B300C4
:10A7A0008BF8B700FEC34300074378008042EB00FC
:10A7B000054278008541780007417800874078009D
:10A7C000074078000EC20200000000007000200068
:10A7D000EAD10200000000008A78EF008CD8BF00A8
:10A7E00031C6B300814F500002003C000040E80039
:10A7F0008CF8B70020C3B300C188210091407800D5
:10A8000080CF50000B0034008B78EF008043EB00CA
:10A810000743780087427800074278008741780034
:10A820000741780087407800074078000EC2020098
:10A83000000000008CD8BF00E54F500015003A0022
:10A8400089D8BF00E14F500009003A008BD8BF0003
:10A85000E14F50000F003A0020C0B30089F8B70064
:10A86000000520006045880000FB2F00080037002D
:10A87000E24F500007003A008BD8BF00E14F500074
:10A8800004003A0089F8B700000520006045880000
:10A89000704588008CD8BF00FE4F500012003A006F
:10A8A0008BD8BF009188210091407800E0CF500004
:10A8B00008003A00E24F500006003A0010C0B30012
:10A8C00089F8B700000520006045880070458800C1
:10A8D00005003700E24F500003003A008978EF008E
:10A8E000AC28EF00AE28EF0080C2B300C188210081
:10A8F0009140780080CF500009003A008BD8BF000B
:10A90000E34F500006003A0010C0B30089F8B700CA
:10A910000105200061458800AE28EF008AF8B700E5
:10A920001008200041458000808F50000300340053
:10A9300051458000808F50000B003C00AC28EF0098
:10A94000AE28EF000041EB008240780000C2B30067
:10A950007AC20200000000000041EB008240780053
:10A9600000C2B300080037000041EB0082407800CD
:10A97000024078007AC20200000000000041EB00B3
:10A98000824078000240780096C202000000000079
:10A99000A888210018447800E04F540022003200BB
:10A9A00066805700D9FC07004FF99700BFF8970061
:10A9B0002FF897005EC20200000000003FF99700E8
:10A9C000AFF897004FF8970096C202000000000011
:10A9D0002FF99700CFF897003FF897007AC202004E
:10A9E000000000008A58EC008AF8B700F1C7B300F5
:10A9F000814F500012003A008A78EF000041EB00CE
:10AA0000824078000240780096C2020000000000F8
:10AA10000041EB0082407800024078007AC20200D8
:10AA2000000000000600370096FC07000041780097
:10AA300088407800014078005EC2020000000000FB
:10AA40004F0478000080FA0000000600EE874700FF
:10AA5000889FBE008A9FBE008C9FBE008E1F78001C
:10AA60000E0078000F077800AE01B1000300090066
:10AA7000001FEB000007780082FC07000041EB009C
:10AA8000804078005EC202000000000084D8EC0024
:10AA900084F8B7008080FB00C508DE0002C2B30066
:10AAA000FA81570082F178007F4060008101E9005F
:10AAB000E78161000041510002427800FA825700AC
:10AAC00084F279008100E800E780600000417800AE
:10AAD00082F27800DFEB97004FEB9700BFEA970018
:10AAE0002FEA97009FE997000FE99700FFE0970092
:10AAF0006FE097000EC202000000000001D8BF0006
:10AB00000080FB000000EA004F00DE008000EB0048
:10AB1000E04F500005003200E190210091407800A4
:10AB20008180FB008100E900CF08DE000EF9B7004C
:10AB3000E08F50000700320001CB80002103B000FD
:10AB400001CB8800401F2000808F5000010034009E
:10AB500000CB8800FED7BF000080FB000000EA00A9
:10AB60004F00DE008000EB00E04F50000500320097
:10AB7000D1902100914078008180FB008100E900A4
:10AB8000CF08DE000DF9B700E08F5000070032005B
:10AB900001CB80002103B10001CB880040ED2F00E4
:10ABA000808F500001003D0000CB88000ACB800060
:10ABB000E00F55005300350098438000A14380000A
:10ABC000C6438000D24380006116B9006142B900DB
:10ABD0000C0642008D864A00018040006102B900E7
:10ABE0000C0642008D864A00B04380006302B90023
:10ABF000CFA2DE000C0642008D864A00060043000C
:10AC00006102B9000C0242008D824A00D0FF2F0081
:10AC10000088B900CF80DE00C3FF2F0003C4B90055
:10AC2000CFC4DE000000440081804C006333B900D3
:10AC3000CFB3DE000000430081804B004211DD00F5
:10AC4000CF91DE0000064100818649000C004200E1
:10AC50008D804A006154B9000801BE00F4B79F001E
:10AC600085BF9F007A040200000000000E7D2000D6
:10AC7000811F7800110009004E08D800CF0078002D
:10AC8000800555006B4588007FB297008FBA97000A
:10AC90000C0052008D805A000801BE007A040200A8
:10ACA00000000000811F7800110009004E08D80044
:10ACB000CF007800000555007A45880081DA2F0022
:10ACC000818F550001003D0061458800810F5500CE
:10ACD00002003D0080DA2F007045880080252000AA
:10ACE00061458000808F500001003400604588007D
:10ACF0008025200071458000808F500011003400B5
:10AD00000F003700F24380000A91B90044ED2F0094
:10AD1000110009004419D800000178000A0141001F
:10AD200062458800E04380000A80B900811F7800F6
:10AD3000110009004408D800CF0078000A00400044
:10AD4000704588001008200041458000808F500029
:10AD50000300340051458000808F500008003C0003
:10AD6000AC28EF00AE28EF0001C2B30080C0B300F2
:10AD70001AC102000000000001C2B3000500370044
:10AD80008040EB0080C0B3001AC102000000000048
:10AD90008040EB00B0C0B3001AC102000000000008
:10ADA0004F0778004F06BE004F05BE004F04BE009F
:10ADB000EF00B10000000600889FBE000004BE0046
:10ADC0000041EB0089407800084078005EC2020034
:10ADD000000000000041EB00894078000840780046
:10ADE0007AC20200000000000041EB0089407800B8
:10ADF0000840780096C20200000000004F04BE0028
:10AE000000000600889FBE0010CB8000800040003C
:10AE10008080400000468000E00F500001003D00AF
:10AE20000000EA008080400010468000E00F5000E3
:10AE300001003D000000EA008080400020468000C4
:10AE4000E00F500001003D000000EA0000804000DB
:10AE50004200DE0010CB880018002000ED0F5000EB
:10AE6000010036000004EB0011C0B300EE0F5000EB
:10AE700003003E008040EB000000EB0004003700C0
:10AE800011D9BF000080FB000000E9004F00DE0088
:10AE90008000FD0011F9B7008000FD00E00F5000B8
:10AEA000050032000041EB0082407800F0C0B300A2
:10AEB0005EC202000000000010CB8000ED0F5000C9
:10AEC00011003E008618EC0030C48800E50F5000E9
:10AED00007003400EA0F500001003A008638EF0006
:10AEE0000041EB008240780000C2B300030037004D
:10AEF0000041EB0082407800024078005EC2020010
:10AF000000000000030037005EFB07008000EB003C
:10AF1000A9FF0700B0468000E00F50000400320097
:10AF2000D628EF0050002000EAD102000000000007
:10AF3000A1438000803E2000808F50001700340025
:10AF4000B2438000800F510014003400C2438000DF
:10AF5000800F510011003400E2438000800F510047
:10AF600003003C00F2438000800F51000B003400CE
:10AF70002008200042458000800F51000700340067
:10AF800052458000800F510004003400AC28EF00CF
:10AF9000AE28EF00180020006600370093438000C1
:10AFA000803E2000C2438000808F51000A003C0098
:10AFB000808F500008003C00B4438000800F520096
:10AFC00005003C00800F510003003C00D44380008A
:10AFD000800F520045003400D0438000450020001F
:10AFE00080037800811F7800110009008500D800D7
:10AFF0008003FD00CF00780054002000000378009B
:10B00000811F7800110009008401D8000003FD00B1
:10B01000CF00780086834300B6438000809FBE0047
:10B02000110009000503D800000378004F00BE009E
:10B030008683430000037800811F78001100090017
:10B040000501D8000003FD00CF0078008682430090
:10B0500000037800811F7800110009000400D80067
:10B060000003FD00CF00780086824200801F780038
:10B07000110009008400D800800078004F0078009B
:10B0800064002000809FBE00110009008401D800E8
:10B09000800178004F00BE0083804000A6FF2F0093
:10B0A000811F7800110009000600D8000003780015
:10B0B000CF00780006804000B6FF2F00809FBE00C2
:10B0C000110009000601D800000378004F00BE00FF
:10B0D00006014000028042000000EA00604588004E
:10B0E000850251007545880012003700E343800057
:10B0F000F1438000808F510002003C00808F50009F
:10B100000A00340042002000811F7800110009006D
:10B110008201D800CF007800604588001100090046
:10B120008200D8007045880002003700AC28EF008C
:10B13000AE28EF001008200041458000808F5000AD
:10B140000300340051458000808F50000B003C000C
:10B15000AC28EF00AE28EF000041EB008240780001
:10B1600000C2B3007AC20200000000000041EB0000
:10B170008240780000C2B300080037000041EB00B5
:10B1800082407800024078007AC20200000000008D
:10B190000041EB00824078000240780096C2020035
:10B1A0000000000080DA2F0061458000808F500091
:10B1B00001003D006045880080DA2F007145800065
:10B1C000808F500001003D007045880080252000E0
:10B1D00061458000808F5000010034006045880088
:10B1E0008025200071458000808F500001003400D0
:10B1F00070458800084078008000EB00E04F540064
:10B200000500320001912100914078008180FB000F
:10B210008100E900CF08DE0010F9B700E08F500090
:10B220000300320040002000EED1020000000000C8
:10B2300010C0B300E00F5400030032000040EB00E8
:10B240008000EB0005003700F1902100914078006C
:10B250008180FB008100E900CF08DE000FF9B70014
:10B26000E08F5000030032000080EB00EAD10200C2
:10B27000000000004F04BE00000006000400FA00B9
:10B28000889FBE008A9FBE00984380000005EB00A7
:10B290001000200091032000808040008180400049
:10B2A00002802000E2807800888F50000200340085
:10B2B00000057800010478000000E800E40F500069
:10B2C000F4FF3400E0CA800062051500220020006F
:10B2D000801F7800110009000200D800800078006B
:10B2E0004F00780001D5B900C9DA2000890F540059
:10B2F0000C00340001FA2000810F540007003C00CC
:10B3000088845400809FBE00110009008204D80088
:10B31000800478004F00BE00110037008004EA006E
:10B320000F00370071BB2000810F540002013C0068
:10B33000813EB100810F54000B00340089C12F0001
:10B340008884440092FF2F00809FBE0011000900F6
:10B350008204D800800478004F00BE00C912B000FB
:10B36000808F540001003400800478008000EA00DF
:10B37000818F540001003D0081047800311F2000BE
:10B38000810F54000A003C000188210091407800A0
:10B39000E0CF50000300320060458800704588000F
:10B3A00007003700AC28EF00AE28EF00040037009C
:10B3B0000A804400704588000A8054006045880077
:10B3C00080D8BF004240A9001400340081D8BF00DB
:10B3D000120032006C8057004CFA07006FF19700A2
:10B3E000DFF097004FF097005EC2020000000000FF
:10B3F0005FF19700CFF097006FF0970096C20200C0
:10B40000000000004FF19700EFF097005FF0970009
:10B410007AC20200000000000400370019FA070099
:10B42000800078000000EB0063FE07000788210021
:10B4300097437800E0CF5300160032007FD8BF005A
:10B440005E59B4007FF8B700FE4F5000020036008E
:10B450005EF9EF0004003700E04F500002003A00B0
:10B4600010C0B3005EF9B700F5872100954278005F
:10B470008580FB004309DE00C408DE0081437800BC
:10B480000243780004C2B300854178000040EB001D
:10B49000070037000743780005C2B3000542780073
:10B4A00085417800074178008740780007407800A0
:10B4B0000EC202000000000001D8BF000080FB00A7
:10B4C0000000EA004F00DE008000EB00E04F50007B
:10B4D00005003200C1902100914078008180FB007E
:10B4E0008100E900CF08DE000CF9B700E08F5000C2
:10B4F00007003200E1CA80002103B000E1CA8800E1
:10B50000401F2000808F500001003400E0CA8800F6
:10B51000FED7BF000080FB000000EA004F00DE0005
:10B520008000EB00E04F500005003200B190210098
:10B53000914078008180FB008100E900CF08DE00A7
:10B540000BF9B700E08F500007003200E1CA80001D
:10B550002103B100E1CA880040ED2F00808F500028
:10B5600001003D00E0CA880010C0B300411F200068
:10B57000810F540003003C000040EB008000EB0012
:10B5800005003700A1902100914078008180FB00E8
:10B590008100E900CF08DE000AF9B700E08F500013
:10B5A0000300320060002000EAD102000000000029
:10B5B000E00F55000D003A00E08F540060003A00A3
:10B5C00081D8BF005E003A00401F2000800F540069
:10B5D0005B00340010C0B30081F8B7007000200099
:10B5E000EAD1020000000000010037008178EF007E
:10B5F0001008200041458000808F50000300340077
:10B6000051458000808F500008003C00AC28EF00BE
:10B61000AE28EF0001C2B30080C0B3001AC102001F
:10B620000000000001C2B300050037008040EB00BD
:10B6300080C0B3001AC10200000000008040EB008F
:10B64000B0C0B3001AC102000000000080D8BF00E3
:10B65000020032000040E90080F8B700D8ECAB00EF
:10B660003B003200F1F72F0080CD200010886000F1
:10B670008078EF00724480008E28EF000004EB0019
:10B680001000200071042000808040008181400073
:10B6900004802000E4817900828F51000200340090
:10B6A00000047800030178008180400003802000BE
:10B6B000818041008008EB000000E800E60F5000A8
:10B6C000F0FF340080BB2000800F510020003400C8
:10B6D000F84488009C08ED00E20F50001C003E007A
:10B6E00010C0B300E20F5400030032000040EB0032
:10B6F0008000EB0005003700919021009140780018
:10B700008180FB008100E900CF08DE0009F9B70065
:10B71000E08F50000300320070002000EAD10200E8
:10B7200000000000E20F540009003A0060C0B300BE
:10B7300080F8B700060037008004EB0008FF3700F0
:10B74000301F2000800F5400A8FF3400A8FF3700EE
:10B750004F05BE004F04BE000080FA000000060046
:10B760000400FA00881F7800000478006000B80028
:10B7700091FD07008043EB00074378008742780083
:10B7800007427800874178000741780087407800B9
:10B79000074078000EC20200000000008040EB006D
:10B7A00000C1B3001AC10200000000008040EB009D
:10B7B00010C1B3001AC10200000000008040EB007D
:10B7C00040C1B3001AC10200000000008040EB003D
:10B7D00050C1B3001AC10200000000008040EB001D
:10B7E00020C1B3001AC10200000000008040EB003D
:10B7F00030C1B3001AC10200000000008040EB001D
:10B8000060C1B3001AC10200000000008040EB00DC
:10B8100070C1B3001AC10200000000008040EB00BC
:10B82000014078001AC10200000000008040EB00D7
:10B8300010C0B3001AC10200000000006140B8004F
:10B84000E80F5000E08F580056003E0000600100F5
:10B850000800370009003700130037000F003700D9
:10B860004D0037001400370024003700480037002F
:10B87000490037000000210048003700A0A5020061
:10B8800000000000F1F72F0080CD2000108860003C
:10B890009C28EF009E28EF000300370000102000D6
:10B8A00012890200000000004000200012890200FE
:10B8B000000000000E003700400020001289020046
:10B8C00000000000000120001289020000000000BA
:10B8D0008040EB00E0C1B3001AC10200000000008C
:10B8E000CE28EF00F1BF2F0080CD2000108860002F
:10B8F000AC28EF00AE28EF002A003700A0F929009D
:10B9000070A8020000000000E00F500020003A0084
:10B91000D0BF9F00E0BF9F0021002000668057003D
:10B92000FEA80200000000002100200064805700F3
:10B93000FEA8020000000000C0CA8000DFB8970027
:10B94000808F500004003A00D0CA8000EFB8970002
:10B95000808F50000B0032006000B800BEA80200CB
:10B9600000000000210020008095210046A902006F
:10B970000000000021002000A095210046A902003F
:10B98000000000000000EB0070A8020000000000B2
:10B99000AC28EF00AE28EF00400020001289020022
:10B9A000000000004F0478000080FA00000006004C
:10B9B0007E58EC007EF8B70041C6B300814F5000BE
:10B9C0002200360050C6B3007EF8B70000D8BF0092
:10B9D0000080FB000000EA004F00DE008000EB006A
:10B9E000E04F500005003200819021009140780026
:10B9F0008180FB008100E900CF08DE0008F9B70074
:10BA0000E08F500011003200A0C3800054FF0700F7
:10BA1000C0C38000E00F500002003A000040210047
:10BA200015003700A1C38000810F500004003A00C8
:10BA30000000EB0021FA07007438EF000300370024
:10BA40001EFA07007818F8007418F900DCE6020006
:10BA500000000000E00F500004003A00FCB50200B6
:10BA6000000000007000600006003200A0C38000EB
:10BA70003BFF070000402000128902000000000088
:10BA8000E9F83700A0C3800001002000E70F500054
:10BA9000E08F58005D003E000060010007003700A5
:10BAA0005400370054003700540037005700370067
:10BAB000530037005300370053003700FED7BF0054
:10BAC0000080FB000000EA004F00DE008000EB0079
:10BAD000E04F500005003200719021009140780045
:10BAE0008180FB008100E900CF08DE0007F9B70084
:10BAF000E08F5000040032008080EB00C0C3800063
:10BB0000B7F80700C0C38800FFD7BF000080FB0064
:10BB10000000EA004F00DE008000EB00E04F500024
:10BB20000500320061902100914078008180FB0087
:10BB30008100E900CF08DE0006F9B700E08F500071
:10BB4000040032008080EB00C0C38000A4F807002E
:10BB5000C0C3880001D8BF000080FB000000EA00DD
:10BB60004F00DE008000EB00E04F50000500320087
:10BB700051902100914078008180FB008100E90014
:10BB8000CF08DE0005F9B700E08F50000400320056
:10BB900011002000C0C3800091F80700C0C38800D6
:10BBA00002D8BF000080FB000000EA004F00DE006A
:10BBB0008000EB00E04F5000050032004190210072
:10BBC000914078008180FB008100E900CF08DE0011
:10BBD00004F9B700E08F500004003200110020008B
:10BBE000C0C380007EF80700C0C38800C0C38000C7
:10BBF0009FF83700A1FD370094FB370081FC370028
:10BC0000ACFA3700F5F93700C9F807000000060064
:10BC1000B0C388000000EB00A8F90700B0C38000A3
:10BC2000E00F5000020032007838EF0003003700C8
:10BC300010002000C0C388008DF80700B046200027
:10BC4000E488040000000000004020000A8902008F
:10BC500000000000800078000080EB00E08F5000C2
:10BC600001003200A0C38000000006000200FA00BC
:10BC7000F0BF9F0001017800CF80DE00E40F50008C
:10BC8000E08F580010003E00006001000400370003
:10BC900005003700060037000700370008003700AE
:10BCA000120888000E003700620888000C00370078
:10BCB000720888000A003700D208880008003700A0
:10BCC000E2088800060037008F81E900421020005A
:10BCD000014D200000E72900BEEB0200000000003B
:10BCE0000080FA00000006000200FA00F0BF9F008A
:10BCF000EA0F500019003E00120020000010DD0085
:10BD000082412000020160000D003A00000178002D
:10BD10006220B20003003A006100600015003A00A2
:10BD20000E003700E1806000C308DD00800880005D
:10BD30000030A10001007000800888000D0037006D
:10BD4000E1806000C308DD00F00880000030A10041
:10BD500001007000F0088800060037008F81E900BC
:10BD600042102000A146200000E72900BEEB02009F
:10BD7000000000000080FA00000006000200FA0047
:10BD8000F0BF9F0001017800CF80DE00EA0F500075
:10BD9000E08F580034003E00006001000A003700C8
:10BDA00011003700180037001F0037002600370049
:10BDB0002D0037002C0037002B0037002A003700F9
:10BDC0000900370018003700630161004410DD00EE
:10BDD00022088000F1FC2F000101610000017100C8
:10BDE0002208880026003700630161004410DD004E
:10BDF00082088000F1FC2F00010161000001710048
:10BE0000820888001E003700630161004410DD00D5
:10BE100092088000F1FC2F00010161000001710017
:10BE20009208880016003700630161004410DD00AD
:10BE3000F2088000F1FC2F00010161000001710097
:10BE4000F20888000E003700630161004410DD0035
:10BE500002098000F1FC2F00010161000001710066
:10BE600002098800060037008F81E9004210200097
:10BE7000214A200000E72900BEEB0200000000007C
:10BE80000080FA00000006000200FA00F0BF9F00E8
:10BE9000401ADE0005002000E90F500003003200C8
:10BEA000EA0F500007003A000300370062088800DC
:10BEB0007408880009003700D2088800E408880068
:10BEC000060037008F81E90042102000A14F2000BA
:10BED00000E72900BEEB0200000000000080FA002D
:10BEE00000000600E80F5000020034000000D000FF
:10BEF0007100500000000600800078001000200053
:10BF0000E88F500001003C000000EB00000006003C
:10BF10000200FA00889FBE008A1F7800C0BF9F0001
:10BF200000047800EC0F540006003600E88157004A
:10BF300042102000E115200000E72900BEEB0200BE
:10BF40000000000008007800E6FF07000005780008
:10BF5000E98221004250DD0000804400900078001A
:10BF60000110A1000100A00001087800080078007D
:10BF7000E1FF0700E00F5000040032000A00E80073
:10BF80004200DD00008044001000A0004F05780052
:10BF90004F04BE000080FA0000000600D1FF070039
:10BFA0004200DD000080E800C182210061007800CD
:10BFB00061006000000006000200FA00889FBE00D9
:10BFC000D0BF9F000104780080047800EC8F5400FB
:10BFD00004003600E681570042102000E1192000DD
:10BFE0000C00370009007800BEFF07004200DD00AA
:10BFF0000080E800C1822100610078000000D100CB
:10C000006140600006003A00E681570032102000CF
:10C01000211A200000E72900BEEB0200000000000A
:10C020006148B900EA0F5000E08F58002A003E0036
:10C03000006001000A0037000F00370014003700CD
:10C04000190037001E003700230037002200370098
:10C0500021003700200037000700370012003700AA
:10C060004F44DD002008800000F0A10008007000AF
:10C07000200888001C0037004F44DD008008800045
:10C0800000F0A1000800700080088800160037004A
:10C090004F44DD009008800000F0A100080070000F
:10C0A00090088800100037004F44DD00F008800041
:10C0B00000F0A10008007000F00888000A003700B6
:10C0C0004F44DD000009800000F0A100080070006E
:10C0D0000009880004003700E68157004210200064
:10C0E000511C2000CBFF37004F04BE000080FA0037
:10C0F000000006008000EB00AFFF370011002000B9
:10C10000ADFF37000200FA00F0BF9F00CF80DE00D5
:10C11000EA0F5000E08F580018003E000060010058
:10C120000A0037000C0037000D0037000F00370001
:10C130001000370011003700100037000F003700E3
:10C140000E003700030037000700370002088800A0
:10C150001000370043088800320888000D003700BF
:10C16000520888000B003700B3088800A208880036
:10C1700008003700C2088800060037008F81E900F8
:10C1800042102000D11E200000E72900BEEB020073
:10C19000000000000080FA00000006002F04B0003C
:10C1A000889FBE008A9FBE008C9FBE008E1F7800B5
:10C1B000D0A79F00E2A79F00F3A79F0081AF9F0039
:10C1C0006000B8006011B800909F9F00A19F9F0081
:10C1D000B29F9F00C39F9F000E0078000F0778005A
:10C1E0006E04B10001EA290007000900311F780040
:10C1F000000778005FA69700EC0F56000500360098
:10C20000A3FC2F008F81410042102000211020004C
:10C210000E0037000C00780032FF07008000780025
:10C22000C208DD008180E800C2822100E28078003F
:10C230008100D100E1C0600007003A00A3FC2F009C
:10C240008F814100321020006110200000E729009A
:10C25000BEEB0200000000008FA89700E08F5000A6
:10C2600013003200E38F500011003200E68F5000BF
:10C270000F003200E98F50000D003200E18F4000C6
:10C2800025003200E28F400023003200E38F40009F
:10C2900021003200E48F40001F00320003FD2F0018
:10C2A0008F81410052102000B1102000E7FF3700BD
:10C2B0006FA19700FFA19700929F9F00A39F9F00EF
:10C2C0000001EB00B29F9F00C29F9F008206780092
:10C2D000698710000E003700A40020000500200030
:10C2E0006033B8001F989700AF9897003F99970068
:10C2F000CF9997007A06020000000000909F9F00EF
:10C30000A19F9F00B29F9F00C39F9F008D06E800E2
:10C310008E8F5600F0FF3500E80F5600A1003C005C
:10C320008040EB000C0078006FFE07000FA997001B
:10C33000E00F5100880035001F9C9700AF9C9700CC
:10C340003F9D9700CF9D9700DAEA020000000000B1
:10C3500090B79F00A1B79F008003EB00B7B79F0085
:10C360000000EB00C0B79F001FB29700AFB297006C
:10C370003FB39700CFB397000440E10005C8E10048
:10C3800006D0E10007D8E1001F0039001F98970090
:10C39000AF9897003F999700CF999700D0AF9F0033
:10C3A000E1AF9F00F2AF9F0083B79F00DAEA02007F
:10C3B000000000000004BE004FB597008A05780019
:10C3C00004F02F00F50F20006033B8000800BE0015
:10C3D0000A01BE007A060200000000005FAA970072
:10C3E000EFAA97007FAB97008FB397000020E10082
:10C3F00001A8E10002B0E10003B8E10002003E0044
:10C400004FB697000600370023FB2F008F814100B5
:10C4100012102000D11120008CFF37000C06E8001C
:10C420001F989700AF9897003F999700CF99970072
:10C4300090B79F00A1B79F00B2B79F00C3B79F00FE
:10C44000DAEA0200000000004261DD00A3FB2F00D9
:10C450008F814100028141001202BE00D4B79F00CB
:10C46000E5B79F008002EB00F5B79F000003EB00EB
:10C4700086BF9F000004BE000A0020000B002000C1
:10C48000F4FF2F00050020006033B8000800BE0054
:10C490000A01BE007A060200000000005FB29700A9
:10C4A000EFB297007FB397008FBB97007A06020028
:10C4B000000000001FB29700AFB297003FB3970093
:10C4C000CFB397000020E10001A8E10002B0E10035
:10C4D00003B8E100D1FF3E001F989700AF98970086
:10C4E0003F999700CF99970090B79F00A1B79F0001
:10C4F000B2B79F00C3B79F00DAEA02000000000055
:10C500000004BE000FBD97008A0578005FB2970057
:10C51000EFB297007FB397008FBB97000800BE0073
:10C520000A01BE007A060200000000000203BE00FD
:10C530000002BE001FB09700AFB097003FB1970058
:10C54000CFB19700A2050200000000000205BE0066
:10C550000004BE000C0037006FA09700FFA09700FA
:10C56000E10F4000E08F580005003600C3FC2F00AB
:10C570008F814100121020007112200033FF37001C
:10C580000286EA000004BE008C0078005FA09700DD
:10C59000FAFD0700880078005FA09700B3FD070050
:10C5A0008C00370011C0B3000C007800CEFD0700EE
:10C5B0008FA89700E08F50007D0035001F9C9700EA
:10C5C000AF9C97003F9D9700CF9D9700DAEA02004D
:10C5D00000000000D0B79F00E1B79F008003EB0090
:10C5E000F7B79F000000EB0080BF9F005FB297008D
:10C5F000EFB297007FB397008FBB97000440E10034
:10C6000005C8E10006D0E10007D8E10020003900AC
:10C610001F989700AF9897003F999700CF99970080
:10C62000D0AF9F00E1AF9F00F2AF9F0083B79F00A4
:10C63000DAEA0200000000000004BE000FBD97000F
:10C640008A05780004F02F00F5FF2F00F60F200078
:10C65000070020000800BE000A01BE007A060200A2
:10C66000000000005FAA9700EFAA97007FAB970039
:10C670008FB397000020E10001A8E10002B0E100C3
:10C6800003B8E10002003E000FBF9700060037002C
:10C6900023FB2F008F81410012102000A1132000E6
:10C6A000EAFE37000E07E8001F989700AF98970042
:10C6B0003F999700CF999700D0B79F00E1B79F00AF
:10C6C000F2B79F0083BF9F00DAEA0200000000007B
:10C6D0000001BE004270DD00A1FB2F008F804000F2
:10C6E000008040001006BE000C00BE007A0402006C
:10C6F000000000000004BE000005EB008A05780081
:10C700000802BE000A03BE005FB09700EFB09700BA
:10C710007FB197008FB99700A205020000000000CA
:10C72000F4FF2F00F5FF2F006033B8000400E10094
:10C730000588E1000690E1000798E100D9FF3E007E
:10C740000800BE000A01BE0090B79F00A1B79F007D
:10C75000B2B79F00C3B79F001F9C9700AF9C970084
:10C760003F9D9700CF9D9700DAEA0200000000008D
:10C770000002BE004FB39700860378000800BE0099
:10C780000A01BE00A2050200000000000C02BE006B
:10C790004FB497000803780088037800A2050200D0
:10C7A000000000000205BE000004BE0003003700C8
:10C7B0000187EA006FA49700FFA497008E0078001D
:10C7C0005FA097006DFD07000801BE005FA0970005
:10C7D000ADFD07006011B8005FA0970049FE07009B
:10C7E0004F0778004F06BE004F05BE004F04BE0045
:10C7F0002F04B100000006000200FA00F0BF9F0005
:10C80000CF80DE00EA0F5000E08F580023003E008A
:10C81000006001000A0037000B00370010003700ED
:10C82000110037001B0037001C0037001B003700C9
:10C830001A00370019003700060037000C003700D7
:10C84000000880000100370030088000010020004F
:10C8500018003700320880004008800006003700CA
:10C8600050088000F9FF3700A0088000F7FF37006C
:10C87000A2088000B008800001002000C000DD0098
:10C880000000200003002000020070008380700080
:10C8900008003700C0088000ECFF37008F81E900F6
:10C8A000421020005121200000E72900BEEB0200C9
:10C8B000000000000080FA00000006000400FA00FA
:10C8C000E0BF9F00F1BF9F0001017800E10F510020
:10C8D000040036008F81E9006210200091222000C0
:10C8E0003E0037006FB89700CF80DE00EA0F50009F
:10C8F000E08F580036003E00006001000A0037005B
:10C9000012003700190037002100370028003700D7
:10C910002F0037002E0037002D0037002C00370085
:10C920000900370019003700610161000201410070
:10C93000200880000010A10002007000200888007C
:10C9400005A1A9002800370013A1A9006101610019
:10C9500002014100800880000010A1000200700068
:10C960008008880011A1A9001F0037006101610043
:10C9700002014100900880000010A1000200700038
:10C980009008880013A1A9001700370021A1A90071
:10C990006101610002014100F00880000010A10067
:10C9A00002007000F00888001FA1A9000E003700E7
:10C9B0006101610002014100000980000010A10036
:10C9C000020070000009880021A1A90006003700BC
:10C9D000E4815700421020001126200000E72900C2
:10C9E000BEEB0200000000000080FA00000006001C
:10C9F0000200FA00F0BF9F0001017800CF80DE0046
:10CA0000EA0F5000E08F58002F003E000060010048
:10CA10000A00370010003700160037001C003700EE
:10CA20002200370028003700270037002600370093
:10CA3000250037000800370015003700610161004C
:10CA40004611DD00200880000060A1000200700097
:10CA50002008880022003700610161004611DD00D6
:10CA6000800880000060A10002007000800888003B
:10CA70001B003700610161004611DD009008800055
:10CA80000060A100020070009008880014003700C8
:10CA9000610161004611DD00F00880000060A10026
:10CAA00002007000F00888000D003700610161008D
:10CAB0004611DD00000980000060A1000200700046
:10CAC00000098800060037008F81E900421020002D
:10CAD0004129200000E72900BEEB02000000000011
:10CAE0000080FA00000006000400FA00889FBE00E3
:10CAF0008A1F7800B0BF9F0001057800C2BF9F0069
:10CB000080047800EC8F540004003600EA8157005E
:10CB100042102000812A2000070037004FBC9700F8
:10CB20000800E900E60F500006003600E8815700D3
:10CB300022002000912A200000E72900BEEB02001D
:10CB40000000000009007800E6FC07004200DD005C
:10CB5000C28221000A3178006148B900EA0F500012
:10CB6000E08F58003C003E00006001000A003700E2
:10CB7000130037001C003700240037002D00370059
:10CB800035003700340037003300370032003700FB
:10CB90001500370027003700670464004C40DD00B3
:10CBA00028058000F1FF28000104640000047400DF
:10CBB000280588008460A9009460A8002A00370036
:10CBC000670464004C40DD0038058000F1FF280058
:10CBD00001046400000474003805880084E0A900A2
:10CBE00094E0A8002000370067046400410580003D
:10CBF00080FF2F0000806000080470004805880056
:10CC00008500A9009500A80017003700670464009C
:10CC10004C40DD0088058000F1FF2800010464001D
:10CC200000047400880588008760A9009760A80048
:10CC30000D003700670464009105800080FF2F001D
:10CC40000080600008047000980588008780A900B3
:10CC50009780A80004003700EA81570042102000A6
:10CC6000D12E2000B4FF37004F0578004F04BE00DE
:10CC70000080FA00000006000200FA00F0BF9F00EA
:10CC8000CF80DE00EA0F5000E08F58002A003E00FF
:10CC9000006001000A0037000F0037001400370061
:10CCA000190037001E00370023003700220037002C
:10CCB00021003700200037000D0037001800370032
:10CCC000A00480004300DE00610060009460A800C2
:10CCD0008460A8001E003700A00480004700DE002A
:10CCE0006100600094E0A80084E0A800180037000C
:10CCF000A00480004800DE00610060009500A800EC
:10CD00008500A80012003700B00480004B00DE0050
:10CD1000610060009760A8008760A8000C003700E1
:10CD2000B00480004C00DE00610060009780A80025
:10CD30008780A800060037008F81E900421020009C
:10CD4000F133200000E72900BEEB020000000000E4
:10CD50000080FA00000006000200FA00F0BF9F0009
:10CD6000CF80DE00EA0F5000E08F58001E003E002A
:10CD7000006001000A0037000C0037000E00370089
:10CD80001000370012003700170037001600370078
:10CD90001500370014003700070037000C0037007B
:10CDA000200480004300DE000B00370020048000D8
:10CDB0004700DE0008003700200480004800DE0045
:10CDC00005003700300480004B00DE000200370011
:10CDD000300480004C00DE00610060000080FA003A
:10CDE00000000600060037008F81E9004210200095
:10CDF0001137200000E72900BEEB02000000000010
:10CE00000200FA00F0BF9F0001017800CF80DE0031
:10CE1000EA0F5000E08F580038003E00006001002B
:10CE20000A003700110037001A00370021003700D0
:10CE30002800370031003700300037002F0037005E
:10CE40002E00370013003700220037002004800036
:10CE50004300DE0061006000610161004311DD00FC
:10CE6000210480000130A100070037002004800069
:10CE70004700DE0061006000610161004711DD00D4
:10CE8000210480000170A1008280700021048800CC
:10CE900020003700200480004800DE0061006000B0
:10CEA000610161004811DD00210480000180A100C2
:10CEB000F5FF3700300480004B00DE0061006000A9
:10CEC000610161004B11DD003104800001B0A1005F
:10CED00007003700300480004C00DE006100600075
:10CEE000610161004C11DD003104800001C0A1002E
:10CEF0008280700031048800060037008F81E900CD
:10CF000042102000613B200000E72900BEEB020038
:10CF1000000000000080FA00000006000200FA0095
:10CF2000F0BF9F00CF80DE00EA0F5000E08F580076
:10CF30001B003E00006001000A0037000C003700B3
:10CF40000E003700100037001200370014003700C1
:10CF500013003700120037001100370007003700B8
:10CF60000C0037009460A9008460A900120037000B
:10CF700094E0A90084E0A9000F0037009500A90003
:10CF80008500A9000C0037009760A9008760A90000
:10CF9000090037009780A9008780A90006003700A4
:10CFA0008F81E90042102000913F200000E7290016
:10CFB000BEEB0200000000000080FA000000060046
:10CFC0000600FA00889FBE008A9FBE008C9FBE00AC
:10CFD000F0B79F008106780000057800EC0F55003F
:10CFE00004003600F281570042102000210C20007E
:10CFF000100037000A00780082BF9F0093BF9F0097
:10D00000B8FB0700000678004264DD000880E800F5
:10D01000C182210061027800614262000FB997006D
:10D020009FB9970006003A00F281570022102000B5
:10D03000610C200000E72900BEEB020000000000A8
:10D04000EB82210008844500980478000910A000B4
:10D050000900A100090C78000A00780082BF9F0037
:10D0600093BF9F00A4FB07000FB997009FB99700DB
:10D07000E00F5000060032000C00E8004200DD0026
:10D08000008045001000A1001820A0000200370019
:10D090000920A100090C78007FB0970082BF9F0093
:10D0A00093BF9F009DFF07008D0078000FB9970088
:10D0B0009FB997007FB0970038FC07008000EB0015
:10D0C0007FB09700FDFD07008000EB007FB0970068
:10D0D00047FE07004F06BE004F05BE004F04BE00CE
:10D0E0000080FA00000006000200FA00F0BF9F0076
:10D0F000CF80DE00EA0F5000E08F58001B003E009A
:10D10000006001000A0037000B0037000C003700F8
:10D110000D0037000E0037001400370013003700F1
:10D1200012003700110037000300370006003700F7
:10D1300021088000070037008108800005003700C3
:10D140009108800003003700F108800001003700DB
:10D1500001098000C408DE00E380600000042000B4
:10D16000E28F500007003A000D0037008F81E90080
:10D17000421020009142200000E72900BEEB02008F
:10D180000000000000102000E38F50000400320077
:10D1900080002000E18F50000100320010002000CC
:10D1A0000080FA000000060090089000E001900066
:10D1B00001814000630179008100E90011089800B5
:10D1C00002007800000006000200FA00889FBE00FE
:10D1D0008004780001047800E08F540003003A00D6
:10D1E00000002800000064006000370000002400F8
:10D1F000E00F54005A0032000802780001003D00A0
:10D200000802EA0009007800E08F540001003D00A8
:10D210000900EA00CF80DE0066815700811F780098
:10D22000110009004488D80001097800CF00780077
:10D230005FB9970003002000C011DD00020020004C
:10D24000809FBE00110009004499D80000017800B9
:10D250004F00BE0001002000C000DD0000002000E3
:10D260000300200002007000838070000181CF0065
:10D27000E00F5100030032000402200002025200BD
:10D28000040037000082CF00E00F5200010032009E
:10D2900070021200EC02520009003B00C22820007C
:10D2A000030020007A04020000000000440BDD00AF
:10D2B0004C00DE0000007300CC88DE002400370044
:10D2C0001200200003002000040378000603E90098
:10D2D000030033000201410083814900FBFF370056
:10D2E0000200500083805800680252000402E900E6
:10D2F000030033008180D1000080D300FBFF3700A2
:10D30000FF0060004580DE00C32ADD00050140000B
:10D310000200410006FC280066007800030220009D
:10D32000018251000482B9000201E80002014100BB
:10D33000660079000180B9000000420081804A0047
:10D34000811F7800110009004308D800CF00780041
:10D35000E00F540002003D00010028000080500052
:10D36000E08F540001003C000000EA004F04BE00C2
:10D370000080FA0000000600889FBE008A9FBE0061
:10D380008C1F780000017800E00F51000C003D0078
:10D3900001002C00810F510003003D000000280017
:10D3A000000041000400370010002800810F5100E8
:10D3B000290032000200EA001A00200008003700AD
:10D3C00000002400800F51000300340000002800FA
:10D3D0000200500001003700020078000005EB0059
:10D3E000C780DE0000017800F207B20081814000B2
:10D3F000E0EB2800E08579000C08200002065600CA
:10D400008100E8008180400060807800CF80DE00ED
:10D41000CF91DE007A040200000000000004BE008C
:10D420006162B9006159B9000400BE007A040200CB
:10D430000000000008004000898048004909DD0024
:10D440004700DE0000007100C788DE00E00F5500D5
:10D45000010032000000EA004F0678004F05BE00D0
:10D460004F04BE000000060001002400010040003F
:10D47000C1FF37000100240001003700C288DE0030
:10D48000808F5000FDFF3C00000178000000EB00A1
:10D4900007003700808140000080D100830F5100D9
:10D4A000020035000301510001004000C288DE0087
:10D4B000E08F5000F7FF3A0000000600889FBE0092
:10D4C0008A9FBE0080027800010078008001EB0096
:10D4D0004A00200059002000180037000A01B80057
:10D4E000811F7800110009004999D800CF00780009
:10D4F0000001EB00820178000D003700820341003B
:10D50000878342001703780004024200048242002D
:10D5100014047800880553004240A9000300340039
:10D52000880B7800060A7800130020000201E8004A
:10D5300000024100810F5200F0FF3900E10F50005E
:10D54000E6FF3E00E08F5100E9FF3A004F05BE00C4
:10D550004F04BE0000000600889FBE008A1F7800AE
:10D5600000047800080078000FFF0700000578002D
:10D57000080078000CFF070080047800080078009D
:10D5800009FF07008000EB0007003700C80190008A
:10D590000A0145000982440064B179000A05E800E7
:10D5A0008904E8008100E800808F5000F7FF39000F
:10D5B0004F0578004F04BE0000000600889FBE00A3
:10D5C0008A1F78000004780008007800F6FE070043
:10D5D0008004780008007800F3FE0700000578005A
:10D5E00008007800F0FE07008000EB000A05450007
:10D5F00005003700C8019000098144006AB1790034
:10D600008904E8008100E800808F5000F9FF3900AC
:10D610004F0578004F04BE0000000600889FBE0042
:10D620008A9FBE000004780008007800DEFE070034
:10D630000005780008007800DBFE07008004780011
:10D6400008007800D8FE0700800578000800780000
:10D65000D5FE0700C80090008B85450061817D00E4
:10D660008000EB0009003700C80290008A014500E5
:10D6700083814200098244000482420094094100EF
:10D680000A05E8008904E8008100E800808F500066
:10D69000F5FF39004F05BE004F04BE000000060034
:10D6A000889FBE008A9FBE000004780008007800B2
:10D6B000BDFE07008005780008007800BAFE07006C
:10D6C0000005780008007800B7FE070080047800A5
:10D6D00008007800B4FE07008000EB000D00370062
:10D6E000480190008B81450083014100098244007C
:10D6F000040241008A02450005014100140278003D
:10D70000920942008B05E8000A05E8008904E80058
:10D710008100E800808F5000F1FF39004F05BE0006
:10D720004F04BE0000000600889FBE008A9FBE0016
:10D7300000047800080078009BFE07008005780050
:10D740000800780098FE07000005780008007800BF
:10D7500095FE0700800478000800780092FE07001C
:10D760008000EB000D003700480190008B814500E0
:10D77000830141000A0245000402410089824400FD
:10D780000501410014027800920952008B05E8005F
:10D790000A05E8008904E8008100E800808F500055
:10D7A000F1FF39004F05BE004F04BE000000060027
:10D7B000889FBE008A9FBE000004780008007800A1
:10D7C00079FE0700800578000800780076FE0700E3
:10D7D000000578000800780073FE070080047800D8
:10D7E0000800780070FE07008000EB000C00370096
:10D7F000480290008B824500898144000A0145005F
:10D80000E4817900640179000299B90002B27A00DA
:10D810008B05E8000A05E8008904E8008100E800BB
:10D82000808F5000F2FF39004F05BE004F04BE004C
:10D8300000000600889FBE008A9FBE008C9FBE002D
:10D840008E1F7800000478000800780056FE07005C
:10D85000800578000800780053FE07000005780076
:10D860000800780050FE0700800478000800780067
:10D870004DFE0700800678000006EB001C00370014
:10D88000C80090000A00450061007800098144004A
:10D8900061017900CF91DE00E00F5100E08F590067
:10D8A0000B0032000A05E8008904E8000B874500F8
:10D8B0000E874000CF80DE002C0402000000000034
:10D8C000000F78008B05E8000C06E8000800370020
:10D8D00023002000730498007001440071002900A7
:10D8E0000800780082C50200000000000200370036
:10D8F0008D0F5600E2FF39004F0778004F06BE003B
:10D900004F05BE004F04BE0000000600889FBE0009
:10D910008A9FBE00000478000800780022FE0700FD
:10D9200080057800080078001FFE070000057800D9
:10D93000080078001CFE07008004780008007800CA
:10D9400019FE07008000EB000F003700480190002F
:10D950008A014500E28179000A05E80089824400D5
:10D960008904E8000B8245000402410062817A00CC
:10D97000830F51000100340003017800020A78008F
:10D980008B05E8008100E800808F5000EFFF390030
:10D990004F05BE004F04BE0000000600889FBE0079
:10D9A0008A9FBE000004780008007800FEFD070092
:10D9B0008005780008007800FBFD0700000578006E
:10D9C00008007800F8FD070080047800080078005F
:10D9D000F5FD07008000EB000F00370048019000C4
:10D9E0008A014500E28179000A05E8008982440045
:10D9F0008904E8000B8245000402410062817A003C
:10DA0000830F510001003D0003017800020A7800F5
:10DA10008B05E8008100E800808F5000EFFF39009F
:10DA20004F05BE004F04BE0000000600889FBE00E8
:10DA30008A9FBE008C1F78000004780008007800E0
:10DA4000D9FD07000006780008007800D6FD070021
:10DA50008005780008007800D3FD070000057800F5
:10DA600008007800D0FD07008004780008007800E6
:10DA7000CDFD07008001EB0014003700C8009000C6
:10DA80000B814500610279008B05E8000A01450021
:10DA9000E10279000A05E80009814400610179008A
:10DAA0008904E800820F520004003C000501780060
:10DAB000840F510001003D00040178000C02460073
:10DAC00082307A000C06E8008301E800808F510064
:10DAD000EAFF39004F0678004F05BE004F04BE0034
:10DAE00000000600889FBE008A9FBE008C9FBE007B
:10DAF0000004780008007800ABFD0700800478007F
:10DB000008007800A8FD070080067800080078006B
:10DB1000A5FD070000067800480590000800780081
:10DB2000A1FD07000001780002014100EA0579002B
:10DB3000080078009CFD0700000578000002200026
:10DB4000808F550005003C000D0378008C007800A4
:10DB50008003EB006011B8000F0037004800900010
:10DB60008984440089044000800CEB0014003700D5
:10DB700001804000650278008100E8000600430053
:10DB8000650078000603E8000482B9000201420043
:10DB900083814A008703E800C80290008A8F5300FF
:10DBA000F3FF3900898444008B05E900030033004A
:10DBB0008381D1000281D300FBFF370082B27C0059
:10DBC0004F06BE004F05BE004F04BE000000060019
:10DBD000889FBE008A9FBE008C1F780000047800DA
:10DBE0000800780070FD07008004780008007800C5
:10DBF0006DFD070000067800080078006AFD070048
:10DC0000800578000800780067FD070000057800AF
:10DC10000800780064FD070000017800E00F510063
:10DC2000250032004802900009804400E401780099
:10DC30000903E8006118B9000C06460003327E00B3
:10DC40008B8445004802900003B27C00170020003E
:10DC50001000370086014300E48179000603E800E4
:10DC60000C024200948F510001003D00030A78002D
:10DC70004802900009024200948F510001003400D4
:10DC8000030A7800611AB9000000420081804A004E
:10DC90008703E80048029000828F5300EDFF3900AF
:10DCA0000A0545000A054200030020002C0402007A
:10DCB00000000000000D78004F0678004F05BE0000
:10DCC0004F04BE0000000600889FBE008A9FBE0071
:10DCD000000478000800780033FD07008005780014
:10DCE0000800780030FD0700000578000800780083
:10DCF0002DFD070080047800080078002AFD070049
:10DD000000027800E00F5200160032000B0178008C
:10DD10008000EB0005002800F0FF27000A05450001
:10DD2000898444004803900082014100E681790023
:10DD30000201E800808F510002003D0001337D00A8
:10DD400003007800858F510003003400C802900062
:10DD500081B27C00830278008100E800848F50004B
:10DD6000F0FF39004F05BE004F04BE000000060062
:10DD7000889FBE0000047800080078000AFD0700B4
:10DD8000800478000800780007FD07008000780014
:10DD9000898444004800900009004000C7FD070046
:10DDA0004F04BE0000000600E8874700889FBE00C1
:10DDB0008A9FBE008C9FBE008E1F780000057800F1
:10DDC0000A007800F8FC0700000778000A007800D5
:10DDD000F5FC0700800678000A007800F2FC0700D6
:10DDE000000678000A007800EFFC07008005780044
:10DDF0000A007800ECFC0700800378000003EB00C9
:10DE00002A003700CA0090000D80460061027800A9
:10DE10000C004600610078000B8145006104790028
:10DE2000CFC4DE00E00F5400E08F5C00170032002A
:10DE30008D06E8000C06E8008B05E8000E0147009F
:10DE400002814000E2B79F00CF80DE00CFA2DE005B
:10DE50000401BE00F6B79F0087BF9F007A0402004E
:10DE6000000000000801BE002C04020000000000B9
:10DE70006FB19700000978000E07E8007FB39700A4
:10DE80000603E8008FBB970008003700230020003E
:10DE90007305980070014500710029000A007800A0
:10DEA00082C502000000000002003700870F530007
:10DEB000D4FF39004F0778004F06BE004F05BE0063
:10DEC0004F04BE008F00B10000000600889FBE0016
:10DED0008A9FBE008C9FBE008E1F780000047800D1
:10DEE00008007800B0FC0700800578000800780082
:10DEF000ADFC07000005780008007800AAFC0700C8
:10DF00008004780008007800A7FC0700000778006C
:10DF10000006EB000C003700C80690000A00450020
:10DF20006D0078000A05E80089804400ED807800E3
:10DF30008904E800A4FC07008B80450080B67800C7
:10DF40008B05E8000C06E8008E0F5600F2FF390042
:10DF50004F0778004F06BE004F05BE004F04BE00BD
:10DF600000000600889FBE008A9FBE008C9FBE00F6
:10DF700000047800080078008BFC0700000578009A
:10DF80000800780088FC070080047800080078000A
:10DF900085FC0700000678008005EB0009003700CB
:10DFA000C8069000098044006D0078008904E800EC
:10DFB000F1FC07008A00450080B678000A05E800F9
:10DFC0008B05E8008C8F5500F5FF39004F06BE0029
:10DFD0004F05BE004F04BE0000000600889FBE0033
:10DFE0008A9FBE008C9FBE00000478000800780065
:10DFF0006DFC070000057800080078006AFC070047
:10E00000800478000800780067FC070000067800AC
:10E010008005EB0009003700C80690000980440025
:10E020006D0078008904E8000FFD07008A004500B4
:10E0300080B678000A05E8008B05E8008C8F550053
:10E04000F5FF39004F06BE004F05BE004F04BE006D
:10E0500000000600EE874700889FBE008A9FBE0032
:10E060008C9FBE008E1F7800000778000E0078009D
:10E070004DFC0700E0B79F000E0078004AFC070047
:10E08000000478000E00780047FC0700CE049000E2
:10E0900088004400698678000804E8000804440009
:10E0A00069037C00000040006904780008007800E3
:10E0B00086BF9F00ECFC0700000578000800780090
:10E0C000ADFC070000047800EFB09700018040002D
:10E0D00000804400D0B79F00CFE6DE00CFD5DE0041
:10E0E0000A01BE000C00BE007A040200000000001D
:10E0F000B0B79F00C1B79F000FBB9700CFB3DE0042
:10E10000CFC4DE000801BE000600BE0086BF9F002F
:10E11000F7B79F007A040200000000000002BE0072
:10E120003FB09700CFB0970004025000858258009E
:10E13000C128DD004F22DE0004827000CFAADE007D
:10E140005FB1970004097800EFB197000300E80081
:10E150004E07900000004000000747000A01BE0083
:10E160000FBB9700FFB397000600BE007A040200C1
:10E17000000000000005BE000801BE000C00BE004B
:10E180007A040200000000000A0040008B80480072
:10E190004109DD004F00DE0000007100CF88DE0085
:10E1A000000F78004F0778004F06BE004F05BE00F5
:10E1B0004F04BE00EF00B10000000600889FBE00C3
:10E1C0008A9FBE008C9FBE00000478000800780083
:10E1D000F5FB07000005780008007800F2FB070057
:10E1E0008004780008007800EFFB07000006780044
:10E1F0008005EB0009003700C80690000980440044
:10E200006D0078008904E8009AFC07008A00450048
:10E2100080B678000A05E8008B05E8008C8F550071
:10E22000F5FF39004F06BE004F05BE004F04BE008B
:10E2300000000600889FBE008A9FBE008004780010
:10E2400009007800D8FB0700000478000900780076
:10E25000D5FB07000005780009007800D2FB070015
:10E260008005780009007800CFFB07008001780066
:10E27000490190008B854500E2837D008000EB0022
:10E28000070037008100E800838F5000040036004B
:10E2900008044400080141000009EB004F0037006A
:10E2A0000A8040000000400062007800E00F50004B
:10E2B000F4FF3A00010078000B0037008100E8000D
:10E2C000838F50000800360008044400E00F50001F
:10E2D0003A0032000000E900870F50003700390093
:10E2E0000000D1003C0037000A82400004024200D6
:10E2F00062027A00E00F5200F0FF32000003EB00F0
:10E3000006007800060278008402780003003700D7
:10E310008502E800838F52000B00310081844200A7
:10E32000809FBE00110009008384D800810478001A
:10E330004F00BE008A84440089844400E2847C004B
:10E34000E08F5400F2FF3A0084845200808F540022
:10E3500003003400048242000483D10009007800E5
:10E36000838F520005003900110037000402E800D5
:10E37000830F5200020039000D00370005027800BB
:10E3800081024200809FBE00110009008382D800F4
:10E39000810278004F00BE008A82420085824200DE
:10E3A000E2827A00E08F5200D7FF3A00EFFF370099
:10E3B00008044400870F500003003D00080441009A
:10E3C000008CEB00050037008100430011000900BC
:10E3D0008380D8008000FD0000317C004F05BE0026
:10E3E0004F04BE0000000600F07F88000000060019
:10E3F00050252600F17F80000088B900926123003B
:10E4000000004100F07F880000000600889FBE00E9
:10E410008A9FBE008C1F78000004780008007800F6
:10E4200061FB070080047800080078005EFB0700AD
:10E43000800578000005EB000700370009804400E4
:10E440004806900000064600E9FF0700000E78002D
:10E450008904E8000A05E8008B0F5500F7FF390032
:10E460004F0678004F05BE004F04BE0000000600B6
:10E47000AA24AB000D00320032828000924090004E
:10E4800000C8B30080CF500007003A0080828000AF
:10E490009040900040C8B30080CF500002003A0086
:10E4A0006840400010419800AA24A90000082000FC
:10E4B00050248800000006000103210091407800EC
:10E4C00000C8B30080CF50002F003A0000CCB3004A
:10E4D0005CF0B70033D0BF00E24F500008003200BC
:10E4E000E34F500017003200E14F500025003A0082
:10E4F00000122100D0828800200120001D0037007A
:10E5000032D0BF000080FB0000004000E11B210072
:10E51000E1007800D1828800D0828000801F7800DE
:10E52000204090005EF0B7004F007800D08280005D
:10E53000801F7800304090005FF0B7004F007800F7
:10E540000000060032D0BF00E24F50000B003E003A
:10E5500032D0BF000080FB0000004000011C210001
:10E56000E1007800D1828800D082800010407800DD
:10E570000080FB00F0828800000006005C70EF0065
:10E58000000006005C70EF00000006003870EF002D
:10E590003970EF0030D0BF007F006000E10F500005
:10E5A0000B003200E20F50000B003200E00F500071
:10E5B0001B003A005CF0A8003810A800108480000E
:10E5C000E10F500016003A003830A8001400370060
:10E5D0005CF0A800120037005CF0A80034D0BF0047
:10E5E0000500330034D0BF006F0060000000400021
:10E5F000A10421000400370034D0BF006F00600088
:10E6000000004000010521006100780010409000EA
:10E61000640060000200320010C0B30038F0B700A0
:10E620005CF0AB000500320080032100D08288003E
:10E630005C10A80020C0B3005EF0B7000000060028
:10E64000F082800081C0B300E70F50000A003E0056
:10E65000F182800056D0BF0002003A0010C0B30023
:10E660000400370056D0BF00E14F500002003A00CE
:10E6700020C0B30056F0B7000180FB005E30B5004B
:10E680008082800001487800800321004083880058
:10E690005C10AB00070032000F003700D082800012
:10E6A000428380003059780042838800D0828800FD
:10E6B0008140E900E0CF5000F8FF3A00000006007A
:10E6C000D0828000428380003059780042838800E5
:10E6D000D08288008140E900E0CF5000F8FF3A0086
:10E6E00000000600881F78008082800010047800F7
:10E6F0004E44DE00614464005050AA000082800055
:10E70000E80F50000A003A0032D0BF000080FB0042
:10E71000B0248800B0248000E00F500002003200D6
:10E720000001200001003700400020000082880026
:10E7300058D0BF00E14F500011003A008003210083
:10E740008182800090009800BDFF070061052100D4
:10E750009140780080828000E2CF500002003A00B1
:10E7600041C8B3000400370081CCB300E04F54002F
:10E770000100320081C8B300114098001200370038
:10E7800062D0BF000F003B0065D0BF000080FB00DF
:10E790006106210091407800C808DD00008070000B
:10E7A0000700320065D0BF000080FB006106210039
:10E7B00091407800C808DD00008070000000010072
:10E7C00062F0A9005870EF004F04780000000600C6
:10E7D0000080FB000181FB000000400000014100BF
:10E7E0004311DD00030021000301410012F0A100EC
:10E7F000E0CF500002003A00A104210001003700E0
:10E80000010521008230780012E0A100640141007E
:10E8100012E0A000000006000001EB002284880046
:10E82000820078004007200056E702000000000048
:10E830008284A90000012000002488000000060056
:10E840008284A800000120005024880010002000CD
:10E85000208488000001EB008000EB0050072000BE
:10E8600056E70400000000000200FA00881F78004C
:10E8700032D0BF00E14F50000B003A0030D0BF0053
:10E880007F40600008003A005CF0A80031D0BF0073
:10E89000E34F500003003A0010002000108488006D
:10E8A000010037008230EF0032D0BF008E003A0006
:10E8B00030D0BF007F406000E24F50008A003A0035
:10E8C00034D0BF006F4060008700320034D0BF00FA
:10E8D0006F006000E20F500083003C000182800066
:10E8E00000022000808F50007F003A005CF0A800FA
:10E8F00034D0BF000A00330034D0BF006F00600086
:10E9000000004000A1042100E1007800E1BF9F0069
:10E9100034D0BF006F0060002107210009003700DC
:10E9200034D0BF006F0060000000400001052100EE
:10E93000E1007800E1BF9F0034D0BF006F006000AD
:10E94000E1062100614478006140640004003A005F
:10E950004FF897000024A100C0FF9F00030037007C
:10E96000CFF897000124A000C1FF9F0034D0BF0062
:10E970000500330034D0BF006F006000000040008D
:10E98000A10421000400370034D0BF006F006000F4
:10E9900000004000010521006FB997008230780027
:10E9A00031D0BF00E34F500018003A006FB8970015
:10E9B0008000EB00908F10000E003D0034D0BF00AF
:10E9C000050033004103210091407800EF80600092
:10E9D0002207210004003700410321009140780004
:10E9E000EF806000E206210062C078000014A00001
:10E9F00000F17800EFB897001141900040C8B300D3
:10EA00000040710090409800370037004FF99700A0
:10EA10000224A200C2FF9F00EFB8970011409000AF
:10EA20000001EB00910F110008003D000074A100EF
:10EA30000064A000904098002200200050002000B8
:10EA400056E7020000000000020037000064A0004A
:10EA5000904098004FF897000024A200C0FF9F004C
:10EA60006244640006003A006FB897000240280034
:10EA70001001610001002800810F510017003A00C9
:10EA800034D0BF00050033004103210091407800DD
:10EA9000EF806000220721000400370041032100BD
:10EAA00091407800EF806000E206210062C07800AB
:10EAB0000014A10000F17800EFB897001140900019
:10EAC000B043B20090409800220020005000200087
:10EAD00056E702000000000003003700904090005D
:10EAE000B143B200114098004F0478000080FA0052
:10EAF000000006005CF0A800AC24EF00AE24EF009C
:10EB00000040EB00020021008081FB000100210099
:10EB1000C219DD00830141008009EB00B3117800C8
:10EB20000040E800EB4F5000F7FF36009424A800A7
:10EB30004470EF009424A90068804000808288001F
:10EB4000318288004182880032D0BF0042F0B70095
:10EB500042D0BF0002003A0000012000060037004A
:10EB600012002000210421001000200056E70200BE
:10EB70000000000000022000008288000000060063
:10EB800030D0BF000046B20035003A0031D0BF009F
:10EB90000080FB0001002000EB0F5000E08F5800C8
:10EBA0002F003E0000600100130037001300370003
:10EBB0002B0037001100370029003700060037000E
:10EBC000090037002100370009003700070037002F
:10EBD0000B003700140037005CF0A8008000200014
:10EBE000008288000000060033FE3700C1FF3700B6
:10EBF000200421000600370064FE37001AFF3700AA
:10EC000034D0BF000080FB0041042100010040001F
:10EC1000D08288005C10A80010C0B3005EF0B7007E
:10EC20005CF0A800000006005CF0A80034D0BF0033
:10EC30000080FB0041042100821F78002203210094
:10EC4000927078004F017800000006000001EB0090
:10EC50008000EB002000200056E7020000000000CA
:10EC6000000006009EC0A9008EA4EF008AA4EF0059
:10EC7000AA24EF00AC24EF00AE24EF002000200017
:10EC800030258800A824EF008644A900F009200060
:10EC900080248800602488008804A80001002100E6
:10ECA0004808DE00C02488000040EB000081FB0023
:10ECB0004211DD00028140000009EB0032117800B2
:10ECC0000040E800EB4F5000F8FF36009424A80005
:10ECD0009624EF0094A4A9009424A90080002000A9
:10ECE00009003700502488005C70EF006270EF006C
:10ECF00031062100914078006370EF004106210049
:10ED0000914078006470EF0051248000E88060003A
:10ED1000F4FF3A0010002000C0838800D0838800F0
:10ED2000E1838800F1838800218488000140780015
:10ED300005052100A40421000081FB00820141009F
:10ED400003834200000BEB00830142008009EB00CB
:10ED5000E306210081717900230721008171790088
:10ED60000040E800E24F5000F3FF36008000210031
:10ED700080828800D00020005025880000032100F8
:10ED80001080880080C0B30000F0B70040C8B30016
:10ED900001F0B7004270EF004030EF0000000600C5
:10EDA000C0838000E00F500024003A0011002000D2
:10EDB000C1838800D0838000E00F50001F003A001C
:10EDC000D18388008205210012417800E24F510072
:10EDD00006003A00818280008048780080CCB30031
:10EDE000818280009040980000000600820521008A
:10EDF00012417800E14F510010003A000084880071
:10EE000080C0B300328280000049780034828000E4
:10EE1000030321001302980042C8B3001242980075
:10EE2000018488004182800080487800418280000F
:10EE30009300980000C8B3009040980000000600BE
:10EE4000308280009040780063D0BF000080FB00DB
:10EE500042062100124178004811DD0000007100D7
:10EE60000181FB00800F51000300360031062100B4
:10EE70009140780064D0BF0063D0BF000080FB00E9
:10EE800042062100124178004811DD0000007100A7
:10EE90008181FB00030050003206210012417800FE
:10EEA00063F0B7004800DE004206210012417800FE
:10EEB00064F0B7000040EB001600370002062100A6
:10EEC000124178000281FB00130621009341780073
:10EED000C819DD000082FB0002817100830321005C
:10EEE00063597A0003062100934178000001FD0078
:10EEF00060F0B7000001FD004811DE00130621009C
:10EF0000934178000001FD0061F0B7000001FD00B1
:10EF10000040E800814F5000E8FF390063D0BF0097
:10EF20000080FB004106210091407800C808DD0008
:10EF300000807000418280000E00320080C0B3006B
:10EF400080487800408280008103210011009800F1
:10EF500001002400328280009280600002003A00AA
:10EF600081CCB3000100370081C8B3001140980084
:10EF70000000060080C0B300804878004182800015
:10EF8000000321009000980040C8B3009040980012
:10EF900065D0BF000080FB00610621009140780031
:10EFA000C808DD00008070000700320065D0BF0097
:10EFB0000080FB006106210091407800C808DD0058
:10EFC000008070000000010062F0A900B0838000A2
:10EFD000E00F500001003A0071FF0700000006003A
:10EFE00058D0BF00E24F500001003A0094FF3700B4
:10EFF0005870EF0000848000E00F500009003A00D4
:10F0000080C0B30041828000804878004182800047
:10F010000003210090009800C0C8B3009040980001
:10F02000000006008030EF00000006007C30EF009A
:10F030007E30EF0058D0BF00E24F500005003A008C
:10F0400080C0B30041828000804878004182800007
:10F050001200370036D0BF000080FB007103210092
:10F0600091407800C808DD0000807000F2828000C6
:10F07000820F50000700310036D0BF000080FB0037
:10F080007103210091407800C808DD000080700005
:10F09000F08288006AFD07008182800080032100E1
:10F0A0009000980080CCB3009040980000000600CB
:10F0B00094A4A9005CF0AB0017003A0062D0BF0036
:10F0C00009003B0020C0B30058F0B700F083800077
:10F0D000E00F500001003A00D4FF07007A30EF0043
:10F0E0007830EF000000060080C0B300418280004D
:10F0F0008048780041828000000321009000980041
:10F10000C0C8B300904098006840500081828000E1
:10F11000904098000000060030D0BF000C003B007B
:10F1200010C0B30058F0B700E0838000E00F50003B
:10F1300001003A00BDFF07007A30EF007830EF00A1
:10F14000B0838000E00F500011003A0014FF370038
:10F1500020C0B30058F0B70080C0B30041828000E7
:10F1600080487800418280000003210090009800D0
:10F1700040C8B300904098007A30EF007830EF003C
:10F18000B0838000E00F500001003A0004FF070048
:10F1900000000600881F78005670EF000004EB00A6
:10F1A000B8838800E8838800F88388000884880092
:10F1B0000800780058F0B70081828000114090006C
:10F1C0000074A10090409800010521001124A200C4
:10F1D00082828000124090000074A10010419800CB
:10F1E0001124A20041828000114090000074A1000F
:10F1F00090409800080078005CF0B700F882880022
:10F200000800780062F0B70063D0BF000800780003
:10F2100063F0B70064D0BF000004FD0064F0B700E5
:10F220000004FD0056FE0700080178008200780007
:10F230003000200056E70200000000009CFF07009D
:10F240004F04780000000600D0C2B30086F0B7007B
:10F250006CD0BF00B00FB20020003A00C106210000
:10F26000914078008181FB00C219DE004219DD0067
:10F27000040021008400410031828800418288001E
:10F280004850AA006402790002C023000202620012
:10F2900002402300820F52000F003A0091029000BA
:10F2A0000082FB00020321009542780005717A007C
:10F2B000110290000402E800940098000040E80069
:10F2C000E74F5000F5FF3600C219DD002000210095
:10F2D00002B07900AFFF370041FF37006CD0BF00AC
:10F2E000B00FB200E80F500001003A00FDFC07002B
:10F2F00000000600889FBE008A1F78000044780046
:10F30000814478000985FB00680065000300320035
:10F310008040EB00084078002DFD07006405650083
:10F320000300320011C0B3000840780028FD070038
:10F330000884FB0008044400A04A200009707C00F7
:10F340004F0578004F04BE0000000600E04F50005B
:10F350000C003A0080C0B3004182800080487800F1
:10F36000418280000003210090009800C0C8B300D3
:10F370009040980068405000818280009040980042
:10F38000000006008180FB000080FB0000004000C0
:10F39000008040004300DD00040021000401400023
:10F3A0009241900041C8B30081C17100134198009F
:10F3B0006400400004004000104190008140710052
:10F3C0001140980000000600804278000582FB0092
:10F3D000E0CF50000300320004024200000521008B
:10F3E0000200370004024200A004210060007A00FD
:10F3F000E00F50001500320012009800034878001A
:10F40000104190000244B2001240980090419000D8
:10F4100082C8B30002C17100124098000581FB0050
:10F42000E0CF50000500320002014100010521003B
:10F43000010141001224A200000006000201410067
:10F44000A1042100010141001224A20000000600D5
:10F4500094A4AB00180032000080FB0000004000C4
:10F4600001052100E10278001501BE00040420001E
:10F470000201620003002000828ABE00E1027800DF
:10F480000204200003002000951A6900959269008B
:10F49000010140001224A200E10178001341900014
:10F4A0000244B20092419800E100780011409000BF
:10F4B0000440680090409800000006000000EB0047
:10F4C000A0248800602488000082880000000600D4
:10F4D00000828000E00F500010003A00A024880055
:10F4E0006024880021002000312588004025880004
:10F4F0008644A900F0092000802488006024880048
:10F500009EC0A800010037009404A8009404AB003A
:10F51000FDFF32001000200000828800000006007D
:10F52000627E2400F10F200012C86000124190009A
:10F5300012409800827E240092816000234098004F
:10F540001241900032409800A27E24009280600018
:10F55000414098001241900052409800917F240051
:10F560009140780061409800A17F2400914078008C
:10F5700071409800B17F24009140780001489800C4
:10F58000C17F24009140780011489800C17E24007A
:10F590009140780021489800D17E24009140780065
:10F5A00031489800E17E240091407800414898005D
:10F5B000F17E24009140780051489800017F24009A
:10F5C0009140780061489800117F240091407800B4
:10F5D00071489800417F24009140780001509800C4
:10F5E000517F24009140780011509800317F240011
:10F5F0009140780021509800717F2400914078005C
:10F6000031509800817F240091407800415098004B
:10F6100000000600889FBE008A9FBE008C9FBE002F
:10F620000004BE000C4020000D0020000006460033
:10F6300081864E00FAFF2F00FB0F200008003700E4
:10F640000800BE00D2BA0200000000008A0F50007D
:10F650008B8F580007003A0062044400E0844C009D
:10F660008C0F54008D8F5C00F5FF39000000EB001B
:10F6700001003700100020004F06BE004F05BE00FD
:10F680004F04BE00000006000001EB001102210043
:10F69000000120006CEA020000000000810120004F
:10F6A000607E240078EA020000000000B4EA020054
:10F6B000000000008000780010002000E27F24009D
:10F6C000928F5000010032000000EB0000000600A5
:10F6D0002E00FA0023FD2F008F814100D20220006E
:10F6E00026BB020000000000100020009FA8970029
:10F6F000E38F5000010032000000EB000080FA00B0
:10F70000000006001600FA00889FBE008A9FBE0017
:10F710007E044000E08448000A4020000B002000E6
:10F720000005450081854D000A003700FE81570025
:10F73000520120000800BE0026BB020000000000AD
:10F740000FE897006100600006003A006E04440074
:10F75000E0844C008A0F54008B8F5C00F3FF39006B
:10F760006044B8000800BE004F05BE004F04BE0054
:10F770000080FA00000006001600FA00889FBE0014
:10F780008A9FBE008C1F7800000678000205BE002C
:10F790008C017800D20220000A00BE0026BB0200C5
:10F7A000000000000C6890000040E800006E980027
:10F7B0007E044500E0844D00004020000100200050
:10F7C0000A0540008B854800CA00370003FE2F0061
:10F7D0008F814100520120000800BE0026BB0200BC
:10F7E00000000000CC6090006FE0970000C0700047
:10F7F00040669800DC6090007FE0970000C07000D9
:10F8000050669800EC6090000FE8970000C0700010
:10F8100060669800FC6090001FE8970000C07000D0
:10F8200070669800CFF097008180FB002C619000FB
:10F830000281FB003C6090004800DD000200700087
:10F8400000804000206698004800DE003066980086
:10F85000BFF097008180FB000C6190000281FB00EB
:10F860001C6090004800DD00020070000080400035
:10F87000006698004800DE0010669800AFF0970020
:10F880008180FB006C5990000281FB007C58900045
:10F890004800DD000200700000804000605E9800BB
:10F8A0004800DE00705E98009FF097008180FB00AA
:10F8B0004C5990000281FB005C5890004800DD002C
:10F8C0000200700000804000405E98004800DE00AA
:10F8D000505E98008FF097008180FB002C599000BB
:10F8E0000281FB003C5890004800DD0002007000DF
:10F8F00000804000205E98004800DE00305E9800E6
:10F90000FFE897008180FB000C5990000281FB000A
:10F910001C5890004800DD0002007000008040008C
:10F92000005E98004800DE00105E9800EFE8970047
:10F930008180FB006C5190000281FB007C509000A4
:10F940004800DD0002007000008040006056980012
:10F950004800DE0070569800DFE897008180FB00C9
:10F960004C5190000281FB005C5090004800DD008B
:10F970000200700000804000405698004800DE0001
:10F9800050569800CFE897008180FB002C519000E2
:10F990000281FB003C5090004800DD000200700036
:10F9A00000804000205698004800DE003056980045
:10F9B000BFE897008180FB000C5190000281FB00A2
:10F9C0001C5090004800DD000200700000804000E4
:10F9D000005698004800DE00105698004C499000F0
:10F9E0000281FB00DC499000C819DD000280710033
:10F9F0006C4990000281FB00FC499000C819DD00B1
:10FA0000828071002FB1970002004000E080480022
:10FA1000404E98004801DE00524E9800614E98001A
:10FA20004808DE00704E98000C4990000281FB00EF
:10FA30009C499000C819DD00028071002C4990009B
:10FA40000281FB00BC499000C819DD008280710072
:10FA50001FB1970002004000E0804800004E98006F
:10FA60004801DE00124E9800214E98004808DE0042
:10FA7000304E98004C4190000281FB00DC41900028
:10FA8000C819DD00028071006C4190000281FB000A
:10FA9000FC419000C819DD00828071000FB1970011
:10FAA00002004000E0804800404698004801DE0027
:10FAB00052469800614698004808DE00704698005B
:10FAC000AFE897008180FB002C4190000281FB0091
:10FAD0003C4090004800DD000200700000804000C3
:10FAE000204698004800DE00304698006E0444002E
:10FAF000E0844C008A0F54008B8F5C0033FF390088
:10FB00004F0678004F05BE004F04BE000080FA008B
:10FB1000000006003200FA00889FBE008A9FBE00E7
:10FB20008C1F78000004BE00E00F5100E08F5900E8
:10FB300008003A000E0078000F0778008E03B1002D
:10FB400015000900001FEB00005FEB0000077800C4
:10FB50000300370080FC2F000F00400006FF070065
:10FB600030002000C0A79F000800BE00A9FE0700CB
:10FB7000E00F5000030032000800BE0084BB02000A
:10FB8000000000000005EB00CC02200051FC2F001B
:10FB90008F8040008105E8001000370081FC2F00B5
:10FBA0008F8040000A804000B0407800C1C79F00AD
:10FBB000B0407800D1C79F00904D78002FA19700EA
:10FBC000BFA197000800BE00C0BB020000000000FB
:10FBD00062044400E0844C00630545008C0F55002E
:10FBE000EEFF36004F0678004F05BE004F04BE0002
:10FBF0000080FA000000060000C023001100200071
:10FC0000B3FE0700E00F500014003A00000024008B
:10FC100011002000AEFE07006011B800E00F500098
:10FC2000080032000000240011002000B5FE07008B
:10FC3000E00F5000E08F580028003A000200240036
:10FC40001300200000C0230011002000B1FF0700B6
:10FC5000E0C12300110020000000060000C02300C6
:10FC600011002000A7FE0700E00F5000E08F5800B1
:10FC70001A003A00000024001100200094FE070042
:10FC8000E00F500008003A0002C0230013002000DB
:10FC900000002400110020009EFF0700E001240066
:10FCA00011002000000006000000240011002000C8
:10FCB00094FE0700E00F5000E08F580007003A0064
:10FCC000020024001300200000C0230011002000C7
:10FCD00090FF0700E0C12300110020000000060093
:10FCE0001A00FA00889FBE008A9FBE008C1F780011
:10FCF0000005EB00F028200081458000808F500037
:10FD00002E003400BCFF07000004BE000BFE2F00D5
:10FD10008F8545000B00780001FE0700D0FD2F0005
:10FD20000F0040000006E8000E0037008A80450002
:10FD300031407800C0DF9F0031407800D0DF9F0065
:10FD4000114E78006FA99700FFA997000800BE0028
:10FD5000C0BB02000000000062044400E0844C00CC
:10FD600063054500F40F5500F0FF36000200240043
:10FD700013002000820F5400838F5C0006003A00BD
:10FD800002C02300130020000800BE0061FF07002E
:10FD90001A002000090037001A0020000440240047
:10FDA00015002000840F5400858F5C0003003A008A
:10FDB00000C023001100200056FF07000A00780051
:10FDC0004F0678004F05BE004F04BE000080FA00C9
:10FDD00000000600303F8200E10F400002003200C8
:10FDE000617E24008008E800245E0200000000001C
:10FDF000E00F500006003D00717F240011407800A4
:10FE0000E14F40000A0032008048E8000800370057
:10FE1000E8004000627E2400E2C07800E1CF4000AC
:10FE2000030032008140E800680141000171780060
:10FE30008464AB000F003200DCE60200000000002A
:10FE4000E00F500006003200403F8200E10F40000A
:10FE500008003200817E24008008E80000000600CF
:10FE6000503F8200E10F400002003200A17E2400DA
:10FE70008008E800000006000080FB00C300DE00F0
:10FE8000927F240002814000C308DD000100500081
:10FE9000110020000008DD0012497000000006007B
:10FEA00061052000810F50000B0039008100E8003F
:10FEB000810F500004003600F0804000810F500098
:10FEC00005003A000200370070C0B300EAFF3700B7
:10FED00000C1B300E8FF0700000006002106200073
:10FEE000810F500011003E008180E900810F500019
:10FEF0001D003100F1032000810F500007003E007B
:10FF0000E6805000810F500015003100A002B100C2
:10FF1000E40F50001C003E000F0037000005B10048
:10FF2000E50F500018003E000D003700510620007C
:10FF3000810F500004003E008100E900810F500055
:10FF40000D0031000A00370061062000810F5000CB
:10FF50000D003A000A003700F0C0B3000700370078
:10FF600080C0B30005003700E0C0B30003003700D5
:10FF700090C0B3000100370010C1B300BEFF3700CE
:10FF800000C1B300BCFF0700000006000100200014
:10FF90007B005000E0805800EF0F5000E08F5800C9
:10FFA0001F003E00006001000F0037000E00370008
:10FFB0000D0037000E0037000F0037000E0037002D
:10FFC0000D003700080037000D0037000E00370025
:10FFD0000D0037000E0037000D0037000C00370011
:10FFE0000F0037000C003700A0C0B3000900370035
:10FFF000D0C0B30007003700C0C0B3000500370011
:020000040001F9
:1000000020C1B30003003700B0C0B30001003700C7
:1000100030C1B30098FF370070C1B30096FF0700EE
:100020000000060012CD800023CD80006100410059
:10003000E080490010CD880021CD880002302A00E0
:1000400023002000820F5000838F580007003A00E1
:10005000A239EF00A439EF00817F2400114078001D
:10006000E14F4000010032008048E8000000060037
:100070000001EB0011022100000120006CEA0200E7
:100080000000000081012000607E240078EA020068
:1000900000000000B4EA020000000000F03F8A0007
:1000A0000000060020C0B30073FF3700A019EC0069
:1000B00000CD880001A62E00810F500002003A00FA
:1000C000A039EF0043FF070000000600889FBE0034
:1000D0008A1F780050778000617780008004EB00F1
:1000E00018002000EAFF2F00910F100033003600A7
:1000F00074003700880044000100400010005500E3
:1001000001002000F00F5000E08F580022003E0058
:1001100000600100100037000F0037000E003700AC
:100120000D0037000C0037000B0037000C003700C3
:10013000190037000C0037000B0037000C003700A7
:1001400015003700100037000B0037000C00370097
:100150000F0037000E003700F0C0B3000D0037006D
:1001600080C0B3000B003700E0C0B30009003700C7
:1001700000C1B3000700370010C1B300050037000D
:1001800070C0B3000300370040C1B3000100370066
:1001900050C1B30038FF07008800E8000100780074
:1001A000EC0EB4000001780062807800808F54006B
:1001B00001003100800478000884E8006077800046
:1001C000900F5400CBFF39003A0037006177800070
:1001D00008004400610078004C01DE0003002000AC
:1001E000ED0F5100E08F590030003E000260010029
:1001F0000D0037002D003700190037000D003700C3
:100200000F003700110037001300370027003700B8
:1002100026003700140037001100370016003700A1
:10022000200037001A003700890F54001F003900E2
:10023000240037000A00600028FF07001B00370079
:100240000A00600016FF0700180037000A0060006F
:1002500022FF0700020037000A00600010FF0700BD
:100260000884E800140037004400DD004480DE000C
:1002700008004000070037000800E80000004000C8
:100280006100780015FF0700630444000A0037008E
:100290000A006000808F5400040031008004780060
:1002A000020037000A00600038FF07000804E80079
:1002B00001003700FAFF200050778000800F5400C3
:1002C000C2FF39004F0578004F04BE000000060051
:1002D000D17E240011407800E14F4000010032003F
:1002E0008048E80079FF3700E7FC0700E00F500086
:1002F00003003A00607E24000C0009000018EB00A7
:100300004027AB000300320010C0B300DAFE070044
:100310004027A900807F24008040EB0090CF100090
:1003200004003A00313F8200005A2000808F5000C4
:10033000060036006AFE0700E00F5000030032009E
:10034000607E24000C0009000018EB00C17E240030
:1003500011407800E14F4000010032008048E80081
:10036000000006001C00FA00889FBE008A9FBE00A5
:100370008C1F7800000678005C019000EC01900072
:100380000C0078000E4C02000000000008C02300A2
:1003900019002000FA3F24001B0020000800BE00C6
:1003A000D2BA020000000000E0AF9F00F1AF9F0052
:1003B000A3FD2F008F81410032002000C1FD2F00DE
:1003C0008F8040000C0078008C4902000000000083
:1003D0005FA89700E30F500025003A006204440034
:1003E000E0844C008A0F54008B8F5C00EBFF3600DA
:1003F00000FE2F000F00400049FC0700A3FD2F0066
:100400008F8141005201200001FE2F008F804000AB
:100410000C0078008C49020000000000607E24007F
:100420000C0009000018EB0000C0230011002000A0
:1004300078FC0700E00F50000400320000C02300E9
:100440001100200084BB0200000000000000240016
:10045000110020006FFC0700E00F50000400320084
:10046000000024001100200084BB020000000000F6
:100470004F0678004F05BE004F04BE000080FA0012
:1004800000000600C1C68000E08F5000130032005B
:10049000DED8EC00DEF8B700FF4F50000400340057
:1004A000E3806000C1C6880000CEB300DEF8B7006C
:1004B000C0C68000E00F500008003200E18D21002E
:1004C000914078008100FB0001003B008100EA00C0
:1004D000E0C0B3001AC102000000000010C0B30069
:1004E000C1C68000E08F5000030032000040EB00E6
:1004F0008000EB0005003700A193210091407800B7
:100500008180FB008100E900CF08DE003AF9B700E6
:10051000E08F5000040032008040EB00E0C0B300E8
:100520001AC102000000000000000600889FBE0003
:100530000000EB0002C2B300E17F2100E14178003E
:10054000218E2100E0CF510007003200E141780008
:10055000E3C141008370780082CF51000300360070
:100560008270780001003700837078000000E80096
:10057000E40F5000F0FF3400E4D8BF000B0032005D
:100580000802200039022000418E210091407800AD
:10059000084078001AC10200000000000804E800CA
:1005A000890F5400F8FF34001C003700218E210011
:1005B00091407800E0CF50000300320010C2B30039
:1005C0001AC1020000000000318E21009140780025
:1005D000E0CF50000300320020C2B3001AC1020075
:1005E00000000000518E210091407800E0CF5000C3
:1005F0000300320000C2B3001AC102000000000074
:10060000618E210091407800E0CF5000030032005D
:1006100030C2B3001AC10200000000000000EB006D
:10062000218E210091407800E0CF500004003A0074
:10063000E4D8BF000080FB000000E9004F00DE00AE
:100640008000EB00E04F50000500320021942100B3
:10065000914078008180FB008100E900CF08DE0036
:1006600042F9B700E08F5000040032008040EB00F8
:1006700010C2B3001AC10200000000000000EB002D
:10068000318E210091407800E0CF500004003A0004
:10069000E4D8BF000080FB000000E9004F00DE004E
:1006A0008000EB00E04F5000050032001194210063
:1006B000914078008180FB008100E900CF08DE00D6
:1006C00041F9B700E08F5000040032008040EB0099
:1006D00020C2B3001AC10200000000000000EB00BD
:1006E000518E210091407800E0CF500004003A0084
:1006F000E4D8BF000080FB000000E9004F00DE00EE
:100700008000EB00E04F5000050032000194210012
:10071000914078008180FB008100E900CF08DE0075
:1007200040F9B700E08F5000040032008040EB0039
:1007300000C2B3001AC10200000000000000EB007C
:10074000618E210091407800E0CF500004003A0013
:10075000E4D8BF000080FB000000E9004F00DE008D
:100760008000EB00E04F500005003200F1932100C3
:10077000914078008180FB008100E900CF08DE0015
:100780003FF9B700E08F5000040032008040EB00DA
:1007900030C2B3001AC10200000000004F04BE00C6
:1007A000000006002AD9BF000080FB000000E9001D
:1007B0004F00DE008000EB00E04F500005003200EB
:1007C00081942100914078008180FB008100E90044
:1007D000CF08DE0048F9B700E08F50000400320077
:1007E0008040EB00D0C1B3001AC10200000000003D
:1007F0002AD9BF00050032002A79EF0001C2B300F8
:10080000D0C1B3001AC102000000000000000600C1
:10081000881F7800EA58EC00EAF8B700EA4F500069
:1008200023003A00EA78EF003146800050092000AA
:10083000808F500006003C008040EB0060C2B30097
:100840001AC102000000000001C2B3001500370009
:1008500080112000808F50000600340001C2B300D8
:100860006E4040001AC10200000000008040EB0012
:100870000C0037006109B100C508DD002208200026
:10088000110009008200D80080007800014478003F
:1008900060C2B3001AC102000000000001C2B30030
:1008A00088C0500070C2B3001AC1020000000000EE
:1008B0004F04780000000600889FBE0029248000B5
:1008C000E884640041003200088E2100184478005A
:1008D000E04F54000E003A008840780050C0B3004A
:1008E0001AC10200000000008840780060C0B30018
:1008F0001AC10200000000008840780070C0B300F8
:100900001AC102000000000010C0B300E0F8B700F8
:10091000E1D8BF0012002000010032000001FB00FE
:1009200071C0B300EA0F510007003C002300200013
:10093000801F7800110009000301D80080007800B2
:100940004F0078008140E80000C04000E1F8B700A7
:1009500041C6B300814F500015003400DF58EC0051
:10096000DFF8B70011C0B3008000FD00E1F8B70068
:100970008000FD00E34F500001003A00DF78EF00F7
:10098000F88D210018447800E04F540008003A0028
:100990008840780070C0B3001AC102000000000057
:1009A0008840780060C0B3001AC102000000000057
:1009B000DFD8BF0065404000118E210091407800D3
:1009C0001AC1020000000000B0003700804580001E
:1009D000B208B400883E20000880B900A8F82000C2
:1009E000809FBE00110009004888D80000047800EC
:1009F0004F00BE00E0D8BF00270032000900780099
:100A0000E0F8B70050182000800F54000A003600AC
:100A100001C2B30050C0B3001AC1020000000000C0
:100A200001C2B30060C0B3001AC1020000000000A0
:100A300001C2B3001500370080162000800F54005B
:100A40000600360001C2B30050C0B3001AC1020054
:100A50000000000001C2B30008003700401520006C
:100A6000800F54000C00360001C2B30050C0B30028
:100A70001AC10200000000008940780060C0B30085
:100A80001AC10200000000008940780070C0B30065
:100A90001AC102000000000010C0B300511820006D
:100AA000810F540003003E000040EB008000EB008B
:100AB00005003700E1932100914078008180FB0020
:100AC0008100E900CF08DE003EF9B700E08F50005A
:100AD0000C00320001C2B30050C0B3001AC10200C2
:100AE0000000000001C2B30060C0B3001AC10200E0
:100AF0000000000001C2B30070C0B3001AC10200C0
:100B00000000000071E92F008880400010C0B30091
:100B1000F78F5000030036000040EB008000EB0030
:100B200005003700D1932100914078008180FB00BF
:100B30008100E900CF08DE003DF9B700E08F5000EA
:100B40000C00320001C2B30050C0B3001AC1020051
:100B50000000000001C2B30060C0B3001AC102006F
:100B6000000000008040EB0070C0B3001AC102001A
:100B700000000000B1EA2F008880400010C0B300E0
:100B8000EE8F5000030036000040EB008000EB00C9
:100B900005003700C1932100914078008180FB005F
:100BA0008100E900CF08DE003CF9B700E08F50007B
:100BB0000C00320001C2B30050C0B3001AC10200E1
:100BC000000000008040EB0060C0B3001AC10200CA
:100BD000000000008040EB0070C0B3001AC10200AA
:100BE0000000000010C0B30041152000810F540028
:100BF000030036000040EB008000EB0005003700EA
:100C0000B1932100914078008180FB008100E900D0
:100C1000CF08DE003BF9B700E08F5000080032003B
:100C20008040EB0060C0B3001AC102000000000069
:100C30008040EB0070C0B3001AC102000000000049
:100C400040152000800F540010003E00E158EC00D9
:100C5000E1F8B700E34F500004003A0001C2B300CE
:100C600050C0B3001AC1020000000000E1D8BF006C
:100C7000E54F5000050034008040EB0050C0B30049
:100C80001AC1020000000000E178EF004F04BE002E
:100C900000000600FED7BF000080FB000000EA0055
:100CA0004F00DE008000EB00E04F500005003200F6
:100CB00071942100914078008180FB008100E9005F
:100CC000CF08DE0047F9B700E08F50000300320084
:100CD00020002000EAD1020000000000FFD7BF0082
:100CE0000080FB000000EA004F00DE008000EB0007
:100CF000E04F5000050032006194210091407800DF
:100D00008180FB008100E900CF08DE0046F9B700D2
:100D1000E08F50000300320020002000EAD10200E2
:100D20000000000000D8BF000080FB000000EA00C7
:100D30004F00DE008000EB00E04F50000500320065
:100D400051942100914078008180FB008100E900EE
:100D5000CF08DE0045F9B700E08F500003003200F5
:100D600030002000EAD102000000000001D8BF00DE
:100D70000080FB000000EA004F00DE008000EB0076
:100D8000E04F50000500320041942100914078006E
:100D90008180FB008100E900CF08DE0044F9B70044
:100DA000E08F50000300320020002000EAD1020052
:100DB0000000000002D8BF000080FB000000EA0035
:100DC0004F00DE008000EB00E04F500005003200D5
:100DD00031942100914078008180FB008100E9007E
:100DE000CF08DE0043F9B700E08F50000300320067
:100DF00020002000EAD102000000000000000600F0
:100E0000889FBE008A9FBE008C1F78000000EB0008
:100E1000238621000285210091032000808040006C
:100E20008180400004802000E480780000024000BF
:100E3000E3027A00818F520001003D0081317A0087
:100E4000E08F50000500320000024000E2027A000C
:100E5000818F52000100340001317A000000E80067
:100E6000E60F5000ECFF34004045800081C3800055
:100E7000808F500001003D0080C3880050458000F5
:100E800091C38000808F500001003D0090C3880016
:100E90000004EB000C0220008BFA2900080144003A
:100EA00000852100E0007900900320000800400048
:100EB00000004000038020006300780023862100AA
:100EC00063057900010555000100500001003B0059
:100ED0000000EB000C80B900809FBE0011000900EB
:100EE0004A08D800000578004F00BE00EB447C00A3
:100EF0008A407800094078001AC102000000000012
:100F0000E20F540005003A008944E8008A40780066
:100F1000094078001AC10200000000000804E8003F
:100F2000E60F5400DDFF340082C38000404580009E
:100F3000E00F500001003D000000EB00080220001F
:100F40000880B900811F7800110009004208D8000C
:100F5000CF0078008040780060C1B3001AC1020061
:100F60000000000093C38000524580000800780014
:100F7000E00F510001003D000001EB000090B900BE
:100F8000811F7800110009004308D800CF007800C5
:100F90008040780070C1B3001AC102000000000058
:100FA0004F0678004F05BE004F04BE00000006004B
:100FB000889FBE0020468000F40F50003D003C009A
:100FC0001146800000468000E46802000000000036
:100FD00022002000110009000200D800037D20003B
:100FE00003014000F1F92000C8012000810F5100E9
:100FF0001C0036000277210002024000B8012000E8
:10100000810F5200170036000471220004024000D4
:10101000A8012000810F520012003600046B23004B
:101020000402400098012000810F52000D0036009C
:1010300088012000F5D52600850F520009003E00EA
:10104000830150006C044400818F5100050036007C
:1010500002005000F8012000810F500001003E0006
:101060006604440029468000E08F540001003D00E2
:101070008904EA00F48414008984440001003B00E0
:101080008004EB0040C78000E00F500003003500F3
:101090008040EB001AC10200000000008940780087
:1010A000084078001AC102000000000048C788000C
:1010B0000700370040C78000E00F500003003500F4
:1010C0008040EB001AC1020000000000E8B8EF0009
:1010D0004F04BE0000000600FFD7BF00FE57B70058
:1010E0000158B7000258B70008003200EBD8BF0023
:1010F00006003200FCB50200000000000002B20051
:101100000200320028B7020000000000F17F210039
:101110009140780002D8BF00E37F210013C1700026
:1011200003802100134171001380210013417100DD
:10113000004171000281FB000201E9004F11DE0055
:101140000001FD00EBF8B7000001FD00E0CF50000A
:1011500013003200E04F500011003200EC58EC0058
:10116000ECF8B70041C6B300814F50000D003600C7
:101170008140E800814F500006003A00FCB50200B3
:10118000000000000002B20002003A0020B7020096
:101190000000000060C6B300ECF8B70000000600D5
:1011A000EC78EF000000060067006000C800DD007A
:1011B000F2058000F08F2F00000061000100700038
:1011C000F005880000000600881F78000004780001
:1011D000E0C68000E00F500002003A008AC0A9007B
:1011E0009AC0A80000002100000064000500320041
:1011F000FCB50200000000006100600001003A0040
:1012000008C0A10008007800DC38B7004F0478005F
:1012100000000600DC18B600000006008AC0A80026
:10122000000006008080EA008000FD00DC38B60087
:101230008000FD0001002100010060000600320076
:10124000FCB50200000000000002B2000200320003
:1012500028B7020000000000E0C68000E00F500048
:1012600001003A009AC0A90000000600A28D2100EA
:1012700012417800DC98AB00180032007146800003
:10128000E08F50000B0032000080FB00810F500007
:10129000030034004300DE00804F5100030039009A
:1012A000E04F5100060032000240E900DAF8B700D2
:1012B000030037008000FD00DAF8B7008000FD0071
:1012C000A18D210091407800814F51000300320030
:1012D000E0C1B3001AC102000000000000000600D7
:1012E000818D2100E00F500003003D006700600089
:1012F00091087000000006000080EA00910860007C
:1013000000000600881F780000047800611BB80008
:101310000002EB00F10F5300E08F5B0064003E0021
:10132000066001001100370012003700130037007B
:101330001400370015003700160037002B00370067
:1013400030003700310037003200370033003700FB
:10135000360037003A0037003D00370040003700C4
:1013600043003700470037004A003700020ADD001B
:101370004F003700028ADE004D00370001024100B5
:101380004B00370002825000490037000192B9003B
:1013900047003700E00F51000F003A0020052800F9
:1013A000E00F50000400320082007800080078004E
:1013B0005280020000000000230020007304980007
:1013C00070014400710029000800780082C5020005
:1013D0000000000029003700000278001100090019
:1013E0008200D8000002FD0031003700801F780025
:1013F000110009008200D800010278004F00780037
:101400002B0037000102710029003700010269003A
:10141000270037000102610025003700140020007A
:10142000828F500015003A002100370002816800C9
:101430000202EA00020172004F12DE001C003700B7
:1014400014002000828F500019003C000B00370070
:1014500014002000828F500015003D000700370067
:1014600014002000828F5000110035000300370067
:1014700014002000828F50000D0034000002EB00A9
:101480000B00370014002000E08F500003003200F2
:1014900007003700E08F5000040032000202EA002B
:1014A000020272004F22DE000100370001027800C4
:1014B000040078004F04780000000600E18F50001F
:1014C0000400320005003900E28F500007003A00A6
:1014D00004003700E00F500005003D000000EA0066
:1014E000000006000080EA00000006000000EB009B
:1014F000000006008000EB000108980071009800D1
:101500002118980020019000010978003001900016
:101510000201410040009000560704000000000056
:10152000200190009201780010002000090037008F
:101530000002400062027A00810F520004003A006B
:101540000000E80000004000620078000000060093
:101550000080E800830F5000F5FF3900000005000F
:101560000600FA00889FBE008A1F780000047800F9
:10157000A80090000808900000014000E1047900F4
:101580004C49DE0003002000EE0F5100E08F5900AF
:10159000F1003E00026001000E003700110037002C
:1015A00019003700220037002D00370038003700BF
:1015B0004B003700750037007E0037008E00370083
:1015C00091003700B7003700C8003700D00037005F
:1015D000DA003700780090000000A1007004980045
:1015E000DD003700E8009000180890000000E800D7
:1015F000100C980000004000C44CDD00C4CCDE009C
:1016000089307800BE003700E8019000180990008A
:101610000201E800120C9800020141000000E800FD
:1016200000004000610078008031790054003700EC
:1016300068019000180890000000E800100C980065
:1016400000004000F1FF200081846400C800900089
:1016500089844400E1847C0009317800A8003700C7
:1016600018089000F1FF2000818464004801900078
:1016700089844400E801900080004000E380780005
:1016800001B17C000000E900100C98009C003700BC
:101690000001E80002014100E10179001809900011
:1016A00002014100E80090000281400092007800B1
:1016B000838F500003003900A0BF9F00B3BF9F007D
:1016C00015003700F0FF200080846400898040000E
:1016D0004800900081804000608978002800370031
:1016E0000001E800020141006101790068029000F8
:1016F000980890008101E90083814100E48179002C
:1017000081804000E4807800828F5000130039000F
:10171000A0BF9F00B2BF9F00C1BF9F00200020005C
:1017200070049800630020006C815700610029005C
:101730000800780082C50200000000002005280093
:10174000E00F5000840032008000EB0008007800B9
:1017500052800200000000007F003700F0FF2000F0
:1017600080846400898040004800900081804000AF
:1017700003B07800180890000080E900100C980071
:10178000080890000080E8005F003700180D900006
:101790000A054500680090000A05400089007800AD
:1017A000F10FB2001A00780044FF0700000D780026
:1017B00053003700E8009000180890000001400036
:1017C0000000E900000040008981FB006101790010
:1017D000E100780008007800CAFE07009808900031
:1017E0008100E900110C98006801900081804000A0
:1017F00000B1780042003700C44CDD00C4CCDE00EC
:101800000080440040003700E80090001808900075
:10181000000140000000E900000040008981FB0059
:1018200061017900E100780008007800B5FE07004A
:10183000980890008180E900110C980088089000B9
:10184000E00F5000050032000930B20022002000F5
:1018500003302000838F540006003A00A801900056
:101860000101E8000201410063017900E00F50002E
:101870000500320081804000280090008100400077
:101880001190A0000300370081804000818041005A
:101890001190A1000808900002014000020C98007D
:1018A0002D0037000081E80002014100E1017900CC
:1018B0000000E800000040006101780002014100E2
:1018C0004800900002014000F1FF20008180640088
:1018D000838141000800780082C5020000000000FA
:1018E000080890006300400007003700F1FF200067
:1018F000818064000800780008AB0200000000004E
:10190000080890000000E800000C98001200370062
:1019100068019000980890008100E800110C980080
:1019200081804000810041008008E800F0FF200035
:1019300080846400090C98000700370018089000A4
:101940006801900080004000E2807800010C98005F
:101950000000E900100C98004F0578004F04BE000D
:101960000080FA00000006000000FA00889FBE0018
:101970008A9FBE008C9FBE0080047800810578009D
:101980000F0678000B0078006607020000000000D8
:1019900000047800E3064400650044000000A10054
:1019A000808747000C05780020052800E00F5000D4
:1019B000040032008B007800090078005280020099
:1019C0000000000020002000F004980009089000AA
:1019D000000D780028459800630045000801780054
:1019E0008B00780046070200000000008D0178009F
:1019F0000A017800910029000900780082C50200E0
:101A0000000000008C0778004F06BE004F05BE00A6
:101A10004F04BE000080FA00000006008000EB00CA
:101A20000B0037006A81400002014100600179002B
:101A300080099000830F510004003A00F0009000EC
:101A40000110A00071009800100005008100E8005E
:101A500020199000828F5000F2FF3900000005002D
:101A6000889FBE000004BE00780090000020A00007
:101A700070049800E08F54000D003200030037001E
:101A800008007800B6FE07008904E900780090009D
:101A900065006000E50F500009003A00E08F540037
:101AA000F7FF3A000600370008007800ACFE070098
:101AB0007800900065006000E50F5000FAFF3200EA
:101AC000780090000020A100700498004F04BE0030
:101AD00000000600A01990000041EB00EF8F5100BC
:101AE00006003E006A814100020141000130790098
:101AF0008301E8002318980012C0B3000240780068
:101B000000000600010178008000EB0012003700A1
:101B10006A8240000402420060027A00820F520092
:101B20000C003A000301E900221898000600370073
:101B3000EA81400003824100EB8140008381410043
:101B4000633278008100E800828F5000F8FF39008E
:101B5000100005008100E800A0199000838F50005C
:101B6000EBFF3900000005008000EB002118980011
:101B7000000006000400FA0080089000E1BF9F000A
:101B8000F0009000F1BF9F004300200064815700E7
:101B9000A100290082C50200000000000080FA00B8
:101BA00000000600889FBE000004BE007800900080
:101BB0000020A00070049800E08F54001B00320049
:101BC000070037000800780094FF0700E00F50007E
:101BD0000E003A000800780061FE07008904E90061
:101BE0007800900065006000E50F500013003A0097
:101BF000E08F5400F3FF3A0010003700080078002F
:101C000086FF0700E00F50000600320078009000C9
:101C10000010A0007004980008007800D5FF0700AD
:101C200009003700080078004DFE0700780090009A
:101C300065006000E50F5000F0FF32007800900072
:101C40000020A100700498004F04BE0000000600B0
:101C5000F0019000618161000B003200E2816100BF
:101C60000001EB00828F510007003A00201990001C
:101C7000E00F510002003200CAFF070001003700E8
:101C800077FF070012002000020078000000060025
:101C9000889FBE00000478000800780020FE07003E
:101CA00080047800E08F5400130032007800900028
:101CB0006100600006003200700144002300200033
:101CC000810029000800780082C5020000000000A1
:101CD000090C98000080EB00100C9800F8009000B0
:101CE0000100A00071049800E28060000200320050
:101CF000080078009FFF0700090078004F04BE002D
:101D0000000006000400FA00881F78000004780034
:101D100000002A00808F500004003A00080078007C
:101D2000E6C50200000000007E00370012007800C7
:101D3000980F50007B003A000280E8000302E9009F
:101D4000F2FF2500F3FF2F0001014100E08149006F
:101D5000EE0F5100E08F590072003E00026001005A
:101D60000E0037001A003700210037002C00370022
:101D700031003700360037002C00370036003700BE
:101D80004200370045003700470037004C0037005D
:101D9000590037005C0037005F0037009001780081
:101DA0000402E9008000EB000700370003814000D7
:101DB00002014100280390008100E8008182400078
:101DC000E0827A0005337900848F5000F7FF3900F4
:101DD00020002000700498008080EB00080078004C
:101DE000ABFF0700E00F50004E003A000F00370035
:101DF000780090000010A10070049800080078009E
:101E00005CFF070080162800E00F500045003200FC
:101E100008007800688102000000000041003700DF
:101E2000780090000010A00070049800080078006E
:101E300050FF07003B003700780090006100600011
:101E40003800320008007800C5FD0700F7FF3700B2
:101E500020002000F4FF370090007800D1BF9F00E1
:101E6000080078001BFF07000080FB00E0BF9F0018
:101E70004300200066815700B10029000800780067
:101E800082C50200000000002600370090007800A4
:101E9000080078001BFF07002200370008007800C8
:101EA00031FF07001F0037001001900090007800FC
:101EB00008007800B0C502000000000019003700DB
:101EC000900178000402E9008000EB000700370071
:101ED0000381400002014100480390008100E800B6
:101EE00081824000E0827A0005337900848F5000BF
:101EF000F7FF39000B0037000800780018AB02002C
:101F0000000000000700370008007800DCAA02008B
:101F1000000000000300370008007800FCAA02005F
:101F2000000000004F0478000080FA000000060066
:101F300092007800E08F50000600350078FD070021
:101F400013002000E00F50000F0032008001EB0072
:101F50000D00370013002000F4FF2900848F50008B
:101F600009003600120190008001EB000402E80035
:101F7000848F500004003200900169000300EA00E1
:101F800083017000CF19DE00030078000000060016
:101F900090089000E0019000018140006301790009
:101FA0008100E90011089800020078000000060096
:101FB0000002EB0002712200A5002000811F7800C2
:101FC000110009000280D80080017800010078002B
:101FD000CF007800E08F510004003A00E00F52007B
:101FE00002003A00E10F510003003A0004C3B300BD
:101FF00084D8410014002000809FBE001100090019
:102000000581D800000178004F00BE00E00F5100AC
:10201000EAFF3A000100780000000600E4FF070034
:10202000E1C2B3000148780071C7B30001687800CD
:10203000F6C0500001687800F5C0400001687800E3
:102040008040EB001140980000000600889FBE0011
:102050008A1F780000047800C80490000800780007
:10206000CBFF070000004000E9047800480590001D
:1020700008007800C6FF070000004000EA00780072
:10208000EF8F540008003200E08F54000600350046
:1020900070022000808F540003003C00094078004B
:1020A0001AC10200000000004F0578004F04BE0076
:1020B000000006000E00FA00881F78008E007800ED
:1020C0000F0778000E01B10005000900001FEB00AA
:1020D000005FEB000107780001C7B30081F79F00A4
:1020E00040049000AAFF0700000040006804780048
:1020F00010002000128902000000000036D102000A
:10210000000000000000EB00E10F4400040032007A
:10211000EF80570008007800C0FF0700708057006C
:10212000D0D10200000000004F0478000080FA00C7
:10213000000006000E00FA00881F78008E0078006C
:102140000F0778000E01B10005000900001FEB0029
:10215000005FEB000107780021C7B30081F79F0003
:10216000400490008AFF07000000400068047800E7
:10217000E10F440003003A007AA7020000000000CB
:102180000900370010002000128902000000000042
:10219000EF80570008007800A0FF0700708057000C
:1021A0001AA70200000000004F0478000080FA0027
:1021B000000006000E00FA00881F78008E007800EC
:1021C0000F0778000E01B10005000900001FEB00A9
:1021D000005FEB000107780021C7B30081F79F0083
:1021E000400490006AFF0700000040006804780087
:1021F00010002000128902000000000036D1020009
:10220000000000000000EB00E10F44000400320079
:10221000EF8057000800780080FF070070805700AB
:10222000D0D10200000000004F0478000080FA00C6
:10223000000006000E00FA00881F78008E0078006B
:102240000F0778000E01B10005000900001FEB0028
:10225000005FEB000107780031C7B30081F79F00F2
:10226000400490004AFF0700000040006804780026
:1022700010002000128902000000000036D1020088
:102280000000000008007800EAD102000000000011
:1022900080007800E08F500006003200EF80570089
:1022A000080078005DFF070070805700D0D1020061
:1022B000000000004F0478000080FA0000000600D3
:1022C000E6874700889FBE008A9FBE008C9FBE00A5
:1022D0008E1F780000047800C80490000800780081
:1022E0002BFF070000004000E9047800480590003B
:1022F0000800780026FF0700000040006A0578000B
:10230000C80590000800780021FF07000000400089
:10231000EB05780048069000080078001CFF0700D5
:10232000000040006C067800C806900008007800A5
:1023300017FF070000004000ED06780048079000F6
:102340000800780012FF0700000040006E077800C8
:10235000C800900008007800F1B79F000CFF07004C
:1023600000004000FFB0970061037800C8009000B3
:1023700008007800F1B79F0086BF9F0004FF0700A8
:1023800000004000FFB097006104780000102000BA
:102390001289020000000000884378000FBB9700FC
:1023A0008E4278000D4278008C4178000B41780015
:1023B0008A407800094078000EC202000000000048
:1023C0004F0778004F06BE004F05BE004F04BE0009
:1023D0006F00B10000000600889FBE008A9FBE000B
:1023E00000047800C804900008007800E8FE0700A8
:1023F00000004000E90478004805900008007800DB
:10240000E3FE0700000040006A057800C805900060
:1024100008007800DEFE0700000040006B01780035
:102420008A407800094078005EC202000000000087
:102430004F05BE004F04BE0000000600889FBE008E
:102440008A9FBE0000047800C8049000080078004D
:10245000CFFE070000004000E90478004805900026
:1024600008007800CAFE0700000040006A057800F6
:10247000C805900008007800C5FE07000000400075
:102480006B0178008A407800094078007AC2020027
:10249000000000004F05BE004F04BE000000060013
:1024A000889FBE008A9FBE0000047800C804900088
:1024B00008007800B6FE070000004000E90478003C
:1024C0004805900008007800B1FE070000004000B9
:1024D0006A057800C805900008007800ACFE070087
:1024E000000040006B0178008A40780009407800C5
:1024F00096C20200000000004F05BE004F04BE005F
:1025000000000600889FBE008A9FBE008C1F7800D6
:1025100000047800C8049000080078009CFE0700C2
:1025200000004000E9057800C80490000800780029
:1025300097FE07000000400069057800C80490007D
:102540000800780092FE070000004000E9047800CF
:1025500048069000080078008DFE0700000040004B
:102560006C047800200020001289020000000000A6
:102570008B40780000C2B3001AC1020000000000C6
:102580008A40780030C2B3001AC102000000000087
:102590008940780010C2B3001AC102000000000098
:1025A0008840780020C2B3001AC102000000000079
:1025B0004F0678004F05BE004F04BE000000060025
:1025C000E6874700889FBE008A9FBE008C9FBE00A2
:1025D0008E1F780000047800C8049000080078007E
:1025E0006BFE070000004000E9007800C80490007E
:1025F0000800780081BF9F0065FE070000004000D2
:1026000069077800C80490000800780060FE0700A1
:1026100000004000E9067800C80490000800780037
:102620005BFE07000000400069067800C8049000C7
:102630000800780056FE070000004000E905780019
:10264000C80490000800780051FE07000000400018
:1026500069057800C8049000080078004CFE070067
:1026600000004000E904780048019000080078006C
:10267000F2B79F0046FE0700000040007FB19700C0
:10268000620478004000200012890200000000006F
:102690008FB8970000C1B3001AC10200000000000B
:1026A0008E40780010C1B3001AC102000000000083
:1026B0008D40780040C1B3001AC102000000000044
:1026C0008C40780050C1B3001AC102000000000025
:1026D0008B40780020C1B3001AC102000000000046
:1026E0008A40780030C1B3001AC102000000000027
:1026F000894078000040EB001AC102000000000091
:102700008840780010C0B3001AC102000000000029
:102710004F0778004F06BE004F05BE004F04BE00B5
:102720006F00B10000000600889FBE008A1F78007D
:1027300000047800C80490000800780014FE070028
:1027400000004000E9047800480590000800780087
:102750000FFE0700000040006A04780040002000DF
:1027600012890200000000008940780060C1B300B7
:102770001AC10200000000008840780070C1B30058
:102780001AC10200000000004F0578004F04BE008F
:1027900000000600881F780040049000FCFD070040
:1027A0000000400068047800000420001289020044
:1027B0000000000088407800D0C1B3001AC10200B8
:1027C000000000004F04780000000600881F780019
:1027D00040049000EEFD070000004000680478000F
:1027E00000012000128902000000000088407800EB
:1027F000E0C1B3001AC10200000000004F047800DD
:1028000000000600889FBE008A1F78000004780040
:10281000C804900008007800DDFD070000004000BB
:10282000E90478004805900008007800D8FD07000A
:10283000000040006A047800002020001289020095
:10284000000000008940780060C2B3001AC1020095
:10285000000000008840780070C2B3001AC1020076
:10286000000000004F0578004F04BE000000060085
:10287000889FBE008A1F780000047800C80490007A
:1028800008007800C2FD070000004000E90478005D
:102890004805900008007800BDFD070000004000DA
:1028A0006A04780010002000128902000000000075
:1028B00036D102000000000088007800090078008E
:1028C0000CD20200000000004F0578004F04BE004B
:1028D00000000600889FBE0000047800C804900035
:1028E00008007800AAFD07000000400000804400B6
:1028F0008000EB00F30F2000D2082000018240008E
:10290000040240000508200014824200830F520098
:10291000050036006181290008007800B48C0200AF
:1029200000000000050037008100E800828F5000A1
:10293000F2FF340002E50200000000004F04BE0078
:1029400000000600881F78004004900090FD0700FA
:102950000000400068007800E00F500003003200E3
:1029600096A502000000000002003700A0A50200AA
:10297000000000004F047800000006000E00FA007E
:10298000889FBE008A1F780000047800C804900069
:10299000080078007EFD070000004000690578000F
:1029A000080078007AFD0700800478000E007800A7
:1029B0000F0778004E01B10005000900001FEB0071
:1029C000005FEB000007780051C7B300C1EF9F0024
:1029D000E10F450008003A000000EB0070A802007B
:1029E00000000000480090008984440089044000F1
:1029F000800CEB0014003700F38057000A007800C9
:102A00006BFD0700E1C2B3000148780041C6B30086
:102A100001687800E3C0500001687800F3C040000E
:102A2000016878008040EB001140980089844400E0
:102A300048009000890440007480570070A802008C
:102A400000000000800C78004F0578004F04BE00A5
:102A50000080FA0000000600889FBE008A9FBE002A
:102A600000047800C80590000800780048FD0700C1
:102A7000800478000800780045FD07000005780014
:102A80000800780042FD0700800078000A05450034
:102A9000480090000A05400081804000898444007D
:102AA0000980450046A9020000000000000DD10089
:102AB0004F05BE004F04BE0000000600889FBE0008
:102AC0008A9FBE0000047800C805900008007800C6
:102AD0002FFD070080047800080078002CFD070017
:102AE000000578000800780029FD070080007800C4
:102AF0000A054500480090000A054000818040001A
:102B00008984440009804500FEA8020000000000FE
:102B1000000DD1004F05BE004F04BE0000000600AE
:102B2000889FBE0000047800C80490000800780068
:102B300017FD070000004000E90478000800780055
:102B400013FD070080007800818040004804900059
:102B5000010444006148B900000040008180480041
:102B6000BEA8020000000000000C78004F04BE0068
:102B700000000600889FBE000004EB00890E2000C4
:102B8000803E200020EB0200000000000804E80066
:102B9000890F5400FAFF36004F04BE000000060003
:102BA00001C2B30080C0B3001AC1020000000000DF
:102BB000F0FF07008040EB0080C0B3001AC10200A4
:102BC0000000000001C2B30090C0B3001AC10200AF
:102BD00000000000E7FF07008040EB0090C0B3005A
:102BE0001AC102000000000001C2B300A0C0B3007F
:102BF0001AC1020000000000DEFF07008040EB0069
:102C0000A0C0B3001AC102000000000001C2B3005E
:102C1000B0C0B3001AC1020000000000D5FF0700D9
:102C20008040EB00B0C0B3001AC1020000000000F9
:102C300001C2B300C0C0B3001AC10200000000000E
:102C4000CCFF07008040EB00C0C0B3001AC10200F7
:102C50000000000001C2B300D0C0B3001AC10200DE
:102C600000000000C3FF07008040EB00D0C0B300AD
:102C70001AC102000000000001C2B30020C0B3006E
:102C80001AC1020000000000BAFF07008040EB00FC
:102C900020C0B3001AC102000000000001C2B3004E
:102CA00030C0B3001AC1020000000000B1FF0700ED
:102CB0008040EB0030C0B3001AC1020000000000E9
:102CC00001C2B30040C0B3001AC1020000000000FE
:102CD000A8FF07008040EB0040C0B3001AC1040009
:102CE0000000000001C2B30020C2B3001AC10200FC
:102CF000000000009FFF07008040EB0020C2B300EF
:102D00001AC102000000000001C2B30001407800B7
:102D10001AC102000000000096FF07008040EB008F
:102D200000C2B3001AC102000000000001C2B300DB
:102D300030C2B3001AC10200000000008DFF07007E
:102D40008040EB0030C2B3001AC102000000000056
:102D500001C2B30010C2B3001AC10200000000009B
:102D600084FF07008040EB0010C2B3001AC10400CA
:102D70000000000001C2B300C0C1B3001AC10200CC
:102D8000000000007BFF07008040EB00C0C1B300E3
:102D90001AC102000000000001C2B30040C2B3002B
:102DA0001AC102000000000072FF07008040EB0023
:102DB00040C2B3001AC102000000000001C2B3000B
:102DC00050C2B3001AC102000000000069FF0700F2
:102DD0008040EB0050C2B3001AC1020000000000A6
:102DE00001C2B300F0C1B3001AC10200000000002C
:102DF00060FF07008040EB00F0C1B3001AC1020081
:102E00000000000001C2B30080C1B3001AC102007B
:102E10000000000057FF07008040EB0080C1B300B6
:102E20001AC102000000000001C2B30090C1B3004B
:102E30001AC10200000000004EFF07008040EB00B6
:102E400090C1B3001AC102000000000001C2B3002B
:102E5000A0C1B3001AC102000000000045FF070036
:102E60008040EB00A0C1B3001AC1020000000000C6
:102E700001C2B300B0C1B3001AC1020000000000DB
:102E80003CFF07008040EB00B0C1B3001AC1040052
:102E90000000000001C2B30000C1B3001AC102006B
:102EA0000000000033FF07008040EB0000C1B300CA
:102EB0001AC102000000000001C2B30010C1B3003B
:102EC0001AC10200000000002AFF07008040EB004A
:102ED00010C1B3001AC102000000000001C2B3001B
:102EE00040C1B3001AC102000000000021FF07002A
:102EF0008040EB0040C1B3001AC102000000000096
:102F000001C2B30050C1B3001AC1020000000000AA
:102F100018FF07008040EB0050C1B3001AC1020047
:102F20000000000001C2B30020C1B3001AC10200BA
:102F3000000000000FFF07008040EB0020C1B3003D
:102F40001AC102000000000001C2B30030C1B3008A
:102F50001AC102000000000006FF07008040EB00DD
:102F600030C1B3001AC10400000000008040EB0033
:102F700050C0B3001AC1020000000000C5FF0700E6
:102F800001C2B300D0C1B3001AC1020000000000AA
:102F9000F8FE07008040EB00D0C1B3001AC1020068
:102FA0000000000001C2B300E0C1B3001AC102007A
:102FB00000000000EFFE07008040EB00E0C1B3001E
:102FC0001AC102000000000001C2B30050C0B300EB
:102FD0001AC1020000000000E6FE07008040EB007E
:102FE00050C0B3001AC102000000000001C2B300CB
:102FF00060C0B3001AC1020000000000DDFE07003F
:103000008040EB0060C0B3001AC102000000000065
:1030100001C2B30070C0B3001AC10200000000007A
:10302000D4FE07008040EB0070C0B3001AC102005C
:10303000000000004FFF07002AFF070001C2B30095
:1030400060C2B3001AC1020000000000C9FE070000
:103050008040EB0060C2B3001AC102000000000013
:1030600001C2B30070C2B3001AC102000000000028
:10307000C0FE07008040EB0070C2B3001AC102001E
:103080000000000001C2B3000040EB001AC10200C2
:1030900000000000B7FE07008040EB000140780010
:1030A0001AC102000000000001C2B300E0C0B3007A
:1030B0001AC1020000000000AEFE07008040EB00D5
:1030C000E0C0B3001AC102000000000001C2B3005A
:1030D00010C0B3001AC1020000000000A5FE0700E6
:1030E0008040EB0010C0B3001AC1020000000000D5
:1030F00001C2B30060C1B3001AC1020000000000A9
:103100009CFE07008040EB0060C1B3001AC10200C2
:103110000000000001C2B30070C1B3001AC1020078
:103120000000000093FE07008040EB0070C1B30078
:103130001AC102000000000099FE37008BFF070053
:1031400001C2B30020C0B3001AC102000000000099
:1031500001C2B30000C1B3001AC1020000000000A8
:1031600001C2B30010C1B3001AC102000000000088
:1031700001C2B30040C1B3001AC102000000000048
:1031800001C2B30020C1B3001AC102000000000058
:1031900001C2B30030C1B3001AC102000000000038
:1031A00001C2B3000040EB001AC1020000000000A1
:1031B00001C2B30010C0B3001AC102000000000039
:1031C00001C2B300E0C1B3001AC102000000000058
:1031D00001C2B30070C2B3001AC1020000000000B7
:1031E00001C2B30080C1B3001AC102000000000098
:1031F00001C2B30090C1B3001AC102000000000078
:1032000001C2B300A0C1B3001AC102000000000057
:1032100001C2B300B0C1B3001AC102000000000037
:1032200001C2B300C0C1B3001AC102000000000017
:1032300001C2B30040C2B3001AC102000000000086
:1032400001C2B30050C2B3001AC102000000000066
:1032500001C2B300F0C1B3001AC1020000000000B7
:1032600001C2B300D0C1B3001AC1020000000000C7
:1032700001C2B30060C1B3001AC102000000000027
:1032800001C2B30070C1B3001AC102000000000007
:1032900001C2B30080C0B3001AC1020000000000E8
:1032A00001C2B300D0C0B3001AC102000000000088
:1032B00001C2B300E0C0B3001AC102000000000068
:1032C00000802000E48802000000000010002000C0
:1032D0009CD904000000000031468000910CB10030
:1032E000A0122000808F500005003E009A19A8000F
:1032F0008040EB00634050001AC102000000000053
:1033000080458000B208B400813E20000180B900F1
:10331000A2F82000811F7800110009004288D8001F
:10332000CF007800C018B10011022000810F5000BA
:1033300005003E008040EB00D0C0B3001AC102007F
:10334000000000009A39A800914380005138B10074
:10335000A0C12000808F500005003E008040EB009F
:1033600000C1B3001AC10200000000009A59A80071
:10337000A14380005138B100A0C12000808F5000CF
:1033800005003E008040EB0010C1B3001AC10200EE
:10339000000000009A79A800B14380005138B100C4
:1033A000A0C12000808F500005003E008040EB004F
:1033B00040C1B3001AC10200000000009A99A800A1
:1033C000C14380005138B100A0C12000808F50005F
:1033D00005003E008040EB0020C1B3001AC102008E
:1033E000000000009AB9A800D14380005138B10014
:1033F000A0C12000808F500005003E008040EB00FF
:1034000030C1B3001AC10200000000009AD9A80020
:10341000E14380005138B100A0C12000808F5000EE
:1034200005003E008040EB00014078001AC1020018
:10343000000000009AF9A800F14380005138B10063
:10344000A0C12000808F500005003E008040EB00AE
:1034500010C0B3001AC10200000000009B19A800B0
:10346000414580005106B100E0312000808F5000BE
:1034700005003E008040EB0060C1B3001AC10200AD
:10348000000000009B39A800514580005106B100A2
:10349000E0312000808F500005003E008040EB00AE
:1034A00070C1B3001AC10200000000009B59A800BF
:1034B00050468000E00F500003003A004046800074
:1034C000E00F5000050032008040EB00D0C1B30097
:1034D0001AC10200000000009B79A80080022000B1
:1034E00061468000808F50000C00340080468000D0
:1034F000810C2000810F500008003400B112200020
:10350000810F500005003C009B99A8008040EB0013
:10351000E0C1B3001AC10200000000009BB9A8007E
:103520008040EB00C0C1B3001AC1020000000000DF
:103530009BD9A8008040EB0050C2B3001AC1020022
:1035400000000000C0428000E00F50001100320077
:103550008040EB0090C1B3001AC1020000000000DF
:103560008040EB00B0C1B3001AC1020000000000AF
:103570008040EB0040C2B3001AC10200000000000E
:103580008040EB00F0C1B3001AC10200000000004F
:103590009BF9A800D0428000E00F500005003200E7
:1035A0008040EB0080C1B3001AC10200000000009F
:1035B0009C19A800E0428000E00F50000500320096
:1035C0008040EB00A0C1B3001AC10200000000005F
:1035D0009C39A800CEE6020000000000E00F500079
:1035E000050032008040EB00E0C0B3001AC10200C9
:1035F000000000009C59A800C008EC00E20F500039
:103600000B003E00C208EC00E20F500008003E0034
:1036100020468000F40F5000050034008040EB008D
:1036200080C0B3001AC10200000000009C79A8000D
:10363000F0FF2F00F1002000D2CC8000E3CC80000E
:10364000800F5100818F590008003A008040EB0044
:1036500020C0B3001AC102000000000001C2B30084
:1036600030C0B3001AC10200000000009E19EC0037
:10367000F0CC8800710C2000810F500002003E0049
:103680008100E8006145880072F32F0000014100CD
:10369000610C2000810F510002003E0081F32F00D9
:1036A00061458800F2E62F0000014100610C200016
:1036B000810F510003003E00AC28EF008180E8003C
:1036C0007145880072DA2F0000014100610C200072
:1036D000810F510002003E0081F32F0071458800E8
:1036E000F2CD2F0000014100E1182000810F5100B0
:1036F00002003E00AE28EF0000000600014B200053
:10370000810F500001003A009E39EF0000000600D2
:103710000080FB00401388006002AB00FEFF320017
:103720004013800000000600401F2000B0CC88003D
:1037300000C0EB00F6FF070000C0EB00F4FF07003D
:10374000E14F400003003200B1CC8000E08F500018
:10375000F9FF3A0000000600CDC2A80000C0EB004F
:10376000EBFF3700CDC2A900EFFF070011002000DA
:10377000E14F400002003200F7FF07008000EB003D
:103780000100780000000600CDC2A800C9C2A9004F
:10379000B0132000101388006422EF0061E2A8003B
:1037A00000000600EFFF0700EBFF0700C9C2A800FA
:1037B00061E2A900B619A80000000600889FBE00BB
:1037C000800478000104780040062000A0CC880026
:1037D00000C0EB00CEFF070080417800E1CF410040
:1037E00004003A00A2CC8000E00F5100F8FF3A003C
:1037F000220037000001EB00E2CF41001F003A0039
:10380000F20F2000421388006002AB00FEFF32007E
:1038100041138000090078000158780042138800A5
:103820006002AB00FEFF32004113800001587800B7
:10383000421388006002AB00FEFF3200411380009B
:1038400001587800421388006002AB00FEFF32008E
:1038500041138000014878006404540002003200E3
:103860008004E800E7FF370000C0EB00A8FF070076
:1038700000C0EB00A6FF0700120020000200780045
:103880004F04BE0000000600889FBE008A1F78001B
:103890008004780001447800A3FF07000001EB00DA
:1038A000E14F400019003A000840780098FF0700F7
:1038B00012002000E34F44001400320008202000D2
:1038C0000905E8001940780091FF07008984E800A5
:1038D0001A4078008EFF07000884E900F8FF3A00DC
:1038E00000C0EB008AFF070000C0EB0088FF070064
:1038F00000C0EB0086FF07007F0060001200200080
:10390000E50F500001003200080178000200780045
:103910004F0578004F04BE0000000600889FBE00DF
:103920008A1F7800004578000204BE00E04F550071
:1039300006003D006011B80070C3B300F7FF070038
:10394000E14F50002A003E000A74A10082FF0700E8
:1039500084FF07008000780000C0EB00E08F50007B
:10396000230032000A4078000064A00068FF0700CE
:103970004848DE000100200065FF07004048DE00E7
:103980000100200062FF07004849DD004840DE00DA
:1039900000007100C848DE005DFF070008407800A5
:1039A0005BFF070050C9B300E04F55000400320030
:1039B0006E405000E84F55000100320010C0B300C7
:1039C00053FF0700EC4F550002003A0000C0EB0027
:1039D0004FFF0700A8C0B30000C0EB004CFF07007A
:1039E000E04F500002003D000844E900FAFF3A00B1
:1039F0004F0578004F04BE00000006000400FA00E6
:103A0000889FBE008A1F78008040780010C0B300F5
:103A1000E0CF500088003A005116800000002400DA
:103A2000008060008300320057FF070061E2A900B8
:103A30001113800030FE2F00008060004001B300B1
:103A40001013880011138000C0FF2F000080600059
:103A50000000A0001013880061E2A800A9C0B30014
:103A600000C0EB002AFF07008944E900FCFF3A0090
:103A70006011B80009407800A8FF070000457800F1
:103A800009447800E14F550059003A00803E20007B
:103A9000A0CC8800A21A20000300200080C0B30040
:103AA0009EFF0700E14F500033003A0000C0EB00DA
:103AB00017FF07008880FB00804178006A8157006B
:103AC00003F178000844E800E34F5400F7FF3600A4
:103AD0000044EB000FF89700E14F500044003A001B
:103AE000A0CAB3009FF8970080CF500040003A0072
:103AF000A0CC8000E00F5000060032000200200041
:103B00000300240090CAB30084FF0700E04F500078
:103B1000F7FF3A00A8CC8000E00F540034003200D8
:103B20006011B800A0C3B3007CFF07000044EB00A5
:103B3000884F50002E003A0000C0EB00F4FE070052
:103B40008980FB00804178006A81570003F178008A
:103B50008944E800E3CF5400F7FF3600EFF0970008
:103B60000180FB000004B20048C0B3002000320016
:103B7000C8C0B3001E0037006011B80090CAB3007F
:103B800066FF070028C0B30099CAB300E14F500098
:103B9000020036000A44780088447800A0CC8000F7
:103BA000E00F5000050032006011B80009407800B5
:103BB0005AFF0700E04F5000F8FF3A00A0CC800009
:103BC000E00F500007003200022020000300200018
:103BD00000C1B30051FF0700E04F500003003A005E
:103BE0000300370000447800010037000044EB0078
:103BF0000880FB00C0CC8800D7FE0700E04F5400CF
:103C00000B003200B619A90061E2A900111380006F
:103C100030FE2F00008060008001B3001013880088
:103C2000300020006222B70061E2A80001003700E6
:103C3000DCFE0700B6D9BF004F0578004F04BE0078
:103C40000080FA00000006008040780010C0B30039
:103C5000E0CF500001003A00B6D9BF0000000600D6
:103C6000889FBE008A1F7800810478000444780091
:103C700044002000E04F50002F003A00E04F540075
:103C80002D003200B6D9BF00610060003400200072
:103C900029003A009879AB0004003A004918DD0089
:103CA000C711DE00830170004911DD00E14F5400AF
:103CB0000B003A0010C1B30018FF07000045780060
:103CC000E04F550018003A0001202000090078005C
:103CD000BAFE0700E00F500012003A001200370051
:103CE00020C1B3000DFF0700E04F50000E003A0066
:103CF0000120200009007800B0FE0700E00F50000E
:103D0000040032000844E900020032000920B0003B
:103D1000F7FF37006011B800C0C0B300FFFE070016
:103D2000010037000A4478008BFE07000882FB0080
:103D30000402EA004F22DE00040078004F057800FC
:103D40004F04BE0000000600889FBE008A9FBE0090
:103D5000810578000204BE0004457800420020007E
:103D6000E04F500040003A00E04F55003E00320066
:103D7000B6D9BF0061006000320020003A003A006E
:103D8000B6D9BF00640060002200200036003A006F
:103D9000C0CC8000E800600004003A00C948DD00A3
:103DA000C744DE00898470004944DD00E14F5500BE
:103DB0000C003A000801BE0080C1B300D7FE070026
:103DC00000447800E04F540023003A00E1CFB300F4
:103DD0000B007800ACFE0700E00F50001B003A001B
:103DE0001D00370066006000040032000A81FB00FD
:103DF0000300200070C9B300C8FE07000801BE0020
:103E000090C1B300C5FE0700E04F500012003A0019
:103E1000C1CFB3000B0078009BFE0700E00F5000FD
:103E2000040032000A45E900020032000B20B00015
:103E3000F7FF3700D1CFB3000000EB0092FE070080
:103E4000E00F5000030032000300370008457800FF
:103E5000010037001AC0B3003FFE07000A81FB00D3
:103E60000201EA004F11DE00020078004F05BE009B
:103E70004F04BE00000006001000FA00889FBE003C
:103E80008A9FBE008041780001407800820478005B
:103E900048002000E0CF5100D4003A00619B21008F
:103EA00091407800E180600038002000CF003A00A7
:103EB0000080FB0001002000EE0F5000E08F580052
:103EC000C8003E00006001000E00370013003700FC
:103ED000480037004A003700C2003700C1003700F1
:103EE000C0003700BF003700BE003700BD003700FC
:103EF0008E00370091003700930037009A0037009A
:103F0000A800370017FE070018002000E00F50003F
:103F1000B500320010FE0700860037006011B800BF
:103F200090C0B3007DFE070018002000E04F500055
:103F3000AD003A0001012000788057001FFE070005
:103F4000E00F5000A80032000FE897008080FB00CF
:103F5000C608DE000FF09700E1CF50000B003A00DA
:103F60001FF197000281FB00080141004800DD00BD
:103F700000014100030020004A18DD00C610DE00E9
:103F8000810070004A10DD003C0037000080FB001B
:103F90004600DE00FFE897008180FB00C208DD00DC
:103FA000010040000000E800EFE89700E3806000B7
:103FB000CA08DD0001004000010020005FEA970010
:103FC0006F426200AFF197008381FB00C719DE00EA
:103FD0008341420083C1E8001FF197006341610003
:103FE0000241410002C141000281FB006901510010
:103FF0001D00370000202000800C78004D003700A5
:10400000CBCC8000648565001E0032006011B800D2
:10401000D0C8B30041FE070018002000E04F500058
:1040200071003A0000C0EB00B9FD0700010120005B
:1040300078805700E1FD0700E00F50006A00320071
:1040400008C3B30000C0EB00B1FD07000844E9005D
:10405000FCFF3A002FF197000281FB004411DE00C3
:1040600000012000010020000201E90003003300EC
:104070000000400081804800FBFF3700808CBE00BC
:104080002C0037006011B80090C0B30023FE070079
:1040900018002000E04F500053003A0001012000BA
:1040A00078805700C5FD0700E00F50004E00320039
:1040B000628465002FF19700BFF097000F00320077
:1040C0000180FB004700DE000000E800F203B200C0
:1040D0000201410002004000DFF197008381FB00F4
:1040E000C619DE008301E9000300DD0001002000A5
:1040F000808CBE000A0478003B0037008180FB0002
:104100004508DE000000E800E3806000C308DD0031
:1041100001004000C207B2004291DE000201E80047
:104120000280B900808CBE002F00370088992100E2
:10413000984C78000004EB002B0037006011B800A9
:1041400090C0B300020037006011B800A0C0B300F7
:10415000F2FD07001800200001012000E04F500090
:1041600021003A00180037006011B800A0C3B30066
:10417000EAFD070018002000E04F50001A003A0046
:104180000044780000C0EB0061FD07008880FB0060
:1041900080F478000844E800E34F5400F9FF36004B
:1041A000E4FF37006011B800D0C8B300DBFD0700A2
:1041B00018002000E04F50000B003A0000C0EB0058
:1041C00053FD070001042000090078007BFD070073
:1041D0000004EB00880F500003003A001800200094
:1041E00001003700480020005BFD07000800780050
:1041F0004F05BE004F04BE000080FA00000006001C
:10420000A0CC8000E00F5000020032000000E90066
:10421000A0CC8800B0CC8000E00F5000020032003B
:104220000000E900B0CC8800000006004300DD007B
:1042300001142000610078004300DE00610060008E
:10424000000006004300DD004114200061007800FA
:10425000000006000102E80004024200255521008A
:1042600065037A00FD015000E2742100868F510041
:104270000D003C00E2C178008341E80003F17800C2
:10428000E3CF51000A003600860F500006003D00C3
:1042900080327A0012C0B3000001FD003DF7B70084
:1042A0000001FD00020037008041EB0003F17800BF
:1042B0008100E8008180400022552100E2807800E2
:1042C000F2FF2700828F50000500320002322000EA
:1042D000000141006308B9004200DE000000510007
:1042E000E00F500001003D000000EB000000060060
:1042F000E00F5000070035000101E8000201410015
:104300002355210063017900E00F510002003400C1
:10431000D0FF37000000EB00000006000021EF0096
:10432000E00F50000A00350081802000810F50000E
:1043300001003600010078007C00B90052B5210070
:10434000000041001008880020C0B30002003700C0
:1043500002A1EF0010C0B3003FF7B7003E77EF00B7
:1043600042C1A9004AC1A90052C1A9005AC1A9006D
:1043700062C1A9006AC1A90072C1A90080FF2F0013
:10438000610E8000008060005000B300600E880065
:10439000B00E880005E1A80000000600881F780024
:1043A0000004EB000200370008007800A5FF0700BA
:1043B000080078009DFF0700E00F5000FAFF3A0068
:1043C0005175210080707C000804E800E60F54005D
:1043D000F7FF34004F04780000000600889FBE00FD
:1043E0008A9FBE008C1F78000004780001067800C8
:1043F000080078008DFF0700E00F500059003200E0
:104400005975210069457C000A40780072C0B300EC
:104410000440BC00880541000800780089FF0700BF
:10442000037621000B8145008031790084792100D9
:104430000C3279008A40E80081747C000000EB00B7
:10444000E4CF500047003A00F5004400818040006E
:1044500008014400E4837800E40279008583530076
:10446000E702440046022000868F53000C0036000D
:104470008582420065B1790065317A006E014400A1
:1044800002014100E2B27900E2327A0061B17900C2
:1044900061317A0031C0B30081747C003100370093
:1044A00085824200E3827A00630279006E01440053
:1044B000020141006301790004015100E3807800AA
:1044C0008580500082805000F38F4000220035002C
:1044D000F38F500020003C000482520083A82F007C
:1044E00083014200F15D2100818F51001A003E00DE
:1044F000614B2E0081004100C3012000801F780025
:10450000110009008380D800800078004F007800F7
:10451000854A2E00850241007C09B90002815200C3
:10452000E20F41000C003500E20F51000A003C0090
:1045300072042000080141000080200002014100B7
:10454000043079000204200008014100020141000A
:1045500001307900100020008040EB0052752100EE
:1045600001717C004F0678004F05BE004F04BE006D
:1045700000000600889FBE008A1F780000057800B2
:104580000004EB00880478008A00780009007800B5
:1045900092FF07000900DD00000474008904E800B0
:1045A000E68F5400F8FF3400E00F54000C00320096
:1045B00020C0B3005CF7B700E7FF2F00012D2000FB
:1045C000810F55000E003E0027002000F10420005E
:1045D000810F55000A0036008003EB000800370009
:1045E000C17521009140780088037800E0CF500029
:1045F000030032008140E900010078005CF7B70059
:10460000080078005E17B70000047800F8BA880048
:10461000C175210091407800E0CF500022003A009F
:10462000E00F5400200032008804CF000901E900A7
:10463000820078001500200010003700730420006D
:104640008281410003834100038020007404200024
:10465000010242000402420063037B00E3017A008E
:10466000830F530004003D008129DD008881610033
:1046700001003200010178008100E800E68F50005F
:10468000EEFF34000204B00002014100018020006E
:10469000E1007900E14488000208200081CD20007B
:1046A000910871005E37EF00070078004F05780031
:1046B0004F04BE0000000600889FBE008A9FBE0017
:1046C0008C9FBE008E1F78000005EB000A04780066
:1046D000FE7C20004D0620009B03200088854500BD
:1046E0008B854500008020008B054000800DEB008D
:1046F000080044000C74210000064600000EEB0088
:1047000008007800C9FE0700E00F500022003200C8
:1047100008007800CBFE07008004780008007800CD
:10472000C2FE0700E00F50001B00320008007800B6
:10473000C4FE0700090E78008E8F54000F003C0065
:104740008D8F540005003400090050008800780067
:10475000E7FE0700800D78000F00370036DD02000D
:1047600000000000E00F50000B003A006385640079
:104770006555B9006A0555000700370036DD0200AF
:1047800000000000E00F500003003A006385640061
:104790000A05E9006555B9009003200008004000B3
:1047A000000040000180200061007800E00F500010
:1047B00002003A00E174210080707C000804E800E7
:1047C000E60F5400C4FF34000A0078004F07780059
:1047D0004F06BE004F05BE004F04BE00000006009D
:1047E000889FBE008A9FBE001B0880008004EB00EB
:1047F00009047800FC854500080078008BFE07005E
:10480000E00F500012003200080078008DFE070013
:104810000005780008004400017421006100780060
:10482000008045008A0F50000900310036DD02008B
:104830000000000080007800E08F500004003A0083
:10484000630065000000E9006500B900800478009D
:104850000804E800E60F5400E7FF34000900780080
:104860004F05BE004F04BE0000000600801F780008
:104870008980A900200020003F77ED0006003A0063
:1048800005E1A90080FF2F00CC21B600D621B6009B
:104890003E77EC0010002000A91A07004F007800B6
:1048A00000400600889FBE0080047800E58F540019
:1048B0000F00320010003E000004EB00E08F5400B7
:1048C00025003A00B5FE07003CD7BF0004003200C7
:1048D00020C0B3003CF7B700F0448000010037006F
:1048E0000080EB008DFE0700090478001A003700F5
:1048F00071FF0700130037000004EB003CD7BF0036
:10490000E24F500014003A00E1732100914078001A
:10491000E0CF500010003200E6CF500005003A0012
:10492000AFFF0700000478009CFE07003E77EC0014
:1049300009003700E6CF5000040036000900780077
:104940000CFF070000047800030037008140E800F6
:10495000010078003EF7B7003CD7BF00E24F50009F
:10496000010032000004EB00080078004F04BE0094
:1049700000000600881F7800000478009AEB02000F
:10498000000000008000EB0022552100F0FF27000E
:104990008100E8008181400062827900E00F5200CE
:1049A00001003A0000B17900E68F5000F8FF3400B2
:1049B00042E1A800120A800001FE2F0001016100FF
:1049C0007200B300120A880041A1A90000C02100B2
:1049D0004021B700020A800083FF2F00030161001D
:1049E0000200A000020A88004201F8004A01F90012
:1049F0004001F8004801F9004201F8005201F900B5
:104A00004001F8005001F9004201F8005A01F90094
:104A10004001F8005801F9004201F8006201F90074
:104A20004001F8006001F9004201F8006A01F90054
:104A3000520B8000010161000230A000520B88007F
:104A40004001F8006801F9006A01F8007201F900FC
:104A50006801F8007001F900CC21EF00CE21EF00D1
:104A6000CC21B700700E800081006000B100B3005F
:104A7000710E880040002000900E8800900E80008B
:104A8000003CB000800E8800CC01F800D601F9008F
:104A9000CE01F800D801F900D001F800DC01F900DE
:104AA000E00E8000003CB000D00E8800670064007B
:104AB000D10580008381600080817100D30588006A
:104AC0008980A9009980A8004F04780000000600A2
:104AD000CC21EF00D621EF004021EF004821EF006C
:104AE0005021EF005821EF006021EF006821EF0016
:104AF0007021EF009980A90005E1A900A4EB020054
:104B0000000000003DD7BF0007003200F028200061
:104B100081458000808F5000030034000000EB00CE
:104B2000A6A9020000000000000006003CD7BF005C
:104B300002003A0010C0B3003CF7B70000000600C6
:104B40003C77EF00000006007E39EF0020002000D7
:104B5000708902000000000080748100E00F5000A6
:104B60000D00320002CC800013CC8000E00F510019
:104B7000E08F59000300320000E922000EE202003B
:104B8000000000008039EF008239EF0000E92200C8
:104B9000FC4B020000000000000006000200FA00CA
:104BA000881F780000047800E48157000208200084
:104BB0008800780000C72200F647020000000000CD
